:0300000002D042E9
:0CD04200787FE4F6D8FD75817102A6C766
:0DCC7B009068E6EEF0A3EFF09068E8EDF0B1
:10CC8800A2AF9200C2AF9068E6E0FEA3E0FFEEFF1D
:10CC98007E008FE39068E6E0FEA3E0FF8FE475E591
:10CCA800029068E8E0FF8FE243E78075E64675E6A4
:0CCCB800B90075E60053E780A20092AFBF
:01CCC400224D
:08002600906922EEF0A3EFF057
:10002E00A2AF9201C2AF906922E0FEA3E0FFEEFF05
:10003E007E008FE375E40075E50343E78075E646C1
:0E004E0075E6B90075E60053E780A20192AF97
:01005C002281
:08CE0F00906924EEF0A3EFF09E
:10CE1700A2AF9202C2AF906924E0FEA3E0FFEEFF4B
:10CE27007E008FE3906924E0FEA3E0FF8FE475E5C1
:10CE37000143E78375E64675E6B90075E60053E7F3
:07CE470080A20292AFAFE2EE
:01CE4E0022C1
:10CA0600906895EFF0906896EBF0A3EAF0A3E9F052
:10CA1600754E01906895E0FFE54ED39F50369068BD
:10CA260099E0FEA3E0FF12CE0F906896E0FBA3E02C
:10CA3600FAA3E0F9EF128E5590689AE004F07006BA
:10CA4600906899E004F0906897E475F001128EF012
:04CA5600054E80BF4A
:01CA5A0022B9
:10C6F00090689BEFF090689CECF0A3EDF090689E42
:08C70000EBF0A3EAF0A3E9F05D
:10C7080090689CE0FEA3E0FF120026754F01906838
:10C718009BE0FFE54FD39F503690689CE0FEA3E076
:10C72800FF90689EE0FBA3E0FAA3E0F9128E0FFDEC
:10C7380012CC7B90689DE004F0700690689CE00441
:0FC74800F090689FE475F001128EF0054F80BFEE
:01C7570022BF
:10C44D00906715E0FFEF702A9067157401F0906604
:10C45D009074F0F0A3E4F07B017A66799290669087
:10C46D00E0FEA3E0FF906899EEF0A3EFF07F80125D
:10C47D00CA06906692E0FFEF70047F0180027F0094
:10C48D00EF30E706906712E4F0229067127401F026
:10C49D007B017A6679927F8012BFA9EF7007906752
:10C4AD00167401F022906716E4F090671FE4F09087
:08C4BD006720E4F0128A2A2234
:108A2A00906692E0FFEFB4810D9067137401F090A5
:108A3A006714E4F08021906692E0FFEFB4820E9012
:108A4A0067137401F09067147401F0800A90671339
:108A5A00E4F0906714E4F0906693E0FF905E03EF11
:108A6A00F0906694E0FF905E04EFF0906695E0FF68
:108A7A00905E05EFF0906696E0FF905E06EFF0904C
:108A8A006697E0FF905E07EFF0906698E0FF905ED1
:108A9A0008EFF0906699E0FF905E09EFF090669A11
:108AAA00E0FF905E0AEFF090669BE0FF905E0BEFAE
:108ABA00F090669CE0FF905E0CEFF090669DE0FF00
:108ACA00905E0DEFF090669EE0FF905E0EEFF090E4
:108ADA00669FE0FF905E0FEFF09066A0E0FF905E69
:108AEA0010EFF09066DDE0FF9056A1EFF09056A1EE
:108AFA00E0FFEF5407FF9050DCEFF09056A1E0FF43
:108B0A00EF5470FFEFC4540FFF9050DDEFF0905612
:108B1A00A1E0FFEF5408FF9067E1EFF09056A1E063
:108B2A00FFEF5480FF9067E2EFF09066DEE0FF907F
:108B3A000C5FEFF09066F8E0FF9050F7EFF0906668
:108B4A00A2E0FFEF540FFF9067E5EFF09066A2E016
:108B5A00FFEF54F0FF9067E6EFF09066A3E0FFEFB7
:108B6A00540FFF9067DCEFF09066A3E0FFEF54F03C
:108B7A00FF9067DDEFF09066A5E0FF9067E8EFF001
:108B8A009066A4E0FF9067E7EFF09066DBE0FFEF06
:108B9A00540FFF9067DEEFF09066DBE0FFEF54F0D2
:108BAA00FF9067DFEFF09066DCE0FF9060E3EFF0A4
:108BBA009066DFE0FF900C55EFF09066E0E0FF90E2
:108BCA000CA5EFF09066E1E0FF905933EFF0906664
:108BDA00E2E0FF90098FEFF09066E3E0FF9050B477
:108BEA00EFF09066E4E0FF900006EFF09066E5E0B3
:108BFA00FF9056ECEFF09066E6E0FF900C97EFF0EE
:108C0A009066E7E0FF9050EEEFF09066E8E0FF90A4
:108C1A005530EFF09066E9E0FF905528EFF0906646
:108C2A00EAE0FF900C91EFF09066EBE0FF900C9673
:108C3A00EFF09066ECE0FF9056AEEFF09066EDE054
:108C4A00FF900CA4EFF09066EEE0FF900003EFF0C7
:108C5A009066EFE0FF900AAEEFF09066F0E0FF90CA
:108C6A005902EFF09066F1E0FF900AA2EFF09066E9
:108C7A00F2E0FF9056B9EFF09066F3E0FF900AA198
:108C8A00EFF09066F4E0FF900AA5EFF09066F5E049
:108C9A00FF9058FFEFF09066F7E0FF9067E4EFF07F
:108CAA009066F6E0FF9067E3EFF0906706E0FF90CA
:108CBA000C4DEFF0906707E0FF900C50EFF09067D3
:108CCA0008E0FF900C51EFF0906709E0FF900C5418
:108CDA00EFF090670AE0FF900C58EFF090670BE016
:108CEA00FF900C5DEFF090670CE0FF900C5EEFF0E8
:108CFA0090670DE0FF900C60EFF090670EE0FF9038
:0F8D0A000C79EFF090670FE0FF9050D9EFF02257
:1098F30090687274F2F0A3E4F0755200E552C394D9
:10990300024003029AB8AF527E007C047DB3128EEC
:1099130089740A2FF974453EFA7B01906874EBF061
:10992300A3EAF0A3E9F0755000E550C394645074C2
:1099330012D009AF507E0CEF8EF0A4FFAEF090680A
:1099430074E0FBA3E0FAA3E0F9E92FF9EA3EFAAEEB
:1099530002AF01906877EEF0A3EFF0906877E0FE36
:10996300A3E0FF8E538F54755100E551C3940C50FF
:109973002F906872E0FEA3E0FF12CE0FAC53AD54FC
:109983008D828C83EFF0906873E004F0700690682A
:1099930072E004F00554E55470020553055180CA82
:1099A30005508085906872E0FEA3E0FF12CE0F9011
:1099B3006874E0FBA3E0FAA3E0F97582B075830451
:1099C300EF128E67906873E004F07006906872E09F
:1099D30004F0906872E0FEA3E0FF12CE0F9068746B
:1099E300E0FBA3E0FAA3E0F97582B1758304EF12FB
:1099F3008E67906873E004F07006906872E004F07C
:109A0300906872E0FEA3E0FF12CE0F906874E0FB53
:109A1300A3E0FAA3E0F97582B2758304EF128E67AF
:109A2300906874E0FBA3E0FAA3E0F97582B0758354
:109A330004128E28FFEFD394644015906874E0FB02
:109A4300A3E0FAA3E0F97582B0758304E4128E678C
:109A5300906874E0FBA3E0FAA3E0F97582B1758323
:109A630004128E28FFEFD394644015906874E0FBD2
:109A7300A3E0FAA3E0F97582B1758304E4128E675B
:109A8300906874E0FBA3E0FAA3E0F97582B27583F2
:109A930004128E28FFEFD394024015906874E0FB04
:109AA300A3E0FAA3E0F97582B2758304E4128E672A
:059AB30005520298FFBE
:019AB800228B
:10915F0090687974F2F0A3E4F0755500E555C39467
:10916F0005501D906879E0FEA3E0FF12002690687D
:10917F007AE02400F0906879E03402F0055580DC45
:10918F0090687974F2F0A3E4F0755700E557C39433
:10919F00024003029354AF577E007C047DB3128EBE
:1091AF0089740A2FF974453EFA7B0190687BEBF0C6
:1091BF00A3EAF0A3E9F0755500E555C39464507424
:1091CF0012D009AF557E0CEF8EF0A4FFAEF0906871
:1091DF007BE0FBA3E0FAA3E0F9E92FF9EA3EFAAE50
:1091EF0002AF0190687EEEF0A3EFF090687EE0FE94
:1091FF00A3E0FF8E588F59755600E556C3940C5057
:10920F002F906879E0FEA3E0FFAC58AD598D828CAA
:10921F0083E0FD12CC7B90687AE004F070069068D2
:10922F0079E004F00559E55970020558055680CAD2
:10923F000555808590687BE0FBA3E0FAA3E0F97504
:10924F0082B0758304128E28FFEFD394644015907B
:10925F00687BE0FBA3E0FAA3E0F97582B0758304A5
:10926F00E4128E6790687BE0FBA3E0FAA3E0F97548
:10927F0082B1758304128E28FFEFD394644015904A
:10928F00687BE0FBA3E0FAA3E0F97582B175830474
:10929F00E4128E6790687BE0FBA3E0FAA3E0F97518
:1092AF0082B2758304128E28FFEFD394024015907B
:1092BF00687BE0FBA3E0FAA3E0F97582B275830443
:1092CF00E4128E67906879E0FEA3E0FF90687BE080
:1092DF00FBA3E0FAA3E0F97582B0758304128E2820
:1092EF00FD12CC7B90687AE004F07006906879E00C
:1092FF0004F0906879E0FEA3E0FF90687BE0FBA3A9
:10930F00E0FAA3E0F97582B1758304128E28FD127D
:10931F00CC7B90687AE004F07006906879E004F0F6
:10932F00906879E0FEA3E0FF90687BE0FBA3E0FA92
:10933F00A3E0F97582B2758304128E28FD12CC7BDF
:05934F00055702919B8F
:0193540022F6
:10A6C700756100438E2212CEC412CEF512C44D120C
:10A6D700CF8012AE7412CFAB906712E0FFEF600825
:10A6E700906716E0FFEF601E12D0091295411269BC
:10A6F7005C12C44D12CE8DC29012BDD012CF54AF92
:10A707006112474D80D212D00912701C12695C1277
:10A717009541906717E0FFEFB4010A12915F9067C8
:10A7270017E4F08011906717E0FFEFB40208129862
:10A73700F3906717E4F0906792E0FFEF700302A7CA
:10A74700C7906792E4F0906789E0FFEF70359067F4
:10A7570013E0FFEF602D7B017A4E79B47F00125D25
:10A76700B67B017A4E79B47F0012AFB97B017A4E7E
:10A7770079B47F001200667F0012BAE17F00127B76
:10A7870058803D906789E0FFEF64FF70339067144E
:10A79700E0FFEF602B7B017A4F79B47F01125DB642
:10A7A7007B017A4F79B47F0112AFB97B017A4F7978
:10A7B700B47F011200667F0112BAE17F01127B5854
:10A7C70090679FE0FFEF700302A6DF90679FE4F0BA
:10A7D70012BDD012CF5490679CE0FFEF70109067C6
:10A7E70013E0FFEF60087F0012474D02A6DF906776
:10A7F7009CE0FFEF64FF600302A6DF906714E0FFB1
:0EA80700EF700302A6DF7F0112474D02A6DFAD
:01A815002220
:10CFAB009067E0740DF09067E0E0FF8FE19067E031
:10CFBB00E0FFEF4420FF9067E0EFF09067E0E0FFC9
:03CFCB008FE122D1
:10D009009067E0E0FFEF4410FF9067E0EFF0906772
:06D01900E0E0FF8FE122C0
:10CF8000758921758C7D758ACBC2B975B81043B788
:10CF900010D28CD2A9D2AC43AD1075AF1012D01FF5
:0BCFA00012CE8DC29012D035D2AF220D
:10CEC4007E007F008E648F65756280756300E56304
:10CED4004562601CAE64AF658F828E83E4F00565A5
:10CEE400E56570020564E56315637002156280DE12
:01CEF400221B
:10AE7400756600E566C39402400302AF1CAF6674B6
:10AE8400812FF582E4340CF5837401F0AF667EAD56
:10AE9400EF8EF0A4FFAEF0743F2FF974553EFA7BA9
:10AEA4000112CB04AF667E7BEF8EF0A4FFAEF0748C
:10AEB400942FF974093EFA7B0112CB4FAF667E00E2
:10AEC4007C047DB3128E89740B2FF974003EFA7BD7
:10AED4000112CB9AAF667ECBEF8EF0A4FFAEF07476
:10AEE400B32FF9740A3EFA7B0112CBE5AF667E00FC
:10AEF4007C1C7D23128E8974B82FF9740C3EFA7B66
:10AF04000112CC30AF6674FF2FF582E4345DF58313
:10AF14007401F0056602AE779066717401F0905D7D
:10AF2400FE7401F090674E7401F090674F7401F065
:10AF340090671D7401F090671E7401F0906744746B
:10AF440001F09067457401F090672BE4F090672C52
:10AF5400E4F0906750E4F0906718E4F090674CE4F4
:10AF6400F090674DE4F09067D47457F09067D5740F
:10AF74004DF09067D67445F09067D77453F090679E
:10AF8400D87441F09067D97432F09067DA7452F053
:10AF94009067DB7435F0905944E4F0905945E4F03F
:10AFA400905946E4F0905947E4F0905948E4F09001
:04AFB4005949E4F023
:01AFB8002276
:10D01F00759102759200438E4043C58053C59F534F
:06D02F00C5F843C5012213
:10CFCE0043C508E5C520E408906927E5BEF080F367
:10CFDE00906926E5C6F053C5EF906926E0FEA3E002
:01CFEE00FF43
:01CFEF00221F
:10000E0012C26012BF0F12BA1812A57612B4742261
:10B0EC00753C0112CFCE906731E0FDED25E02423B5
:10B0FC00F8A60608A607906731E0FFEF640460032A
:10B10C0002B216753B00E53BC39405501EAF3BEFF6
:10B11C0025E02423F8E6FE08E6FFAD3BED25E02410
:10B12C002DF8A60608A607053B80DB753A00E53A24
:10B13C00C39404506E753900C37404953AFFE53915
:10B14C00C39F505BAF39EF25E02425F8E6FE08E6F7
:10B15C00FFAD39ED25E02423F8E6FC08E6FDD3ED40
:10B16C009FEC9E4036AF39EF25E02423F8E6F53707
:10B17C0008E6F538AF39EF25E02425F8E6FE08E6B9
:10B18C00FFAD39ED25E02423F8A60608A607AF3954
:10B19C00EF25E02425F8A63708A63805398099054F
:10B1AC003A808B8527218528229067E7E0FEA3E073
:10B1BC00FFC3E5229FE5219E50089055297401F0AC
:10B1CC0080169067E3E0FEA3E0FFD3E5229FE52124
:10B1DC009E4005905529E4F0753C01E53CC394056F
:10B1EC00501EAF3CEF25E0242DF8E6FE08E6FFAD3F
:10B1FC003CED25E02421F8A60608A607053C80DBDB
:10B20C00E53C24FEFF906731EFF0906731E004F0ED
:01B21C00220F
:10C26000309426904EAEE004F09058FFE0FF904EE0
:10C27000AEE0FEEEC39F40279058FBE4F09058FFDD
:10C28000E0FF904EAEEFF08016904EAEE0FFEF7004
:10C29000089058FB7401F08006904EAEE014F03028
:10C2A0009525904EAFE004F09058FFE0FF904EAF20
:10C2B000E0FEEEC39F40259058FCE4F09058FFE06C
:10C2C000FF904EAFEFF022904EAFE0FFEF7007907F
:0DC2D00058FC7401F022904EAFE014F022F3
:10BF0F0020B541906726E0FFEF6039906726E01477
:10BF1F00F0906726E0FFEF70349067E2E0FFEF608C
:10BF2F000C90671CE0FFEF70047F0180027F009090
:10BF3F005932EFF090671CE0FFEF701190672A7491
:10BF4F0001F0800930B506906726740AF020B340DF
:10BF5F00906725E0FFEF6038906725E014F0906759
:10BF6F0025E0FFEF70339067E1E0FFEF600C906723
:10BF7F001BE0FFEF70047F0180027F00905931EFCB
:10BF8F00F090671BE0FFEF70109067297401F022AB
:0ABF9F0030B306906725740AF02203
:10BA180020B25990672FE0FFEF605190672FE01434
:10BA2800F090672FE0FFEF7022906721E0FFEF7042
:10BA38001A90671B7401F09067217401F090673BBE
:10BA48007401F090671F7401F0802A90672FE0FF5F
:10BA5800EF7022906721E0FFEF601A90671BE4F017
:10BA6800906721E4F090671FE4F0800930B20690F7
:10BA7800672F740AF020B457906730E0FFEF604FEB
:10BA8800906730E014F0906730E0FFEF7021906726
:10BA980022E0FFEF701990671C7401F09067227420
:10BAA80001F090673C7401F09067207401F02290D7
:10BAB8006730E0FFEF7021906722E0FFEF60199098
:10BAC800671CE4F0906722E4F0906720E4F02230ED
:09BAD800B406906730740AF022F4
:10A5760030E80302A61190672DE0FFEF700302A6F4
:10A586001190672DE014F090672DE0FFEF60030255
:10A59600A61F9056F5E0FFEF60139056F5E4F09095
:10A5A600593E7401F09067447401F0806C9067E145
:10A5B600E0FFEF600C90671BE0FFEF70047F018007
:10A5C600027F00906727EFF090671BE0FFEF7004B3
:10A5D6007F0180027F00906719EFF090671BE0FF14
:10A5E600EF70047F0180027F00906723EFF0906791
:10A5F600DEE0FFEF600C90671BE0FFEF70047F0169
:10A6060080027F00906737EFF0800E30E80B90678E
:10A616002D7432F0906719E4F030EB0302A6B8907F
:10A62600672EE0FFEF700302A6B890672EE014F0E5
:10A6360090672EE0FFEF600302A6C69056F6E0FF95
:10A64600EF60129056F6E4F090593F7401F090676F
:10A65600457401F0229067E2E0FFEF600C90671C02
:10A66600E0FFEF70047F0180027F00906728EFF023
:10A6760090671CE0FFEF70047F0180027F00906707
:10A686001AEFF090671CE0FFEF70047F0180027FF5
:10A6960000906724EFF09067DFE0FFEF600C9067B3
:10A6A6001CE0FFEF70047F0180027F00906738EFA7
:10A6B600F02230EB0B90672E7432F090671AE4F0BC
:01A6C6002271
:10B47400209726906746E0FFEF601E900A9FE0FF4A
:10B48400EF6016906746E014F0906746E0FFEF70B7
:10B49400119067347401F080093097069067467400
:10B4A4000AF020EA26906747E0FFEF601E900AA0AA
:10B4B400E0FFEF6016906747E014F0906747E0FF05
:10B4C400EF70119067357401F0800930EA069067D7
:10B4D40047740AF030971290673EE0FFEF600A90DD
:10B4E400673EE4F090672BE4F020973B900A9FE0DE
:10B4F400FFEF7033906748E0FFEF602B906748E000
:10B5040014F0906748E0FFEF70269067DEE0FFEFED
:10B51400600C90671BE0FFEF70047F0180027F00E6
:10B52400906740EFF0800930970690674874FAF00E
:10B5340030EA1290673FE0FFEF600A90673FE4F063
:10B5440090672CE4F020EA3A900AA0E0FFEF703212
:10B55400906749E0FFEF602A906749E014F0906734
:10B5640049E0FFEF70259067DFE0FFEF600C906724
:10B574001CE0FFEF70047F0180027F00906741EFC1
:0CB58400F02230EA0690674974FAF022C9
:10CEF50090673A74FFF090673974FFF090673D745E
:10CF0500FFF090673AE0FF90DD00EFF0906739E0C1
:10CF1500FF90EE00EFF090673DE0FF90FF00EFF02F
:01CF250022E9
:10B590009068E9EFF09068EAEDF09068EBEBF090DE
:10B5A00068EBE0FFEF607C9068EAE0FFEFF4FF906B
:10B5B00068EAEFF09068E9E0FFEF128F39B5E7171E
:10B5C000B5CA18B6041B0000B68F90673AE0FF902A
:10B5D00068EAE0FEEF5EFF90673AEFF090673AE0CE
:10B5E000FF90DD00EFF022906739E0FF9068EAE01D
:10B5F000FEEF5EFF906739EFF0906739E0FF90EE65
:10B6000000EFF02290673DE0FF9068EAE0FEEF5E19
:10B61000FF90673DEFF090673DE0FF90FF00EFF097
:10B620002222229068E9E0FFEF128F39B65617B652
:10B630003918B6731B0000B68F90673AE0FF906828
:10B64000EAE0FEEF4EFF90673AEFF090673AE0FFD6
:10B6500090DD00EFF022906739E0FF9068EAE0FEAD
:10B66000EF4EFF906739EFF0906739E0FF90EE0002
:10B67000EFF02290673DE0FF9068EAE0FEEF4EFFBA
:10B6800090673DEFF090673DE0FF90FF00EFF02204
:10B6900090674CE0FB7D017F1712B590906750E0FA
:10B6A000FB7D027F1712B59090674DE0FB7D047F14
:10B6B0001712B590906718E0FB7D087F1712B590C0
:10B6C00090672CE0FB7D107F1712B59090672BE000
:10B6D000FB7D207F1712B59090674AE0FB7D407F8D
:10B6E0001712B59090674EE0FB7D017F1812B59060
:10B6F00090671DE0FB7D027F1812B59090674FE0C8
:10B70000FB7D047F1812B59090671EE0FB7D087FDB
:10B710001812B590A2B2E433FD906736E0FB7F18B3
:10B7200012B590906744E0FB7D107F1812B59090A1
:10B730006745E0FB7D207F1812B590906732E0FBF3
:10B740007D407F1812B590906733E0FB7D807F18B5
:10B7500012B59090674BE0FB7D047F1B12B5909073
:10B760006729E0FB7D407F1B12B59090672AE0FBC4
:10B770007D107F1B12B590906720E0FB7D207F1B22
:10B7800012B59090671FE0FB7D807F1B12B5902261
:10701C00755A00E55AC3940240030275CAAF5A74FC
:10702C00EE2FF582E43462F583E0FFEF7003027516
:10703C00C5AF5A74EE2FF582E43462F583E4F0AFF9
:10704C005A74E62FF582E43460F583E4F0AF5A7499
:10705C00E42FF582E43460F583E4F0AF5A74E12F49
:10706C00F582E43460F583E4F0AF5A749D2FF58219
:10707C00E4340AF583E4F0AF5A74712FF582E434EA
:10708C0009F583E4F0AF5A74D92FF582E43460F536
:10709C0083E0FFC007AF5A7E00EF7F00FE74D92F4C
:1070AC00F9745E3EFA7B01D00712BFA9EF700302A0
:1070BC007552AF5A74362FF582E43459F583E4F0E7
:1070CC00E55A7007906732E4F0800AE55AB401057E
:1070DC00906733E4F0AF5A74052FF582E43459F518
:1070EC0083E0FFEF700302744CAF5A74052FF582E6
:1070FC00E43459F583E4F0AF5A74362FF582E43456
:10710C0059F583E4F0AF5A74AC2FF582E4340AF5E8
:10711C0083E4F0D290AF5AEF75F007A42403F58204
:10712C00E4345EF583AF82AE83C006C007AF5AEF7E
:10713C0075F003A424A6F582E4344EF583AD82AC3D
:10714C0083AF5A74002FF582E43459F583E0FB9039
:10715C006867E4F0AF5A7E00EF7F00FE74E82FF50D
:10716C008274603EF583AF82AE83906868EEF0A3C4
:10717C00EFF0D007D00612B34BAF5A74EA2FF5825A
:10718C00E43462F583740EF0AF5A74EC2FF582E49C
:10719C003462F583E4F0D299AF5A7E00EF7F00FEA3
:1071AC0074D92FF9745E3EFA7B01C003C002C00192
:1071BC00AF5A7E00EF7F00FE74B42FF9744E3EFA86
:1071CC007B01906891EBF0A3EAF0A3E9F0AF5A745D
:1071DC00D92FF582E43460F583E0FF906894EFF0EA
:1071EC00D001D002D00312CA5BAF5A7E00EF7F00F1
:1071FC00FE74B52FF582744E3EF583E0FFEFB4427A
:10720C0012AF5A74AF2FF582E4340AF5837401F08F
:10721C000275C5AF5A7E00EF7F00FE74C02FF58259
:10722C00744E3EF583E0FFEF64F5601CAF5A7E00B0
:10723C00EF7F00FE74C02FF582744E3EF583E0FFA5
:10724C00EF64FA60030272F7AF5A74AF2FF582E461
:10725C00340AF583E4F0AF5A7E007C1C7D23128E39
:10726C008974B82FF9740C3EFA7B01C003C002C0BC
:10727C0001AF5A7E00EF7F00FE74C02FF9744E3EB2
:10728C00FA7B01C003C002C0017B017A677954A864
:10729C0001AC02AD03D001D002D0037E007F3012CE
:1072AC008DE9D001D002D00312AD2EAF5A7E00EF83
:1072BC007F00FE74042FF974513EFA7B01C003C0A9
:1072CC0002C001AF5A7E00EF7F00FE74B42FF97438
:1072DC004E3EFA7B01A801AC02AD03D001D002D026
:1072EC00037E017F00128DE90275C5AF5A74AF2F72
:1072FC00F582E4340AF583E4F0AF5A7E00EF7F00A8
:10730C00FE74B42FF9744E3EFA7B01C003C002C068
:10731C0001AF5A7E00EF7F00FE74042FF974513ECA
:10732C00FA7B01A801AC02AD03D001D002D0037EE0
:10733C00017F00128DE9AF5A7E00EF7F00FE74F7DB
:10734C002FF582744E3EF583E0FFEF600302740D5F
:10735C00AF5A7E00EF7F00FE74C12FF582744E3E53
:10736C00F583E0FFEF6061AF5A7E00EF7F00FE74A3
:10737C00C12FF582744E3EF583E0FDAF5A7E00EFCF
:10738C007F00FE74F32FF582744E3EF583EDF0AF63
:10739C005A7E00EF7F00FE74F22FF582744E3EF59C
:1073AC0083E4F0AF5A7E00EF7F00FE74C12FF582AC
:1073BC00744E3EF583E0FFAE5A74012EF582E43430
:1073CC0000F583EFF00275C5AF5A74012FF582E416
:1073DC003400F583E0FDAF5A7E00EF7F00FE74F3BE
:1073EC002FF582744E3EF583EDF0AF5A7E00EF7FA1
:1073FC0000FE74F22FF582744E3EF583E4F00275B4
:10740C00C5AF5A7E00EF7F00FE74F72FF582744EE5
:10741C003EF583E0FDAF5A7E00EF7F00FE74F32F44
:10742C00F582744E3EF583EDF0AF5A7E00EF7F008F
:10743C00FE74F22FF582744E3EF583E4F00275C5AE
:10744C00AF5A74D12FF582E43450F583E0FFEF602E
:10745C0071AF5A74D12FF582E43450F583E4F0AF58
:10746C005A7E00EF7F00FE74D92FF9745E3EFA7BD2
:10747C0001C003C002C001AF5A7E00EF7F00FE7452
:10748C00F72FF974563EFA7B01906891EBF0A3EA62
:10749C00F0A3E9F0AF5A74D92FF582E43460F58388
:1074AC00E0FF906894EFF0D001D002D00312CA5BD9
:1074BC00AF5A74CA2FF582E43467F5837401F00275
:1074CC0075C5AF5A749A2FF582E4340CF583E0FF3E
:1074DC00EF70030275C5AF5A749A2FF582E4340C21
:1074EC00F583E4F0AF5A7E00EF7F00FE74D92FF9DC
:1074FC00745E3EFA7B01C003C002C001AF5A7E002D
:10750C00EF7F00FE74082FF974533EFA7B019068EC
:10751C0091EBF0A3EAF0A3E9F0AF5A74D92FF582FE
:10752C00E43460F583E0FF906894EFF0D001D00272
:10753C00D00312CA5BAF5A74C62FF582E43467F5D8
:10754C00837401F08073AF5A74AC2FF582E4340A63
:10755C00F583E004F0AF5A74AC2FF582E4340AF5ED
:10756C0083E0FF900AA5E0FEEFD39E404CAF5A7427
:10757C00362FF582E43459F5837401F0AF5A74ACAC
:10758C002FF582E4340AF583E014F0755B0CE55BAF
:10759C00D3944B5024AF5A7E00EF7F00FE74B42F6F
:1075AC00F582744E3EF583AF5BE5822FF582E435B0
:0E75BC0083F583E4F0055B80D5055A02701F4D
:0175CA00229E
:10B34B00906862EEF0A3EFF0906864ECF0A3EDF080
:05B35B00906866EBF0B4
:10B36000906868E0FEA3E0FF8E5D8F5E755C00E58F
:10B370005CC39407503C906862E0FEA3E0FF8F82BC
:10B380008E83E0FF906868E0FCA3E0FD8D828C83F3
:10B39000EFF0906869E004F07006906868E004F0EF
:10B3A000906863E004F07006906862E004F0055C69
:10B3B00080BD906866E0FF906868E0FCA3E0FD8DCA
:10B3C000828C83EFF0906869E004F0700690686802
:10B3D000E004F0755C00E55CC39403503C90686445
:10B3E000E0FEA3E0FF8F828E83E0FF906868E0FCC0
:10B3F000A3E0FD8D828C83EFF0906869E004F0702B
:10B4000006906868E004F0906865E004F0700690CB
:10B410006864E004F0055C80BD906867E0FF9068B8
:10B4200068E0FCA3E0FD8D828C83EFF0906869E01A
:10B4300004F07006906868E004F0AD5EAC5D7F0CCF
:10B4400012C0418E5F8F60906868E0FEA3E0FF8FBE
:10B45000828E83E560F0906869E004F07006906881
:10B4600068E004F0906868E0FEA3E0FF8F828E83BE
:03B47000E55FF0A5
:01B4730022B6
:10006600906880EFF0906881EBF0A3EAF0A3E9F0E6
:10007600906881E0FBA3E0FAA3E0F97582417583FD
:1000860000128E28FFEF20E60302012B906881E024
:10009600FBA3E0FAA3E0F9E92432F9EA3400FAC056
:1000A60003C002C001906880E0FF7E06EF8EF0A4D8
:1000B600FFAEF074AC2FF9740C3EFA7B0190689198
:1000C600EBF0A3EAF0A3E9F09068947406F0D0018F
:1000D600D002D00312CA5B906881E0FBA3E0FAA3CA
:1000E600E0F9E92438F9EA3400FAC003C002C00195
:1000F600906880E0FF7E06EF8EF0A4FFAEF07410ED
:100106002FF974553EFA7B01906891EBF0A3EAF063
:10011600A3E9F09068947406F0D001D002D00312DF
:10012600CA5B0201C1906881E0FBA3E0FAA3E0F993
:10013600E92432F9EA3400FAC003C002C00190682B
:1001460080E0FF7E06EF8EF0A4FFAEF074332FF949
:1001560074553EFA7B01906891EBF0A3EAF0A3E9AF
:10016600F09068947406F0D001D002D00312CA5BF6
:10017600906881E0FBA3E0FAA3E0F9E92438F9EA04
:100186003400FAC003C002C001906880E0FF7E061A
:10019600EF8EF0A4FFAEF074BB2FF974503EFA7BDD
:1001A60001906891EBF0A3EAF0A3E9F090689474EB
:1001B60006F0D001D002D00312CA5B906880E0FF3F
:1001C60074E82FF582E43462F583E0FFEF70179050
:1001D6006880E0FF74362FF582E43459F583E0FF3A
:1001E600EF7003020270906880E0FF74FB2FF582C7
:1001F600E43458F583E0FFEF6070906880E0FFEF2D
:1002060025E02400F582E43451F583E475F001120B
:100216008EF0900C55E0FF7E00906880E0FDED25A5
:10022600E02400F582E43451F583E0FCA3E0FDD33D
:10023600ED9FEC9E50030202CE900C55E0FF7E002F
:10024600906880E0FDED25E02400F582E43451F568
:1002560083EEF0A3EFF0906880E0FF74042FF58240
:10026600E43400F5837401F0805E906880E0FFEF6F
:1002760025E02400F582E43451F583E0FEA3E0FF97
:10028600EF4E6044906880E0FFEF25E02400F582A1
:10029600E43451F58374FF75F0FF128EF090688098
:1002A600E0FFEF25E02400F582E43451F583E0FE1B
:1002B600A3E0FFEF4E7011906880E0FF74042FF505
:1002C60082E43400F583E4F0906881E0FBA3E0FA71
:1002D600A3E0F975821E758300128E28FFEF701752
:1002E600906880E0FF749B2FF582E4340AF583E082
:1002F600FFEF7003020389906881E0FBA3E0FAA395
:10030600E0F9758229758300128E28FFEF60309020
:100316006881E0FBA3E0FAA3E0F975822A75830001
:10032600128E28FFEF6018906881E0FBA3E0FAA325
:10033600E0F9758228758300128E28FFEF704090D1
:100346006881E0FBA3E0FAA3E0F9758231758300CA
:10035600128E28FFEF6028906880E0FF74E82FF582
:1003660082E43462F583E0FFEF6018906880E0FF76
:1003760074FB2FF582E43458F583E0FFEF70047FB9
:100386000180027F00906880E0FE749B2EF582E477
:10039600340AF583EFF0906880E0FF74192FF58238
:1003A600E43467F583E0FFEF7030906881E0FBA3EB
:1003B600E0FAA3E0F9758244758300128E28FFEFF8
:1003C60020E017906880E0FF74B92FF582E434507E
:1003D600F583E0FFEF700302046C906881E0FBA3F5
:1003E600E0FAA3E0F9758229758300128E28FFEFE3
:1003F6007018906881E0FBA3E0FAA3E0F975822A01
:10040600758300128E28FFEF6016906880E0FF74F7
:10041600FE2FF582E43444F583E0FFEF6403602E9B
:10042600906880E0FF74FE2FF582E43444F583E0A3
:10043600FFEF64046030906881E0FBA3E0FAA3E07C
:10044600F9758231758300128E28FFEF7018906857
:1004560080E0FF74F72FF582E43458F583E0FFEF70
:1004660060047F0180027F00906880E0FE74B92EF0
:10047600F582E43450F583EFF0906880E0FF74195C
:100486002FF582E43467F583E0FFEF7014906880FF
:10049600E0FF74A82FF582E4340AF583E0FFEF60ED
:1004A6002C906880E0FF74E82FF582E43462F583CF
:1004B600E0FFEF6018906880E0FF74FB2FF582E4A0
:1004C6003458F583E0FFEF70047F0180027F0090CF
:1004D6006880E0FE74A82EF582E4340AF583EFF016
:1004E600906880E0FF74192FF582E43467F583E0A5
:1004F600FFEF602C906880E0FF74E82FF582E4340B
:1005060062F583E0FFEF7014906880E0FF74362F89
:10051600F582E43459F583E0FFEF60047F01800241
:100526007F00906880E0FE749F2EF582E43456F5D5
:1005360083EFF0906880E0FF74FE2FF582E4344488
:10054600F583E0FFEFD394064018906881E0FBA3A3
:10055600E0FAA3E0F9758231758300128E28FFEF69
:100566006019906880E0FF74FE2FF582E43444F54C
:1005760083E0FFEF64036003020704906880E0FFF6
:1005860074F72FF582E43458F583E0FFEF70030229
:100596000704906880E0FF74B92FF582E43450F5C3
:1005A60083E0FFEF6073906881E0FBA3E0FAA3E0CD
:1005B600F9758231758300128E28FFEF600C900961
:1005C6008FE0FF906884EFF0800A9050B4E0FF90CF
:1005D6006884EFF0906880E0FF74562FF582E4346B
:1005E6000CF583E004F0906880E0FF74562FF582E6
:1005F600E4340CF583E0FF906884E0FEEFC39E5080
:100606000302082C906880E0FF74CF2FF582E43453
:1006160050F5837401F002082C906880E0FF749B0B
:100626002FF582E4340AF583E0FFEF70030206BF7C
:10063600906881E0FBA3E0FAA3E0F9758231758347
:1006460000128E28FFEF600C900CA5E0FF906884E6
:10065600EFF0800A905933E0FF906884EFF09068DD
:1006660080E0FF74562FF582E4340CF583E004F045
:10067600906880E0FF74562FF582E4340CF583E031
:10068600FF906884E0FEEFC39E500302082C90683A
:1006960080E0FF74382FF582E43459F5837401F055
:1006A600906884E0FF906880E0FE74562EF582E440
:1006B600340CF583EFF002082C906880E0FF74A8F4
:1006C6002FF582E4340CF583E004F0906880E0FFB7
:1006D60074A82FF582E4340CF583E0FF900006E061
:1006E600FEEFC39E500302082C906880E0FF74E47E
:1006F6002FF582E43456F5837401F002082C9068D5
:1007060080E0FF74562FF582E4340CF583E4F09014
:100716006880E0FF74A82FF582E4340CF583E4F0DA
:10072600906880E0FF74FE2FF582E43444F583E0A0
:10073600FFEF64276041906880E0FF74FE2FF5822A
:10074600E43444F583E0FFEF6424602B906880E096
:10075600FF74FE2FF582E43444F583E0FFEF642551
:100766006015906880E0FF74FE2FF582E43444F54E
:1007760083E0FFEFB40418906881E0FBA3E0FAA3DE
:10078600E0F9758227758300128E28FFEF60047FDB
:100796000180027F00906884EFF0906880E0FF742B
:1007A600CF2FF582E43450F583C083C082E0FF90FA
:1007B6006884E0FEEF5EFFD082D083EFF090688021
:1007C600E0FF74382FF582E43459F583C083C08284
:1007D600E0FF906884E0FEEF5EFFD082D083EFF00A
:1007E600906880E0FF74E42FF582E43456F583C008
:1007F60083C082E0FF906884E0FEEF5EFFD082D087
:1008060083EFF0906880E0FF74B92FF582E43450EE
:10081600F583C083C082E0FF906884E0FEEF5EFF50
:10082600D082D083EFF0906880E0FF74FB2FF582D2
:10083600E43458F583E0FFEF6003020963906880B3
:10084600E0FF74E82FF582E43462F583E0FFEF7091
:1008560003020963906880E0FF74A82FF582E434F0
:100866000AF583E0FFEF6045906880E0FF74F92F9A
:10087600F582E43458F583E004F0906880E0FF7474
:10088600F92FF582E43458F583E0FF900C97E0FEEB
:10089600EFC39E50030209C9906880E0FF74AA2F37
:1008A600F582E4340AF5837401F00209C990688080
:1008B600E0FF749B2FF582E4340AF583E0FFEF60D6
:1008C6005B906880E0FF74F92FF582E43458F58375
:1008D600E004F0906880E0FF74F92FF582E4345864
:1008E600F583E0FF9056ECE0FEEFC39E500302094D
:1008F600C9906880E0FF74CD2FF582E43450F5830B
:100906007401F09056ECE0FF906880E0FE74F92EDA
:10091600F582E43458F583EFF00209C9906880E067
:10092600FF74922FF582E43409F583E004F09068B1
:1009360080E0FF74922FF582E43409F583E0FF909E
:1009460050EEE0FEEFC39E407A906880E0FF74941C
:100956002FF582E4340CF5837401F080669068808C
:10096600E0FF74CD2FF582E43450F583E4F090680F
:1009760080E0FF74AA2FF582E4340AF583E4F09050
:100986006880E0FF74F92FF582E43458F583E4F0CB
:10099600906880E0FF74942FF582E4340CF583E4CC
:1009A600F0906880E0FF74922FF582E43409F583B5
:1009B600E4F0906880E0FF74A82FF582E4340AF52D
:1009C60083E4F0906880E0FF74EF2FF582E4345002
:1009D600F583E0FFEF64466043906880E0FF74EFC4
:1009E6002FF582E43450F583E0FFEF6478602D90B4
:1009F6006880E0FF74EF2FF582E43450F583E0FF62
:100A0600EF64866017906880E0FF74A62FF582E495
:100A1600340AF583E0FFEFD39400406F906881E0DD
:100A2600FBA3E0FAA3E0F9758227758300128E28EE
:100A3600FFEF7057906880E0FF74A62FF582E434CC
:100A46000AF583E004F0906880E0FF74A62FF58233
:100A5600E4340AF583E0FF905530E0FEEFC39E5084
:100A660003020B2D906880E0FF74942FF582E43426
:100A76004EF5837401F0906880E0FF74A62FF5822E
:100A8600E4340AF583E014F0020B2D906880E0FF51
:100A960074EF2FF582E43450F583E0FFEF64847041
:100AA60053906880E0FF74B72FF582E43450F583E5
:100AB600E004F0906880E0FF74B72FF582E43450CC
:100AC600F583E0FF905530E0FEEFC39E40599068F5
:100AD60080E0FF74942FF582E4344EF5837401F0C0
:100AE600906880E0FF74B72FF582E43450F583E018
:100AF60014F08033906880E0FF74942FF582E4341C
:100B06004EF583E4F0906880E0FF74A62FF582E44A
:100B1600340AF583E4F0906880E0FF74B72FF5821D
:100B2600E43450F583E4F0906880E0FF74EF2FF52D
:100B360082E43450F583E0FFEF6467604690688096
:100B4600E0FF74EF2FF582E43450F583E0FFEF64A5
:100B5600856030906880E0FF74EF2FF582E43450B2
:100B6600F583E0FFEF6487601A906880E0FF74A366
:100B76002FF582E4340AF583E0FFEFD394005003A7
:100B8600020C24906881E0FBA3E0FAA3E0F97582E9
:100B960028758300128E28FFEF6030906881E0FB95
:100BA600A3E0FAA3E0F9758229758300128E28FF67
:100BB600EF6018906881E0FBA3E0FAA3E0F9758284
:100BC6002A758300128E28FFEF7053906880E0FF2D
:100BD60074A32FF582E4340AF583E004F09068806C
:100BE600E0FF74A32FF582E4340AF583E0FF905505
:100BF60028E0FEEFC39E4048906880E0FF74082F0F
:100C0600F582E43445F5837401F0906880E0FF7462
:100C1600A32FF582E4340AF583E014F0802290686D
:100C260080E0FF74A32FF582E4340AF583E4F090A4
:100C36006880E0FF74082FF582E43445F583E4F01C
:100C4600906880E0FF74FE2FF582E43444F583E07B
:100C5600FFEFC3940F405B906880E0FF74FE2FF5B2
:100C660082E43444F583E0FFEFD394275044906840
:100C760080E0FF74F72FF582E43458F583E0FFEF48
:100C86006030906881E0FBA3E0FAA3E0F975822862
:100C9600758300128E28FFEF6018906880E0FF745D
:100CA600942FF582E4344EF583E0FFEF70047F0164
:100CB60080027F00906884EFF0906884E0FF90687F
:100CC60081E0FBA3E0FAA3E0F975822375830012A5
:100CD6008E28FEEE5403FEEE6003020D60906881DE
:100CE600E0FBA3E0FAA3E0F975822D758300128E6E
:100CF60028FEEE20E064906881E0FBA3E0FAA3E022
:100D0600F975822F758300128E28FEEE20E04B9037
:100D16006881E0FBA3E0FAA3E0F975822075830001
:100D2600128E28FEEE20E132906881E0FBA3E0FA05
:100D3600A3E0F975822E758300128E28FEEE20E060
:100D460019906881E0FBA3E0FAA3E0F9758230759B
:100D56008300128E28FEEE30E030906881E0FBA31F
:100D6600E0FAA3E0F9758227758300128E28FEEE5D
:100D76006018906880E0FE74F72EF582E43458F52A
:100D860083E0FEEE60047E0180027E00EF4EFF905F
:100D96006884EFF0906884E0FF906881E0FBA3E050
:100DA600FAA3E0F975821E758300128E28FEEE7096
:100DB60018906881E0FBA3E0FAA3E0F975821F753D
:100DC6008300128E28FEEE60047E0180027E00EF14
:100DD6005EFF906884EFF0906884E0FF906880E0A2
:100DE600FE74FE2EF582E43444F583E0FEEE6408DC
:100DF6006015906880E0FE74FE2EF582E43444F5BA
:100E060083E0FEEEB40930906881E0FBA3E0FAA32C
:100E1600E0F9758231758300128E28FEEE70189007
:100E26006880E0FE74F72EF582E43458F583E0FE20
:100E3600EE60047E0180027E00EF4EFF906884EF34
:100E4600F0906884E0FF905508EFF0906884E0FF2A
:100E5600EF6071906880E0FFEF25E02459F582E4A9
:100E6600340CF583E475F001128EF0900C91E0FFDE
:100E76007E00EF7F00FE900C96E0FD7C00EF2DFFDC
:100E8600EE3CFE906885EEF0A3EFF0906880E0FF00
:100E9600EF25E02459F582E4340CF583E0FEA3E067
:100EA600FF906885E0FCA3E0FDC3EF9DEE9C403B10
:100EB600906880E0FF74D72FF582E43450F5837490
:100EC60001F08027906880E0FFEF25E02459F58245
:100ED600E4340CF583E4F0A3E4F0906880E0FF745A
:100EE600D72FF582E43450F583E4F0906880E0FF74
:100EF60074192FF582E43467F583E0FFEF604F90B5
:100F06006880E0FF74492FF582E4340CF583E00431
:100F1600F0906880E0FF74492FF582E4340CF58385
:100F2600E0FFEFC3941E4048906880E0FF74492FAD
:100F3600F582E4340CF583741EF0906880E0FF744B
:100F4600F52FF582E43450F5837401F08022906821
:100F560080E0FF74492FF582E4340CF583E4F090C9
:100F66006880E0FF74F52FF582E43450F583E4F0F1
:100F7600905529E0FFEF6057906880E0FF74B12F2D
:100F8600F582E4340AF583E004F0906880E0FF74AB
:100F9600B12FF582E4340AF583E0FF9056AEE0FE09
:100FA600EFC39E4075906880E0FF74AC2FF582E435
:100FB600344EF5837401F09056AEE0FF906880E001
:100FC600FE74B12EF582E4340AF583EFF0804B907F
:100FD6006880E0FF74AC2FF582E4344EF583E0FFC1
:100FE600EF6037906880E0FF74B12FF582E4340A31
:100FF600F583E014F0906880E0FF74B12FF582E489
:10100600340AF583E0FFEF7011906880E0FF74AC5E
:101016002FF582E4344EF583E4F0906880E0FF74A7
:10102600CF2FF582E43450F583E0FFEF7028906807
:1010360080E0FF74AA2FF582E4340AF583E0FFEF1F
:101046007014906880E0FF749F2FF582E43456F5A3
:1010560083E0FFEF6018906880E0FF74192FF58237
:10106600E43467F583E0FFEF60047F0180027F00D0
:10107600906880E0FE74922EF582E4340AF583EFE0
:10108600F0906881E0FBA3E0FAA3E0F9758244756D
:101096008300128E28FFEF30E170906880E0FFEF4A
:1010A60025E0248DF582E4340CF583E475F0011215
:1010B6008EF0900CA4E0FF7E00906880E0FDED25A8
:1010C600E0248DF582E4340CF583E0FCA3E0FDC357
:1010D600ED9FEC9E500302116E906880E0FF742431
:1010E6002FF582E43455F5837401F0900CA4E0FFEB
:1010F6007E00906880E0FDED25E0248DF582E434E5
:101106000CF583EEF0A3EFF0805E906880E0FFEFD1
:1011160025E0248DF582E4340CF583E0FEA3E0FFA0
:10112600EF4E6044906880E0FFEF25E0248DF58265
:10113600E4340CF58374FF75F0FF128EF09068802E
:10114600E0FFEF25E0248DF582E4340CF583E0FE24
:10115600A3E0FFEF4E7011906880E0FF74242FF536
:1011660082E43455F583E4F0906880E0FF74FE2F46
:10117600F582E43444F583E0FFEF6404707190680F
:1011860080E0FFEF25E024A0F582E4340CF583E44B
:1011960075F001128EF0900003E0FF7E00906880EB
:1011A600E0FDED25E024A0F582E4340CF583E0FCB7
:1011B600A3E0FDC3ED9FEC9E50030212959068805C
:1011C600E0FF74DC2FF582E43456F5837401F09069
:1011D6000003E0FF7E00906880E0FDED25E024A09E
:1011E600F582E4340CF583EEF0A3EFF0021295904D
:1011F6006880E0FF74FE2FF582E43444F583E0FF57
:10120600EF6424602C906880E0FF74FE2FF582E482
:101216003444F583E0FFEF64256016906880E0FFB4
:1012260074FE2FF582E43444F583E0FFEF64277003
:101236005E906880E0FFEF25E024A0F582E4340CA0
:10124600F583E0FEA3E0FFEF4E6044906880E0FF88
:10125600EF25E024A0F582E4340CF58374FF75F0E5
:10126600FF128EF0906880E0FFEF25E024A0F58263
:10127600E4340CF583E0FEA3E0FFEF4E70119068B6
:1012860080E0FF74DC2FF582E43456F583E4F090B9
:101296006880E0FF74922FF582E4340AF583E0FF5C
:1012A600EF6026906880E0FF74962FF582E4340A9A
:1012B600F583E0FFEF7012906880E0FF74902FF5E1
:1012C60082E4340AF5837465F0906880E0FF7492D6
:1012D6002FF582E4340AF583E0FF906880E0FE741F
:1012E600962EF582E4340AF583EFF0906880E0FFED
:1012F60074902FF582E4340AF583E0FFEF60030271
:101306001C27906880E0FF74042FF582E43400F512
:1013160083E0FFEF6026906880E0FF74092FF58276
:10132600E43400F583E0FFEF7012906880E0FF740C
:10133600902FF582E4340AF5837447F0906880E0D4
:10134600FF74042FF582E43400F583E0FF90688093
:10135600E0FE74092EF582E43400F583EFF0906820
:1013660080E0FF74042FF582E43400F583E0FFEF9C
:1013760070047F0180027F00906884EFF09068849B
:10138600E0FFEF603A906880E0FF74CF2FF582E4CB
:101396003450F583E0FFEF6026906880E0FF74E04C
:1013A6002FF582E43450F583E0FFEF7012906880E9
:1013B600E0FF74902FF582E4340AF5837461F090AF
:1013C6006880E0FF74CF2FF582E43450F583E0FFA8
:1013D600906880E0FE74E02EF582E43450F583EFE9
:1013E600F0906884E0FF906880E0FE74CF2EF5826E
:1013F600E43450F583E0FEEE70047E0180027E0048
:10140600EF5EFF906884EFF0906884E0FFEF603A4B
:10141600906880E0FF74382FF582E43459F583E054
:10142600FFEF6026906880E0FF74402FF582E43479
:1014360059F583E0FFEF7012906880E0FF74902FFB
:10144600F582E4340AF5837462F0906880E0FF74F4
:10145600382FF582E43459F583E0FF906880E0FE8A
:1014660074402EF582E43459F583EFF0906884E0F9
:10147600FF906880E0FE74382EF582E43459F583D7
:10148600E0FEEE70047E0180027E00EF5EFF906853
:1014960084EFF0906884E0FFEF603A906880E0FFA8
:1014A60074AA2FF582E4340AF583E0FFEF602690F4
:1014B6006880E0FF744B2FF582E4340CF583E0FF7F
:1014C600EF7012906880E0FF74902FF582E4340A82
:1014D600F5837463F0906880E0FF74AA2FF582E4C8
:1014E600340AF583E0FF906880E0FE744B2EF582A7
:1014F600E4340CF583EFF0906884E0FF906880E0B8
:10150600FE74AA2EF582E4340AF583E0FEEE70043A
:101516007E0180027E00EF5EFF906884EFF09068A7
:1015260084E0FFEF603A906880E0FF74CD2FF5828B
:10153600E43450F583E0FFEF6026906880E0FF74A6
:10154600DE2FF582E43450F583E0FFEF70129068E9
:1015560080E0FF74902FF582E4340AF5837464F01A
:10156600906880E0FF74CD2FF582E43450F583E077
:10157600FF906880E0FE74DE2EF582E43450F58339
:10158600EFF0906884E0FF906880E0FE74CD2EF561
:1015960082E43450F583E0FEEE70047E0180027E24
:1015A60000EF5EFF906884EFF0906884E0FFEF60E4
:1015B60062906880E0FF74E42FF582E43456F58388
:1015C600E0FFEF604E906880E0FF74F12FF582E453
:1015D6003456F583E0FFEF703A906880E0FF74942C
:1015E6002FF582E4344EF583E0FFEF702690688095
:1015F600E0FF74082FF582E43445F583E0FFEF70D1
:1016060012906880E0FF74902FF582E4340AF58327
:101616007427F0906880E0FF74E42FF582E4345676
:10162600F583E0FF906880E0FE74F12EF582E434E5
:1016360056F583EFF0906884E0FF906880E0FE74D2
:10164600E42EF582E43456F583E0FEEE70047E0166
:1016560080027E00EF5EFF906884EFF0906884E081
:10166600FFEF603A906880E0FF74942FF582E434CF
:101676000CF583E0FFEF6026906880E0FF74982FFA
:10168600F582E4340CF583E0FFEF7012906880E099
:10169600FF74902FF582E4340AF5837441F0906864
:1016A60080E0FF74942FF582E4340CF583E0FF901C
:1016B6006880E0FE74982EF582E4340CF583EFF032
:1016C600906884E0FF906880E0FE74942EF582E4D2
:1016D600340CF583E0FEEE70047E0180027E00EF9E
:1016E6005EFF906884EFF0906884E0FFEF603A90C8
:1016F6006880E0FF74942FF582E4344EF583E0FFB2
:10170600EF6026906880E0FF749E2FF582E4344EE9
:10171600F583E0FFEF7012906880E0FF74902FF57C
:1017260082E4340AF5837415F0906880E0FF7494BF
:101736002FF582E4344EF583E0FF906880E0FE7476
:101746009E2EF582E4344EF583EFF0906884E0FF38
:10175600906880E0FE74942EF582E4344EF583E0C2
:10176600FEEE70047E0180027E00EF5EFF906884CC
:10177600EFF0906884E0FFEF603A906880E0FF74D5
:10178600082FF582E43445F583E0FFEF6026906884
:1017960080E0FF749A2FF582E4344EF583E0FFEF84
:1017A6007012906880E0FF74902FF582E4340AF599
:1017B600837416F0906880E0FF74082FF582E43495
:1017C60045F583E0FF906880E0FE749A2EF582E48A
:1017D600344EF583EFF0906884E0FF906880E0FE79
:1017E60074082EF582E43445F583E0FEEE70047E3F
:1017F6000180027E00EF5EFF906884EFF0906884BF
:10180600E0FFEF603A906880E0FF74D72FF582E43E
:101816003450F583E0FFEF6026906880E0FF74E8BF
:101826002FF582E43450F583E0FFEF701290688064
:10183600E0FF74902FF582E4340AF5837406F09085
:101846006880E0FF74D72FF582E43450F583E0FF1B
:10185600906880E0FE74E82EF582E43450F583EF5C
:10186600F0906884E0FF906880E0FE74D72EF582E1
:10187600E43450F583E0FEEE70047E0180027E00C3
:10188600EF5EFF906884EFF0906884E0FFEF603AC7
:10189600906880E0FF74F52FF582E43450F583E01C
:1018A600FFEF6026906880E0FF74FE2FF582E43437
:1018B60050F583E0FFEF7012906880E0FF74902F80
:1018C600F582E4340AF5837494F0906880E0FF743E
:1018D600F52FF582E43450F583E0FF906880E0FE52
:1018E60074FE2EF582E43450F583EFF0906884E0C0
:1018F600FF906880E0FE74F52EF582E43450F5839F
:10190600E0FEEE70047E0180027E00EF5EFF9068CE
:1019160084EFF0906880E0FF74902FF582E4340A3B
:10192600F583E0FFEF6012906880E0FF749E2FF56C
:1019360082E4340CF5837401F0906880E0FF7490C3
:101946002FF582E4340AF583E0FFEFD39460403448
:10195600906880E0FF74902FF582E4340AF583E006
:10196600FFEFC39465501D906880E0FFEF7006900E
:10197600674C7401F0906880E0FFEFB40106906751
:101986004D7401F0906884E0FFEF6052906880E04B
:10199600FF749E2FF582E4340CF583E0FFEF603E82
:1019A600906880E0FF74902FF582E4340AF5837422
:1019B60029F0906880E0FF749E2FF582E4340CF5E0
:1019C60083E4F0906880E0FFEF700590674CE4F0E8
:1019D600906880E0FFEFB4010590674DE4F09068F1
:1019E60080E0FF74902FF582E4340AF583E0FFEF80
:1019F6006003021AAD906884E0FFEF604090688053
:101A0600E0FF74AC2FF582E4344EF583E0FFEF601F
:101A16002C906880E0FF74B52FF582E43450F5838E
:101A2600E0FFEF7018906880E0FF74902FF582E475
:101A3600340AF5837448F09067177401F09068844F
:101A4600E0FFEF6040906880E0FF74AC2FF582E421
:101A5600344EF583E0FFEF702C906880E0FF74B59C
:101A66002FF582E43450F583E0FFEF60189068802C
:101A7600E0FF74902FF582E4340AF5837449F09000
:101A860067177402F0906880E0FF74AC2FF582E46B
:101A9600344EF583E0FF906880E0FE74B52EF58243
:101AA600E43450F583EFF0906880E0FF74902FF5F2
:101AB60082E4340AF583E0FFEF6003021B6A906854
:101AC60084E0FFEF603A906880E0FF74242FF5828F
:101AD600E43455F583E0FFEF6026906880E0FF74FC
:101AE6002C2FF582E43455F583E0FFEF70129068F1
:101AF60080E0FF74902FF582E4340AF5837430F0A9
:101B0600906884E0FFEF603A906880E0FF74242FCD
:101B1600F582E43455F583E0FFEF7026906880E0A7
:101B2600FF742C2FF582E43455F583E0FFEF601245
:101B3600906880E0FF74902FF582E4340AF5837490
:101B460031F0906880E0FF74242FF582E43455F577
:101B560083E0FF906880E0FE742C2EF582E4345515
:101B6600F583EFF0906880E0FF74902FF582E434FF
:101B76000AF583E0FFEF6003021C27906884E0FF0C
:101B8600EF603A906880E0FF74DC2FF582E434560B
:101B9600F583E0FFEF6026906880E0FF74EA2FF59A
:101BA60082E43456F583E0FFEF7012906880E0FF20
:101BB60074902FF582E4340AF5837432F0906884C9
:101BC600E0FFEF603A906880E0FF74DC2FF582E476
:101BD6003456F583E0FFEF7026906880E0FF74EAE4
:101BE6002FF582E43456F583E0FFEF6012906880AB
:101BF600E0FF74902FF582E4340AF5837433F09095
:101C06006880E0FF74DC2FF582E43456F583E0FF4C
:101C1600906880E0FE74EA2EF582E43456F583EF90
:101C2600F0906880E0FF74902FF582E4340AF58323
:101C3600E0FFEF7003021CF3906880E0FF741B2F37
:101C4600F582E43467F583E0FFEF6003021CF3904E
:101C56006880E0FFEF75F00CA424BEF582E43456EC
:101C6600F583AF82AE83C006C007906880E0FF7E32
:101C760000EF7F00FE74B42FF582744E3EF583ADFF
:101C860082AC83906880E0FBD007D006129AB990A8
:101C96006880E0FF7E7BEF8EF0A4FFAEF074942F99
:101CA600F974093EFA7B01C003C002C00190688046
:101CB600E0FF7E0CEF8EF0A4FFAEF074BE2FF97439
:101CC600563EFA7B01C003C002C0017B017A6879E7
:101CD60025A801AC02AD03D001D002D0037E007F5F
:101CE6000C128DE9D001D002D00312A95C90688055
:101CF600E0FF74902FF582E4340AF583E4F09068EF
:101D060080E0FFEF25E024C9F582E43450F583E056
:101D1600FEA3E0FFEF4E6019906880E0FFEF25E03C
:101D260024C9F582E43450F58374FF75F0FF128EF2
:101D3600F0906880E0FF74DC2FF582E43450F58380
:101D4600E0FFEF701D906880E0FFEF25E024C9F505
:101D560082E43450F583E0FEA3E0FFEF4E70030209
:101D6600474C906880E0FF748C2FF582E4340AF5C6
:101D760083E0FFEF602C906880E0FF74192FF582F6
:101D8600E43467F583E0FFEF6018906880E0FF7445
:101D9600542FF582E43459F583E0FFEF70047F0198
:101DA60080027F00906880E0FE74832EF582E43422
:101DB6000CF583EFF0906880E0FF74E22FF582E483
:101DC6003456F583E0FFEF6016906880E0FF74FEFE
:101DD6002FF582E43444F583E0FFEF6403602B9033
:101DE6006880E0FF74EF2FF582E43450F583E0FF5E
:101DF600EF64196015906880E0FF74EF2FF582E4B8
:101E06003450F583E0FFEFB418047F0180027F00B1
:101E1600906880E0FE74E22EF582E43456F583EF96
:101E2600F0906880E0FF74C72FF582E43450F583A4
:101E3600E0FFEF7042906880E0FF74EF2FF582E4D8
:101E46003450F583E0FFEF6467602C906880E0FF14
:101E560074EF2FF582E43450F583E0FFEF6485607C
:101E660016906880E0FF74EF2FF582E43450F58316
:101E7600E0FFEF6487704C906881E0FBA3E0FAA373
:101E8600E0F9758228758300128E28FFEF60309086
:101E96006881E0FBA3E0FAA3E0F975822975830067
:101EA600128E28FFEF6018906881E0FBA3E0FAA38A
:101EB600E0F975822A758300128E28FFEF70047F81
:101EC6000180027F00906880E0FE74C72EF582E4F0
:101ED6003450F583EFF0906880E0FF74D52FF582DB
:101EE600E43450F583E0FFEF7041906880E0FF74C2
:101EF600EF2FF582E43450F583E0FFEF6446602B64
:101F0600906880E0FF74EF2FF582E43450F583E0AB
:101F1600FFEF64786015906880E0FF74EF2FF5821C
:101F2600E43450F583E0FFEFB48618906881E0FB57
:101F3600A3E0FAA3E0F9758227758300128E28FFC5
:101F4600EF6015906880E0FF74EF2FF582E434505F
:101F5600F583E0FFEFB484047F0180027F00906880
:101F660080E0FE74D52EF582E43450F583EFF090D0
:101F76006881E0FBA3E0FAA3E0F97582317583007E
:101F8600128E28FFEF7055906880E0FF74F72FF5EA
:101F960082E43458F583E0FFEF6041906880E0FF0B
:101FA60074342FF582E43459F583E004F0906880A8
:101FB600E0FF74342FF582E43459F583E0FF900A8C
:101FC600AEE0FEEFC39E4036906880E0FF747A2F45
:101FD600F582E4340CF5837401F08022906880E089
:101FE600FF74342FF582E43459F583E4F090688069
:101FF600E0FF747A2FF582E4340CF583E4F0906800
:1020060080E0FF74982FF582E4344EF583E0FFEF0D
:102016006016906880E0FF74FE2FF582E43444F584
:1020260083E0FFEF64036015906880E0FF74EF2F94
:10203600F582E43450F583E0FFEFB448047F018075
:10204600027F00906880E0FE74982EF582E4344E9C
:10205600F583EFF0906880E0FF74DA2FF582E434C0
:1020660056F583E0FFEF6016906880E0FF74FE2F60
:10207600F582E43444F583E0FFEF6403601590686D
:1020860080E0FF74EF2FF582E43450F583E0FFEF34
:10209600B459047F0180027F00906880E0FE74DA04
:1020A6002EF582E43456F583EFF0906880E0FF74F5
:1020B6000E2FF582E43455F583E0FFEF6016906845
:1020C60080E0FF74FE2FF582E43444F583E0FFEFF1
:1020D6006403602B906880E0FF74EF2FF582E43490
:1020E60050F583E0FFEF64626015906880E0FF744E
:1020F600EF2FF582E43450F583E0FFEFB463047FFD
:102106000180027F00906880E0FE740E2EF582E466
:102116003455F583EFF0905508E0FFEF6041906885
:1021260080E0FF74892FF582E4340CF583E004F037
:10213600906880E0FF74892FF582E4340CF583E023
:10214600FF905902E0FEEFD39E4036906880E0FF94
:1021560074FC2FF582E43450F5837401F0802290EC
:102166006880E0FF74FC2FF582E43450F583E4F0D8
:10217600906880E0FF74892FF582E4340CF583E4DF
:10218600F0906880E0FF74DC2FF582E43450F5832C
:10219600E0FFEF20E11D906880E0FFEF25E024C915
:1021A600F582E43450F583E0FEA3E0FFEF4E7003C2
:1021B600022C4F906880E0FF749B2FF582E4340A6E
:1021C600F583E0FFEF703C906880E0FF74B92FF56F
:1021D60082E43450F583E0FFEF7028906880E0FFDA
:1021E60074A82FF582E4340AF583E0FFEF701490AB
:1021F6006880E0FF744E2FF582E4340CF583E0FF2F
:10220600EF6055906880E0FF74FE2FF582E4344459
:10221600F583E0FFEFB40314906880E0FF74F72FB6
:10222600F582E43458F583E0FFEF7028906880E08B
:10223600FF74FB2FF582E43458F583E0FFEF701846
:10224600906880E0FF74E82FF582E43462F583E05D
:10225600FFEF60047F0180027F00906880E0FE74DB
:102266004E2EF582E4340CF583EFF0906880E0FFA3
:1022760074A62FF582E4340CF583E0FFEF60169028
:102286006880E0FF74FE2FF582E43444F583E0FFB6
:10229600EF6403602E906880E0FF74EF2FF582E410
:1022A6003450F583E0FFEFB4191D906881E0FBA37D
:1022B600E0FAA3E0F9758244758300128E28FFEFD9
:1022C60030E3047F0180027F00906880E0FE74A600
:1022D6002EF582E4340CF583EFF0906880E0FF740D
:1022E600852FF582E4340CF583E0FFEF60169068E5
:1022F60080E0FF74FE2FF582E43444F583E0FFEFBF
:102306006403602E906880E0FF74EF2FF582E4345A
:1023160050F583E0FFEFB4191D906881E0FBA3E060
:10232600FAA3E0F9758244758300128E28FFEF3018
:10233600E2047F0180027F00906880E0FE74852EB3
:10234600F582E4340CF583EFF0906880E0FF74903A
:102356002FF582E43409F583E0FFEF60159068807D
:10236600E0FF74FE2FF582E43444F583E0FFEFB41A
:10237600272B906880E0FF74EF2FF582E43450F548
:1023860083E0FFEF64656015906880E0FF74EF2FCF
:10239600F582E43450F583E0FFEFB466047F0180F4
:1023A600027F00906880E0FE74902EF582E4340986
:1023B600F583EFF0906880E0FF749D2FF582E4349A
:1023C60056F583E0FFEF6015906880E0FF74FE2FFE
:1023D600F582E43444F583E0FFEFB4272B90688060
:1023E600E0FF74EF2FF582E43450F583E0FFEF64ED
:1023F600506015906880E0FF74EF2FF582E434504A
:10240600F583E0FFEFB451047F0180027F009068FE
:1024160080E0FE749D2EF582E43456F583EFF0904D
:102426006881E0FBA3E0FAA3E0F9758220758300DA
:10243600128E28FFEF5480FF906880E0FE74F32E22
:10244600F582E43450F583EFF0900C4DE0FFEF6039
:102456005B906880E0FF742A2FF582E43455F5839B
:10246600E0FFEF6016906880E0FF74FE2FF582E4CF
:102476003444F583E0FFEF6403601A906880E0FF60
:1024860074EF2FF582E43450F583E0FF900C4DE0B5
:10249600FEEFB506047F0180027F00906880E0FEB3
:1024A600742A2EF582E43455F583EFF0900C50E053
:1024B600FFEF605B906880E0FF74312FF582E434B3
:1024C60055F583E0FFEF6016906880E0FF74FE2FFD
:1024D600F582E43444F583E0FFEF6403601A906804
:1024E60080E0FF74EF2FF582E43450F583E0FF902F
:1024F6000C50E0FEEFB506047F0180027F00906875
:1025060080E0FE74312EF582E43455F583EFF090C9
:102516000C51E0FFEF605B906880E0FF74992FF547
:1025260082E43456F583E0FFEF6016906880E0FFA2
:1025360074FE2FF582E43444F583E0FFEF64036014
:102546001A906880E0FF74EF2FF582E43450F5832B
:10255600E0FF900C51E0FEEFB506047F0180027F9C
:1025660000906880E0FE74992EF582E43456F58377
:10257600EFF0900C54E0FFEF605B906880E0FF7432
:10258600A42FF582E43456F583E0FFEF60169068D9
:1025960080E0FF74FE2FF582E43444F583E0FFEF1C
:1025A6006403601A906880E0FF74EF2FF582E434CC
:1025B60050F583E0FF900C54E0FEEFB506047F0172
:1025C60080027F00906880E0FE74A42EF582E434D9
:1025D60056F583EFF0900C58E0FFEF605B90688053
:1025E600E0FF74A82FF582E43456F583E0FFEF6030
:1025F60016906880E0FF74FE2FF582E43444F5837C
:10260600E0FFEF6403601A906880E0FF74EF2FF537
:1026160082E43450F583E0FF900C58E0FEEFB506F7
:10262600047F0180027F00906880E0FE74A82EF58A
:1026360082E43456F583EFF0900C5DE0FFEF605BCB
:10264600906880E0FF74B32FF582E43456F583E09A
:10265600FFEF6016906880E0FF74FE2FF582E43489
:1026660044F583E0FFEF6403601A906880E0FF742E
:10267600EF2FF582E43450F583E0FF900C5DE0FE29
:10268600EFB506047F0180027F00906880E0FE744B
:10269600B32EF582E43456F583EFF0900C5EE0FF3E
:1026A600EF605B906880E0FF74BA2FF582E43456E1
:1026B600F583E0FFEF6016906880E0FF74FE2FF56B
:1026C60082E43444F583E0FFEF6403601A90688087
:1026D600E0FF74EF2FF582E43450F583E0FF900CB1
:1026E6005EE0FEEFB506047F0180027F0090688001
:1026F600E0FE74BA2EF582E43456F583EFF0900CC2
:1027060060E0FFEF605B906880E0FF74D62FF58293
:10271600E43456F583E0FFEF6016906880E0FF74BE
:10272600FE2FF582E43444F583E0FFEF6403601A7C
:10273600906880E0FF74EF2FF582E43450F583E073
:10274600FF900C60E0FEEFB506047F0180027F007B
:10275600906880E0FE74D62EF582E43456F583EF59
:10276600F0906881E0FBA3E0FAA3E0F97582417579
:102776008300128E28FFEF30E744906880E0FF74F4
:10278600962FF582E4344EF583E0FFEF70199068DA
:1027960081E0FBA3E0FAA3E0F9758241758300129C
:1027A6008E28FFEF30E7047F0180027F009068806B
:1027B600E0FE74962EF582E4344EF583EFF09068D1
:1027C60080E0FF74EF2FF582E43450F583E0FFEFED
:1027D60064757040906880E0FF74A02FF582E43441
:1027E6004EF583E0FFEF7015906880E0FF74EF2FE1
:1027F600F582E43450F583E0FFEFB475047F018081
:10280600027F00906880E0FE74A02EF582E4344ECC
:10281600F583EFF0906880E0FF74EA2FF582E434E8
:1028260050F583E0FFEF6019906880E0FF74FE2F9B
:10283600F582E43444F583E0FFEF64037003022974
:1028460060906880E0FF74EF2FF582E43450F583E2
:10285600E0FFEF64137003022960906880E0FF7464
:10286600EF2FF582E43450F583E0FFEF6415700333
:10287600022960906880E0FF74EF2FF582E43450FF
:10288600F583E0FFEF64177003022960906880E02B
:10289600FF74EF2FF582E43450F583E0FFEF6420F8
:1028A6007003022960906880E0FF74EF2FF582E4E0
:1028B6003450F583E0FFEF643070030229609068BE
:1028C60080E0FF74EF2FF582E43450F583E0FFEFEC
:1028D60064427003022960906880E0FF74EF2FF570
:1028E60082E43450F583E0FFEF6444606D906880C5
:1028F600E0FF74EF2FF582E43450F583E0FFEF64D8
:10290600586057906880E0FF74EF2FF582E43450EA
:10291600F583E0FFEF64686041906880E0FF74EF44
:102926002FF582E43450F583E0FFEF6469602B9065
:102936006880E0FF74EF2FF582E43450F583E0FF02
:10294600EF64706015906880E0FF74EF2FF582E405
:102956003450F583E0FFEFB471047F0180027F00FD
:10296600906880E0FE74EA2EF582E43450F583EF39
:10297600F0906880E0FF74D32FF582E43450F5833D
:10298600E0FFEF6016906880E0FF74FE2FF582E4AA
:102996003444F583E0FFEF64036041906880E0FF14
:1029A60074EF2FF582E43450F583E0FFEF64216085
:1029B6002B906880E0FF74EF2FF582E43450F583A6
:1029C600E0FFEF64406015906880E0FF74EF2FF53C
:1029D60082E43450F583E0FFEFB454047F018002B3
:1029E6007F00906880E0FE74D32EF582E43450F5C3
:1029F60083EFF0906880E0FF74DE2FF582E43456B2
:102A0600F583E0FFEF6019906880E0FF74FE2FF514
:102A160082E43444F583E0FFEF64037003022B8AFB
:102A2600906880E0FF74EF2FF582E43450F583E080
:102A3600FFEF64147003022B8A906880E0FF74EF46
:102A46002FF582E43450F583E0FFEF64167003023D
:102A56002B8A906880E0FF74EF2FF582E43450F5FE
:102A660083E0FFEF64247003022B8A906880E0FF06
:102A760074EF2FF582E43450F583E0FFEF642570A0
:102A860003022B8A906880E0FF74EF2FF582E4340E
:102A960050F583E0FFEF64267003022B8A9068806E
:102AA600E0FF74EF2FF582E43450F583E0FFEF6426
:102AB600317003022B8A906880E0FF74EF2FF58255
:102AC600E43450F583E0FFEF64327003022B8A9002
:102AD6006880E0FF74EF2FF582E43450F583E0FF61
:102AE600EF64337003022B8A906880E0FF74EF2F47
:102AF600F582E43450F583E0FFEF64387003022B6F
:102B06008A906880E0FF74EF2FF582E43450F583F5
:102B1600E0FFEF6443606D906880E0FF74EF2FF58F
:102B260082E43450F583E0FFEF6449605790688093
:102B3600E0FF74EF2FF582E43450F583E0FFEF6495
:102B4600556041906880E0FF74EF2FF582E43450C1
:102B5600F583E0FFEF6472602B906880E0FF74EF0E
:102B66002FF582E43450F583E0FFEF64756015902D
:102B76006880E0FF74EF2FF582E43450F583E0FFC0
:102B8600EFB480047F0180027F00906880E0FE74CD
:102B9600DE2EF582E43456F583EFF0906880E0FF90
:102BA60074042FF582E43453F583E0FFEF6016904A
:102BB6006880E0FF74FE2FF582E43444F583E0FF7D
:102BC600EF6403606D906880E0FF74EF2FF582E498
:102BD6003450F583E0FFEF64126057906880E0FFA1
:102BE60074EF2FF582E43450F583E0FFEF6445601F
:102BF60041906880E0FF74EF2FF582E43450F5834E
:102C0600E0FFEF6453602B906880E0FF74EF2FF5D0
:102C160082E43450F583E0FFEF64896015906880A4
:102C2600E0FF74EF2FF582E43450F583E0FFEFB454
:102C360090047F0180027F00906880E0FE74042E7D
:102C4600F582E43453F583EFF0906880E0FF74FB7F
:102C56002FF582E43458F583E0FFEF702990688001
:102C6600E0FF74E82FF582E43462F583E0FFEF605D
:102C760015906880E0FF74F12FF582E43450F583F7
:102C86007409F0022E33906881E0FBA3E0FAA3E01A
:102C9600F9758244758300128E28FFEF30E5159092
:102CA6006880E0FF74F12FF582E43450F583740AEE
:102CB600F0022E33906880E0FF74EF2FF582E43443
:102CC60050F583E0FFEFB41815906880E0FF74F1CB
:102CD6002FF582E43450F5837401F0022E339068A8
:102CE60080E0FF74FE2FF582E43444F583E0FFEFC5
:102CF600B42715906880E0FF74F12FF582E4345014
:102D0600F5837402F0022E33906880E0FF74FE2F84
:102D1600F582E43444F583E0FFEFB404159068804F
:102D2600E0FF74F12FF582E43450F5837403F0026A
:102D36002E33906880E0FF74FE2FF582E43444F56C
:102D460083E0FFEF641A6015906880E0FF74FE2F41
:102D5600F582E43444F583E0FFEFB41B15906880F8
:102D6600E0FF74F12FF582E43450F5837404F00229
:102D76002E33906880E0FF74FE2FF582E43444F52C
:102D860083E0FFEFB40F15906880E0FF74F12FF534
:102D960082E43450F5837405F0022E33906880E0A7
:102DA600FF74FE2FF582E43444F583E0FFEFB405AB
:102DB60014906880E0FF74F12FF582E43450F583B7
:102DC6007406F08068906880E0FF74FE2FF582E458
:102DD6003444F583E0FFEFB40614906880E0FF7496
:102DE600F12FF582E43450F5837407F0803F906844
:102DF60081E0FBA3E0FAA3E0F97582417583001236
:102E06008E28FFEF30E414906880E0FF74F12FF510
:102E160082E43450F583740BF08012906880E0FFF2
:102E260074F12FF582E43450F583740CF0906880C9
:102E3600E0FF74832FF582E4340CF583E0FFEF6046
:102E460026906880E0FF74872FF582E4340CF583C2
:102E5600E0FFEF7012906880E0FF74922FF582E435
:102E6600340CF5837490F0906880E0FF74832FF53E
:102E760082E4340CF583E0FF906880E0FE74872ED0
:102E8600F582E4340CF583EFF0906880E0FF74314E
:102E96002FF582E43459F583E0FFEF603E906880B9
:102EA600E0FF74312FF582E43459F583E4F090683D
:102EB60080E0FF74922FF582E4340CF5837491F070
:102EC600906880E0FFEF7005906729E4F0906880D5
:102ED600E0FFEFB4010590672AE4F0906880E0FF18
:102EE600743E2FF582E43459F583E0FFEF602390BA
:102EF6006880E0FF743E2FF582E43459F583E4F0F0
:102F0600906880E0FF74922FF582E4340CF58374A8
:102F160092F0906880E0FF74922FF582E4340CF50D
:102F260083E0FFEF705C906880E0FF74E22FF5822B
:102F3600E43456F583E0FFEF6026906880E0FF7486
:102F4600EF2FF582E43456F583E0FFEF70129068B8
:102F560080E0FF74922FF582E4340CF5837401F05F
:102F6600906880E0FF74E22FF582E43456F583E042
:102F7600FF906880E0FE74EF2EF582E43456F58308
:102F8600EFF0906880E0FF74922FF582E4340CF540
:102F960083E0FFEF705C906880E0FF74C72FF582D6
:102FA600E43450F583E0FFEF6026906880E0FF741C
:102FB600DA2FF582E43450F583E0FFEF7012906863
:102FC60080E0FF74922FF582E4340CF5837402F0EE
:102FD600906880E0FF74C72FF582E43450F583E0F3
:102FE600FF906880E0FE74DA2EF582E43450F583B3
:102FF600EFF0906880E0FF74922FF582E4340CF5D0
:1030060083E0FFEF705C906880E0FF74D52FF58257
:10301600E43450F583E0FFEF6026906880E0FF74AB
:10302600E42FF582E43450F583E0FFEF70129068E8
:1030360080E0FF74922FF582E4340CF5837403F07C
:10304600906880E0FF74D52FF582E43450F583E074
:10305600FF906880E0FE74E42EF582E43450F58338
:10306600EFF0906880E0FF74922FF582E4340CF55F
:1030760083E0FFEF705C906880E0FF747A2FF58242
:10308600E4340CF583E0FFEF6026906880E0FF747F
:103096007F2FF582E4340CF583E0FFEF7012906821
:1030A60080E0FF74922FF582E4340CF5837404F00B
:1030B600906880E0FF747A2FF582E4340CF583E0A3
:1030C600FF906880E0FE747F2EF582E4340CF58371
:1030D600EFF0906880E0FF74922FF582E4340CF5EF
:1030E60083E0FFEF705C906880E0FF74982FF582B4
:1030F600E4344EF583E0FFEF6026906880E0FF74CD
:10310600A42FF582E4344EF583E0FFEF7012906849
:1031160080E0FF74922FF582E4340CF5837405F099
:10312600906880E0FF74982FF582E4344EF583E0D2
:10313600FF906880E0FE74A42EF582E4344EF58399
:10314600EFF0906880E0FF74922FF582E4340CF57E
:1031560083E0FFEF705C906880E0FF74DA2FF58201
:10316600E43456F583E0FFEF6026906880E0FF7454
:10317600E82FF582E43456F583E0FFEF701290688D
:1031860080E0FF74922FF582E4340CF5837406F028
:10319600906880E0FF74DA2FF582E43456F583E018
:1031A600FF906880E0FE74E82EF582E43456F583DD
:1031B600EFF0906880E0FF74922FF582E4340CF50E
:1031C60083E0FFEF705C906880E0FF740E2FF5825D
:1031D600E43455F583E0FFEF6026906880E0FF74E5
:1031E600222FF582E43455F583E0FFEF70129068E4
:1031F60080E0FF74922FF582E4340CF5837407F0B7
:10320600906880E0FF740E2FF582E43455F583E074
:10321600FF906880E0FE74222EF582E43455F58333
:10322600EFF0906880E0FF74922FF582E4340CF59D
:1032360083E0FFEF705C906880E0FF74FC2FF582FE
:10324600E43450F583E0FFEF6026906880E0FF7479
:10325600062FF582E43453F583E0FFEF7012906891
:1032660080E0FF74922FF582E4340CF5837408F045
:10327600906880E0FF74FC2FF582E43450F583E01B
:10328600FF906880E0FE74062EF582E43453F583E1
:10329600EFF0906880E0FF74922FF582E4340CF52D
:1032A60083E0FFEF705C906880E0FF744E2FF5823C
:1032B600E4340CF583E0FFEF6026906880E0FF744D
:1032C600522FF582E4340CF583E0FFEF701290681C
:1032D60080E0FF74922FF582E4340CF5837410F0CD
:1032E600906880E0FF744E2FF582E4340CF583E09D
:1032F600FF906880E0FE74522EF582E4340CF5836C
:10330600EFF0906880E0FF74922FF582E4340CF5BC
:1033160083E0FFEF705C906880E0FF74A62FF58273
:10332600E4340CF583E0FFEF6026906880E0FF74DC
:10333600AA2FF582E4340CF583E0FFEF7012906853
:1033460080E0FF74922FF582E4340CF5837420F04C
:10335600906880E0FF74A62FF582E4340CF583E0D4
:10336600FF906880E0FE74AA2EF582E4340CF583A3
:10337600EFF0906880E0FF74922FF582E4340CF54C
:1033860083E0FFEF705C906880E0FF74852FF58224
:10339600E4340CF583E0FFEF6026906880E0FF746C
:1033A6008B2FF582E4340CF583E0FFEF7012906802
:1033B60080E0FF74922FF582E4340CF5837421F0DB
:1033C600906880E0FF74852FF582E4340CF583E085
:1033D600FF906880E0FE748B2EF582E4340CF58352
:1033E600EFF0906880E0FF74922FF582E4340CF5DC
:1033F60083E0FFEF705C906880E0FF74902FF582A9
:10340600E43409F583E0FFEF6026906880E0FF74FE
:103416008A2FF582E4340AF583E0FFEF7012906894
:1034260080E0FF74922FF582E4340CF5837422F069
:10343600906880E0FF74902FF582E43409F583E00C
:10344600FF906880E0FE748A2EF582E4340AF583E4
:10345600EFF0906880E0FF74922FF582E4340CF56B
:1034660083E0FFEF705C906880E0FF749D2FF5822B
:10347600E43456F583E0FFEF6026906880E0FF7441
:10348600AC2FF582E43456F583E0FFEF70129068B6
:1034960080E0FF74922FF582E4340CF5837423F0F8
:1034A600906880E0FF749D2FF582E43456F583E042
:1034B600FF906880E0FE74AC2EF582E43456F58306
:1034C600EFF0906880E0FF74922FF582E4340CF5FB
:1034D60083E0FFEF705C906880E0FF74F32FF58265
:1034E600E43450F583E0FFEF6026906880E0FF74D7
:1034F600FA2FF582E43450F583E0FFEF70129068FE
:1035060080E0FF74922FF582E4340CF5837424F086
:10351600906880E0FF74F32FF582E43450F583E081
:10352600FF906880E0FE74FA2EF582E43450F5834D
:10353600EFF0906880E0FF74922FF582E4340CF58A
:1035460083E0FFEF705C906880E0FF742A2FF582BD
:10355600E43455F583E0FFEF6026906880E0FF7461
:103566009B2FF582E43456F583E0FFEF70129068E6
:1035760080E0FF74922FF582E4340CF5837425F015
:10358600906880E0FF742A2FF582E43455F583E0D5
:10359600FF906880E0FE749B2EF582E43456F58336
:1035A600EFF0906880E0FF74922FF582E4340CF51A
:1035B60083E0FFEF705C906880E0FF74312FF58246
:1035C600E43455F583E0FFEF6026906880E0FF74F1
:1035D600A62FF582E43456F583E0FFEF701290686B
:1035E60080E0FF74922FF582E4340CF5837426F0A4
:1035F600906880E0FF74312FF582E43455F583E05E
:10360600FF906880E0FE74A62EF582E43456F583BA
:10361600EFF0906880E0FF74922FF582E4340CF5A9
:1036260083E0FFEF705C906880E0FF74992FF5826D
:10363600E43456F583E0FFEF6026906880E0FF747F
:10364600AA2FF582E43456F583E0FFEF70129068F6
:1036560080E0FF74922FF582E4340CF5837427F032
:10366600906880E0FF74992FF582E43456F583E084
:10367600FF906880E0FE74AA2EF582E43456F58346
:10368600EFF0906880E0FF74922FF582E4340CF539
:1036960083E0FFEF705C906880E0FF74A42FF582F2
:1036A600E43456F583E0FFEF6026906880E0FF740F
:1036B600B52FF582E43456F583E0FFEF701290687B
:1036C60080E0FF74922FF582E4340CF5837428F0C1
:1036D600906880E0FF74A42FF582E43456F583E009
:1036E600FF906880E0FE74B52EF582E43456F583CB
:1036F600EFF0906880E0FF74922FF582E4340CF5C9
:1037060083E0FFEF705C906880E0FF74A82FF5827D
:10371600E43456F583E0FFEF6026906880E0FF749E
:10372600BC2FF582E43456F583E0FFEF7012906803
:1037360080E0FF74922FF582E4340CF5837429F04F
:10374600906880E0FF74A82FF582E43456F583E094
:10375600FF906880E0FE74BC2EF582E43456F58353
:10376600EFF0906880E0FF74922FF582E4340CF558
:1037760083E0FFEF705C906880E0FF74B32FF58202
:10378600E43456F583E0FFEF6026906880E0FF742E
:10379600D82FF582E43456F583E0FFEF7012906877
:1037A60080E0FF74922FF582E4340CF5837430F0D8
:1037B600906880E0FF74B32FF582E43456F583E019
:1037C600FF906880E0FE74D82EF582E43456F583C7
:1037D600EFF0906880E0FF74922FF582E4340CF5E8
:1037E60083E0FFEF705C906880E0FF74BA2FF5828B
:1037F600E43456F583E0FFEF6026906880E0FF74BE
:10380600E02FF582E43456F583E0FFEF70129068FE
:1038160080E0FF74922FF582E4340CF5837431F066
:10382600906880E0FF74BA2FF582E43456F583E0A1
:10383600FF906880E0FE74E02EF582E43456F5834E
:10384600EFF0906880E0FF74922FF582E4340CF577
:1038560083E0FFEF705C906880E0FF74D62FF582FE
:10386600E43456F583E0FFEF6026906880E0FF744D
:10387600E62FF582E43456F583E0FFEF7012906888
:1038860080E0FF74922FF582E4340CF5837432F0F5
:10389600906880E0FF74D62FF582E43456F583E015
:1038A600FF906880E0FE74E62EF582E43456F583D8
:1038B600EFF0906880E0FF74922FF582E4340CF507
:1038C60083E0FFEF705C906880E0FF74962FF582CE
:1038D600E4344EF583E0FFEF6026906880E0FF74E5
:1038E600A22FF582E4344EF583E0FFEF7012906864
:1038F60080E0FF74922FF582E4340CF5837433F084
:10390600906880E0FF74962FF582E4344EF583E0EC
:10391600FF906880E0FE74A22EF582E4344EF583B3
:10392600EFF0906880E0FF74922FF582E4340CF596
:1039360083E0FFEF705C906880E0FF74A02FF58253
:10394600E4344EF583E0FFEF6026906880E0FF7474
:10395600B02FF582E4344EF583E0FFEF70129068E5
:1039660080E0FF74922FF582E4340CF5837434F012
:10397600906880E0FF74A02FF582E4344EF583E072
:10398600FF906880E0FE74B02EF582E4344EF58335
:10399600EFF0906880E0FF74922FF582E4340CF526
:1039A60083E0FFEF705C906880E0FF74EA2FF58299
:1039B600E43450F583E0FFEF6026906880E0FF7402
:1039C600EC2FF582E43450F583E0FFEF7012906837
:1039D60080E0FF74922FF582E4340CF5837435F0A1
:1039E600906880E0FF74EA2FF582E43450F583E0B6
:1039F600FF906880E0FE74EC2EF582E43450F58387
:103A0600EFF0906880E0FF74922FF582E4340CF5B5
:103A160083E0FFEF705C906880E0FF74D32FF5823F
:103A2600E43450F583E0FFEF6026906880E0FF7491
:103A3600E22FF582E43450F583E0FFEF70129068D0
:103A460080E0FF74922FF582E4340CF5837436F02F
:103A5600906880E0FF74D32FF582E43450F583E05C
:103A6600FF906880E0FE74E22EF582E43450F58320
:103A7600EFF0906880E0FF74922FF582E4340CF545
:103A860083E0FFEF705C906880E0FF74DE2FF582C4
:103A9600E43456F583E0FFEF6026906880E0FF741B
:103AA600ED2FF582E43456F583E0FFEF701290684F
:103AB60080E0FF74922FF582E4340CF5837437F0BE
:103AC600906880E0FF74DE2FF582E43456F583E0DB
:103AD600FF906880E0FE74ED2EF582E43456F5839F
:103AE600EFF0906880E0FF74922FF582E4340CF5D5
:103AF60083E0FFEF705C906880E0FF74042FF5822E
:103B0600E43453F583E0FFEF6026906880E0FF74AD
:103B16000C2FF582E43455F583E0FFEF70129068C0
:103B260080E0FF74922FF582E4340CF5837438F04C
:103B3600906880E0FF74042FF582E43453F583E047
:103B4600FF906880E0FE740C2EF582E43455F58310
:103B5600EFF0906880E0FF74922FF582E4340CF564
:103B660083E0FFEFD39400402C906880E0FF7492CE
:103B76002FF582E4340CF583E0FFEFC3945A501519
:103B8600906880E0FF749C2FF582E4344EF58374D0
:103B960001F0023E5D906880E0FF74E22FF582E45A
:103BA6003456F583E0FFEF6003023E0A906880E03A
:103BB600FF74C72FF582E43450F583E0FFEF60030E
:103BC600023E0A906880E0FF74D52FF582E43450F7
:103BD600F583E0FFEF6003023E0A906880E0FF7421
:103BE6007A2FF582E4340CF583E0FFEF6003023EA2
:103BF6000A906880E0FF74982FF582E4344EF583CE
:103C0600E0FFEF6003023E0A906880E0FF74DA2F5F
:103C1600F582E43456F583E0FFEF6003023E0A9036
:103C26006880E0FF740E2FF582E43455F583E0FFDB
:103C3600EF6003023E0A906880E0FF74FC2FF58275
:103C4600E43450F583E0FFEF6003023E0A9068809B
:103C5600E0FF744E2FF582E4340CF583E0FFEF604D
:103C660003023E0A906880E0FF74A62FF582E434D2
:103C76000CF583E0FFEF6003023E0A906880E0FFE8
:103C860074852FF582E4340CF583E0FFEF600302C0
:103C96003E0A906880E0FF74902FF582E43409F5BF
:103CA60083E0FFEF6003023E0A906880E0FF749DA8
:103CB6002FF582E43456F583E0FFEF6003023E0AF7
:103CC600906880E0FF74F32FF582E43450F583E0CA
:103CD600FFEF6003023E0A906880E0FF742A2FF52A
:103CE60082E43455F583E0FFEF6003023E0A9068F4
:103CF60080E0FF74312FF582E43455F583E0FFEF61
:103D06006003023E0A906880E0FF74992FF582E412
:103D16003456F583E0FFEF6003023E0A906880E0C8
:103D2600FF74A42FF582E43456F583E0FFEF6003B9
:103D3600023E0A906880E0FF74A82FF582E43456AC
:103D4600F583E0FFEF6003023E0A906880E0FF74AF
:103D5600B32FF582E43456F583E0FFEF6003023EAD
:103D66000A906880E0FF74BA2FF582E43456F58332
:103D7600E0FFEF6003023E0A906880E0FF74D62FF2
:103D8600F582E43456F583E0FFEF7078906880E0C2
:103D9600FF74962FF582E4344EF583E0FFEF7064EE
:103DA600906880E0FF74A02FF582E4344EF583E03E
:103DB600FFEF7050906880E0FF74EA2FF582E434DC
:103DC60050F583E0FFEF703C906880E0FF74D32FDE
:103DD600F582E43450F583E0FFEF7028906880E0C8
:103DE600FF74DE2FF582E43456F583E0FFEF70149E
:103DF600906880E0FF74042FF582E43453F583E085
:103E0600FFEF60047F0180027F00906884EFF090EE
:103E16006880E0FF749C2FF582E4344EF583E0FF62
:103E2600906884E0FEEE70047E0180027E00EE5F04
:103E3600FFEF6023906880E0FF749C2FF582E434E6
:103E46004EF583E4F0906880E0FF74922FF582E4EB
:103E5600340CF58374FFF0906880E0FF74922FF5C0
:103E660082E4340CF583E0FFEF6003023FBF906805
:103E760080E0FF74F82FF582E43450F583E0FF907C
:103E86006880E0FE74F12EF582E43450F583E0FE9E
:103E9600EE6F7003023FBF906880E0FF74F12FF56C
:103EA60082E43450F583E0FF906880E0FE74F82EDB
:103EB600F582E43450F583EFF0906880E0FF74F10A
:103EC6002FF582E43450F583E0FFEF128F393F85FA
:103ED600013F0B023F20033F35043F49053F5D0686
:103EE6003F71073EF6093F990A3FAD0B00003FBF01
:103EF600906880E0FF74922FF582E4340CF58374A9
:103F060041F0023FBF906880E0FF74922FF582E493
:103F1600340CF5837440F0023FBF906880E0FF7474
:103F2600922FF582E4340CF5837443F0023FBF9080
:103F36006880E0FF74922FF582E4340CF5837444B4
:103F4600F08076906880E0FF74922FF582E4340C5E
:103F5600F5837445F08062906880E0FF74922FF5D7
:103F660082E4340CF5837446F0804E906880E0FF5E
:103F760074922FF582E4340CF5837447F0803A90FE
:103F86006880E0FF74922FF582E4340CF583744266
:103F9600F08026906880E0FF74922FF582E4340C5E
:103FA600F5837448F08012906880E0FF74922FF5D4
:103FB60082E4340CF5837449F0906880E0FF74F174
:103FC6002FF582E43450F583E014F0906880E0FF2A
:103FD60074F12FF582E43450F583E0FFEFD39407B4
:103FE6004012906880E0FF74F12FF582E43450F5BA
:103FF600837407F0906880E0FF74202FF582E43424
:1040060055F583E4F0906880E0FF74262FF582E48E
:104016003455F583E4F0906881E0FBA3E0FAA3E071
:10402600F9758226758300128E28FFEFD39400401F
:1040360017906880E0FF74202FF582E43455F583ED
:10404600E0FFEF4401FFEFF0906881E0FBA3E0FAA8
:10405600A3E0F9758241758300128E28FFEF30E0E8
:1040660017906880E0FF74202FF582E43455F583BD
:10407600E0FFEF4402FFEFF0906881E0FBA3E0FA77
:10408600A3E0F9758241758300128E28FFEF30E1B7
:1040960017906880E0FF74202FF582E43455F5838D
:1040A600E0FFEF4404FFEFF0906881E0FBA3E0FA45
:1040B600A3E0F9758231758300128E28FFEF601731
:1040C600906880E0FF74202FF582E43455F583E094
:1040D600FFEF4408FFEFF0906881E0FBA3E0FAA34E
:1040E600E0F9758228758300128E28FFEF6017901D
:1040F6006880E0FF74202FF582E43455F583E0FFF5
:10410600EF4410FFEFF0906881E0FBA3E0FAA3E034
:10411600F975821E758300128E28FFEF601790686E
:1041260080E0FF74202FF582E43455F583E0FFEF3D
:104136004420FFEFF0906881E0FBA3E0FAA3E0F9EA
:10414600758244758300128E28FFEF30E71790685A
:1041560080E0FF74202FF582E43455F583E0FFEF0D
:104166004440FFEFF0906881E0FBA3E0FAA3E0F99A
:10417600758244758300128E28FFEF30E61790682B
:1041860080E0FF74202FF582E43455F583E0FFEFDD
:104196004480FFEFF0906881E0FBA3E0FAA3E0F92A
:1041A60075822A758300128E28FFEF60179068804B
:1041B600E0FF74262FF582E43455F583E0FFEF44E3
:1041C60001FFEFF0906881E0FBA3E0FAA3E0F97548
:1041D6008229758300128E28FFEF6017906880E0B1
:1041E600FF74262FF582E43455F583E0FFEF440291
:1041F600FFEFF0906881E0FBA3E0FAA3E0F9758297
:1042060027758300128E28FFEF6017906880E0FF05
:1042160074262FF582E43455F583E0FFEF4408FF5A
:10422600EFF0906880E0FF74262FF582E43455F5B0
:1042360083C083C082E0FF906881E0FBA3E0FAA31D
:10424600E0F9758244758300128E28FEEE5410FE46
:10425600EF4EFFD082D083EFF0906881E0FBA3E0C1
:10426600FAA3E0F9758241758300128E28FFEF30BC
:10427600E517906880E0FF74262FF582E43455F543
:1042860083E0FFEF4440FFEFF0900C5FE0FFEF5458
:10429600FBFF906884EFF0900C5FE0FFEF30E10EDB
:1042A600906884E0FFEF4404FF906884EFF0906824
:1042B60080E0FF74202FF582E43455F583E0FF900B
:1042C6006884E0FEEF5EFF906880E0FE740A2EF5DB
:1042D60082E43455F583EFF0906880E0FF74262F72
:1042E600F582E43455F583E0FF9050F7E0FEEF5E8B
:1042F600FF906880E0FE748E2EF582E4340AF58322
:10430600EFF0900C5FE0FFEF30E226906881E0FB73
:10431600A3E0FAA3E0F9758243758300128E28FFA5
:10432600906880E0FE74A22EF582E43456F583EFA1
:10433600F0906880E0FF74E82FF582E43462F5833C
:10434600E0FFEF7014906880E0FF74362FF582E48A
:104356003459F583E0FFEF6019906880E0FF7492AE
:104366002FF582E4340CF583E0FFEF64416003022D
:1043760046D5906880E0FF741B2FF582E43467F51C
:1043860083E0FFEF60030246D5906880E0FF7492F9
:104396002FF582E4340CF583E0FFEF700302450E3F
:1043A600906880E0FF74922FF582E4340CF583E088
:1043B600FFEFB4FF11906880E0FF74922FF582E45E
:1043C600340CF583E4F0906880E0FF74FE2FF582EC
:1043D600E43444F583E0FFEFB40419906880E0FF0D
:1043E60074922FF582E4340CF583E0FFEF644360AA
:1043F600030246D5906880E0FFEF75F00CA42477A1
:10440600F582E43409F583AF82AE83C006C0079017
:104416006880E0FF7E00EF7F00FE74B42FF58274A3
:104426004E3EF583AD82AC83906880E0FBD007D02A
:1044360006129C6F906880E0FF7E007C047DB312BC
:104446008E89740B2FF974003EFA7B01C003C002FB
:10445600C001906880E0FF7E0CEF8EF0A4FFAEF006
:1044660074772FF974093EFA7B01C003C002C001BC
:104476007B017A687935A801AC02AD03D001D00280
:10448600D0037E007F0C128DE9D001D002D003123A
:10449600AAA2906880E0FF7E007C047DB3128E891C
:1044A600740A2FF974453EFA7B01C003C002C001AD
:1044B600906880E0FF74572FF582E4345BF583E063
:1044C600FFC007906880E0FF7E0CEF8EF0A4FFAE81
:1044D600F074772FF974093EFA7B01C003C002C05D
:1044E600017B017A687915A801AC02AD03D001D031
:1044F60002D0037E007F0C128DE9D007D001D002D6
:10450600D00312A4200246D5906880E0FF741E2FC7
:10451600F582E43455F583E0FF906880E0FE740A86
:104526002EF582E43455F583E0FEEE6F704F906809
:1045360080E0FF74942FF582E4340AF583E0FF905F
:104546006880E0FE748E2EF582E4340AF583E0FE80
:10455600EEB50729906880E0FF74B12FF582E43448
:1045660056F583E0FF906880E0FE74A22EF582E4A3
:104576003456F583E0FEEE6F70030246D5906880F0
:10458600E0FF74922FF582E4340CF5837499F09071
:104596006880E0FFEF75F00CA42477F582E4340917
:1045A600F583AF82AE83C006C007906880E0FF7EC9
:1045B60000EF7F00FE74B42FF582744E3EF583AD96
:1045C60082AC83906880E0FBD007D006129C6F9087
:1045D6006880E0FF7E007C047DB3128E89740A2F0A
:1045E600F974453EFA7B01C003C002C001906880A1
:1045F600E0FF74572FF582E4345BF583E0FFC007D4
:10460600906880E0FF7E0CEF8EF0A4FFAEF074772A
:104616002FF974093EFA7B01C003C002C0017B0179
:104626007A687915A801AC02AD03D001D002D00397
:104636007E007F0C128DE9D007D001D002D0031284
:10464600A420906880E0FF74DC2FF582E43450F5F6
:1046560083E0FFEF20E21A906880E0FFEF25E02478
:10466600C9F582E43450F583E0FEA3E0FFEF4E6027
:104676005E906880E0FF7E007C047DB3128E8974B4
:104686000B2FF974003EFA7B01C003C002C00190F3
:104696006880E0FF7E0CEF8EF0A4FFAEF074772FFB
:1046A600F974093EFA7B01C003C002C0017B017A9E
:1046B600687935A801AC02AD03D001D002D0037EE3
:1046C600007F0C128DE9D001D002D00312AAA2906D
:1046D6006880E0FF740A2FF582E43455F583E0FF25
:1046E600906880E0FE741E2EF582E43455F583EF63
:1046F600F0906880E0FF748E2FF582E4340AF5832B
:10470600E0FF906880E0FE74942EF582E4340AF5AA
:1047160083EFF0906880E0FF74A22FF582E43456B0
:10472600F583E0FF906880E0FE74B12EF582E434F4
:1047360056F583EFF0906880E0FF74922FF582E4DF
:06474600340CF583E4F0E1
:01474C00224A
:10BAE100906928EFF0906928E0FF74002FF582E457
:10BAF1003445F583E0FFEF700302BBA2906928E0B3
:10BB0100FF741B2FF582E43467F583E0FFEF6003D8
:10BB110002BBA2906928E0FF74002FF582E434454E
:10BB2100F583E4F0906928E0FFEF75F014A4240791
:10BB3100F582E43459F583AF82AE83906928E0FD44
:10BB4100128033906928E0FF7ECBEF8EF0A4FFAE28
:10BB5100F074B32FF9740A3EFA7B01C003C002C02E
:10BB610001906928E0FF7E14EF8EF0A4FFAEF0741F
:10BB7100072FF974593EFA7B01C003C002C0017B53
:10BB8100017A6779A9A801AC02AD03D001D002D036
:10BB9100037E007F14128DE9D001D002D00312ABD5
:02BBA100E82298
:105DB6009068C2EFF09068C3EBF0A3EAF0A3E9F0B5
:105DC6009068C3E0FBA3E0FAA3E0F9758226758329
:105DD60000128E28FFEFC3940350149068C2E0FFB0
:105DE60074F72FF582E43458F5837401F08011902E
:105DF60068C2E0FF74F72FF582E43458F583E4F0C7
:105E06009068C3E0FBA3E0FAA3E0F97582317583DD
:105E160000128E28FFEF60189068C3E0FBA3E0FA3B
:105E2600A3E0F9758227758300128E28FFEF7014A0
:105E36009068C2E0FF74F72FF582E43458F583E0EA
:105E4600FFEF70139068C2E0FF748C2FF582E43484
:105E56000AF583E4F080129068C2E0FF748C2FF597
:105E660082E4340AF5837401F09060E3E0FFEF60AA
:105E7600030267889068C3E0FBA3E0FAA3E0F97524
:105E8600821D758300128E28FFEF128F395ED304B0
:105E96005EFD056049065FE4085FF909605D0C5F19
:105EA6007B105F90115F12195F271A5F3C1B600D14
:105EB6001F5FBA245FCF255EE8335F51345F6635D6
:105EC6005FA53760213960353A000060719068C27D
:105ED600E0FF74422FF582E43459F5837403F0022F
:105EE60060829068C2E0FF74422FF582E43459F56F
:105EF600837403F00260829068C2E0FF74422FF55B
:105F060082E43459F5837404F00260829068C2E03A
:105F1600FF74422FF582E43459F583740FF0026062
:105F2600829068C2E0FF74422FF582E43459F5830B
:105F3600740FF00260829068C2E0FF74422FF5820F
:105F4600E43459F583740FF00260829068C2E0FF72
:105F560074422FF582E43459F5837424F00260828A
:105F66009068C2E0FF74422FF582E43459F58374D9
:105F760025F00260829068C2E0FF74422FF582E449
:105F86003459F5837405F00260829068C2E0FF74AC
:105F9600422FF582E43459F5837405F0026082904D
:105FA60068C2E0FF74422FF582E43459F583742702
:105FB600F00260829068C2E0FF74422FF582E434FA
:105FC60059F583741AF00260829068C2E0FF744249
:105FD6002FF582E43459F583741AF00260829068D2
:105FE600C2E0FF74422FF582E43459F5837406F05B
:105FF6000260829068C2E0FF74422FF582E4345951
:10600600F5837406F080759068C2E0FF74422FF540
:1060160082E43459F5837428F080619068C2E0FF09
:1060260074422FF582E43459F5837422F0804D9042
:1060360068C2E0FF74422FF582E43459F583742276
:10604600F080399068C2E0FF74422FF582E434593B
:10605600F5837404F080259068C2E0FF74422FF542
:1060660082E43459F5837408F080119068C2E0FF29
:1060760074422FF582E43459F583E4F09068C3E066
:10608600FBA3E0FAA3E0F975820C758300128E2853
:10609600FFEF128F3962A01161F812640515626173
:1060A6001661E317657F19620D1A637220618F21ED
:1060B60061B92263332362222462372563B12664E1
:1060C6002F2763F02863C62962762A65942B64AD70
:1060D6002C65FD2D61A42E635D3063483163093361
:1060E600628B3962B54062CA41617A426483436415
:1060F6005944661248646E49670E59641A6064C250
:106106007164D77265017364447465167565E888B1
:1061160063DB9061CE91638792639C956627996550
:10612600BE9A64989B631E9D65D3A1674DA267388E
:10613600A362DFA462F4A565A9A6656AA866A5A9F7
:1061460066BAAA6651AB667BAC624CB36690B4661F
:1061560066B5652BB66540B76555B866E4B966CFD2
:10616600BA66F9BE6761C0663CC264ECC36723C405
:10617600000067759068C2E0FF74982FF582E434DA
:106186000AF5837410F00267D49068C2E0FF749831
:106196002FF582E4340AF5837411F00267D490680F
:1061A600C2E0FF74982FF582E4340AF5837411F087
:1061B6000267D49068C2E0FF74982FF582E4340A2F
:1061C600F5837412F00267D49068C2E0FF74982FCA
:1061D600F582E4340AF5837413F00267D49068C23A
:1061E600E0FF74982FF582E4340AF5837414F00204
:1061F60067D49068C2E0FF74982FF582E4340AF5FC
:10620600837416F00267D49068C2E0FF74982FF585
:1062160082E4340AF5837417F00267D49068C2E00A
:10622600FF74982FF582E4340AF5837418F0026738
:10623600D49068C2E0FF74982FF582E4340AF5839F
:106246007419F00267D49068C2E0FF74982FF58243
:10625600E4340AF5837423F00267D49068C2E0FF41
:1062660074982FF582E4340AF5837425F00267D416
:106276009068C2E0FF74982FF582E4340AF58374BF
:1062860027F00267D49068C2E0FF74982FF582E485
:10629600340AF5837428F00267D49068C2E0FF746C
:1062A600982FF582E4340AF5837429F00267D490B6
:1062B60068C2E0FF74982FF582E4340AF5837435DA
:1062C600F00267D49068C2E0FF74982FF582E43438
:1062D6000AF5837435F00267D49068C2E0FF7498BB
:1062E6002FF582E4340AF5837436F00267D4906899
:1062F600C2E0FF74982FF582E4340AF5837436F011
:106306000267D49068C2E0FF74982FF582E4340ADD
:10631600F5837437F00267D49068C2E0FF74982F53
:10632600F582E4340AF5837439F00267D49068C2C2
:10633600E0FF74982FF582E4340AF5837439F0028D
:1063460067D49068C2E0FF74982FF582E4340AF5AA
:10635600837440F00267D49068C2E0FF74982FF50A
:1063660082E4340AF5837441F00267D49068C2E08F
:10637600FF74982FF582E4340AF5837442F00267BD
:10638600D49068C2E0FF74982FF582E4340AF5834E
:106396007444F00267D49068C2E0FF74982FF582C7
:1063A600E4340AF5837445F00267D49068C2E0FFCE
:1063B60074982FF582E4340AF5837445F00267D4A5
:1063C6009068C2E0FF74982FF582E4340AF583746E
:1063D60046F00267D49068C2E0FF74982FF582E415
:1063E600340AF5837447F00267D49068C2E0FF74FC
:1063F600982FF582E4340AF5837448F00267D49046
:1064060068C2E0FF74982FF582E4340AF583744974
:10641600F00267D49068C2E0FF74982FF582E434E6
:106426000AF5837450F00267D49068C2E0FF74984E
:106436002FF582E4340AF5837451F00267D490682C
:10644600C2E0FF74982FF582E4340AF5837451F0A4
:106456000267D49068C2E0FF74982FF582E4340A8C
:10646600F5837452F00267D49068C2E0FF74982FE7
:10647600F582E4340AF5837452F00267D49068C258
:10648600E0FF74982FF582E4340AF5837453F00222
:1064960067D49068C2E0FF74982FF582E4340AF559
:1064A600837457F00267D49068C2E0FF74982FF5A2
:1064B60082E4340AF5837459F00267D49068C2E026
:1064C600FF74982FF582E4340AF5837460F002674E
:1064D600D49068C2E0FF74982FF582E4340AF583FD
:1064E6007462F00267D49068C2E0FF74982FF58258
:1064F600E4340AF5837462F00267D49068C2E0FF60
:1065060074982FF582E4340AF5837463F00267D435
:106516009068C2E0FF74982FF582E4340AF583741C
:1065260064F00267D49068C2E0FF74982FF582E4A5
:10653600340AF5837465F00267D49068C2E0FF748C
:10654600982FF582E4340AF5837466F00267D490D6
:1065560068C2E0FF74982FF582E4340AF583746705
:10656600F00267D49068C2E0FF74982FF582E43495
:106576000AF5837467F00267D49068C2E0FF7498E6
:106586002FF582E4340AF5837471F00267D49068BB
:10659600C2E0FF74982FF582E4340AF5837473F031
:1065A6000267D49068C2E0FF74982FF582E4340A3B
:1065B600F5837474F00267D49068C2E0FF74982F74
:1065C600F582E4340AF5837475F00267D49068C2E4
:1065D600E0FF74982FF582E4340AF5837476F002AE
:1065E60067D49068C2E0FF74982FF582E4340AF508
:1065F600837478F00267D49068C2E0FF74982FF530
:1066060082E4340AF5837479F00267D49068C2E0B4
:10661600FF74982FF582E4340AF5837479F00267E3
:10662600D49068C2E0FF74982FF582E4340AF583AB
:106636007480F00267D49068C2E0FF74982FF582E8
:10664600E4340AF5837480F00267D49068C2E0FFF0
:1066560074982FF582E4340AF5837481F00267D4C6
:106666009068C2E0FF74982FF582E4340AF58374CB
:1066760081F00267D49068C2E0FF74982FF582E437
:10668600340AF5837482F00267D49068C2E0FF741E
:10669600982FF582E4340AF5837482F00267D49069
:1066A60068C2E0FF74982FF582E4340AF583748497
:1066B600F00267D49068C2E0FF74982FF582E43444
:1066C6000AF5837485F00267D49068C2E0FF749877
:1066D6002FF582E4340AF5837486F00267D4906855
:1066E600C2E0FF74982FF582E4340AF5837487F0CC
:1066F6000267D49068C2E0FF74982FF582E4340AEA
:10670600F5837488F00267D49068C2E0FF74982F0E
:10671600F582E4340AF5837489F00267D49068C27E
:10672600E0FF74982FF582E4340AF5837490F00242
:1067360067D49068C2E0FF74982FF582E4340AF5B6
:10674600837491F00267D49068C2E0FF74982FF5C5
:1067560082E4340AF5837492F080739068C2E0FF95
:1067660074982FF582E4340AF5837493F0805F9071
:1067760068C2E0FF74982FF582E4340AF583E4F0EA
:10678600804C9068C3E0FBA3E0FAA3E0F975820CA5
:10679600758300128E28FF9068C2E0FE74982EF56D
:1067A60082E4340AF583EFF09068C3E0FBA3E0FAD5
:1067B600A3E0F975821D758300128E28FF9068C2CA
:1067C600E0FE74422EF582E43459F583EFF09068CA
:1067D600C2E0FF74982FF582E4340AF583E0FFEFF8
:1067E60060369068C2E0FF74982FF582E4340AF5AB
:1067F60083E0FF9068C2E0FE74EF2EF582E4345029
:10680600F583EFF09068C2E0FF742E2FF582E43432
:1068160055F583E4F00268AF9068C2E0FF742E2F4E
:10682600F582E43455F583E004F09068C2E0FF7425
:10683600FE2FF582E43444F583E0FFEF64276041E0
:106846009068C2E0FF74FE2FF582E43444F583E0DD
:10685600FFEF6424602B9068C2E0FF74FE2FF58280
:10686600E43444F583E0FFEF642560159068C2E0E8
:10687600FF74FE2FF582E43444F583E0FFEFB404A1
:10688600289068C2E0FF742E2FF582E43455F58314
:10689600E0FFEFD3940640119068C2E0FF74EF2F3B
:1068A600F582E43450F583E4F09068C2E0FF74EFBB
:1068B6002FF582E43450F583E0FFEF6450601590C5
:1068C60068C2E0FF74EF2FF582E43450F583E0FFF1
:1068D600EFB451129068C2E0FF74B22FF582E4342F
:1068E6004EF5837401F09068C2E0FF74422FF58282
:1068F600E43459F583E0FFEFB427119068C2E0FF56
:1069060074B22FF582E4344EF583E4F09068C2E069
:10691600FF74B22FF582E4344EF583E0FFEF702367
:106926009068C2E0FF74422FF582E43459F583E0A3
:10693600FF9068C2E0FE74FE2EF582E43444F583CF
:10694600EFF0229068C2E0FF74FE2FF582E4344433
:06695600F5837403F0223A
:108033009068ECEEF0A3EFF09068EEEDF09068EE50
:10804300E0FFEF75F018A42400F582E43465F583AE
:10805300E0FEA3E0FF9068ECE0FCA3E0FD8D828CE2
:1080630083EFF09068EEE0FFEF75F018A42402F5BB
:1080730082E43465F583E0FEA3E0FF9068ECE0FC66
:10808300A3E0FD8D828C83A3EFF09068EEE0FFEF19
:1080930075F018A42404F582E43465F583E0FEA3A7
:1080A300E0FF9068ECE0FCA3E0FD8D828C83A3A34A
:1080B300EFF09068EEE0FFEF75F018A42406F58268
:1080C300E43465F583E0FEA3E0FF9068ECE0FCA3F5
:1080D300E0FD8D828C83A3A3A3EFF09068EEE0FF15
:1080E300EF75F018A42408F582E43465F583E0FE07
:1080F300A3E0FF9068ECE0FCA3E0FD8D828C83E5B8
:10810300822404F582E5833400F583EFF09068EE72
:10811300E0FFEF75F018A4240AF582E43465F583D3
:10812300E0FEA3E0FF9068ECE0FCA3E0FD8D828C11
:1081330083E5822405F582E5833400F583EFF0902F
:1081430068EEE0FFEF75F018A4240CF582E43465C3
:10815300F583E0FEA3E0FF9068ECE0FCA3E0FD8D77
:10816300828C83E5822406F582E5833400F583EF70
:10817300F09068EEE0FFEF75F018A4240EF582E4AA
:108183003465F583E0FEA3E0FF9068ECE0FCA3E038
:10819300FD8D828C83E5822407F582E5833400F527
:1081A30083EFF09068EEE0FFEF75F018A42410F56C
:1081B30082E43465F583E0FEA3E0FF9068ECE0FC25
:1081C300A3E0FD8D828C83E5822408F582E5833468
:1081D30000F583EFF09068EEE0FFEF75F018A4244C
:1081E30012F582E43465F583E0FEA3E0FF9068ECCA
:1081F300E0FCA3E0FD8D828C83E5822409F582E512
:10820300833400F583EFF09068EEE0FFEF75F0182C
:10821300A42414F582E43465F583E0FEA3E0FF9023
:1082230068ECE0FCA3E0FD8D828C83E582240AF5F3
:1082330082E5833400F583EFF09068EEE0FFEF759D
:10824300F018A42416F582E43465F583E0FEA3E078
:10825300FF9068ECE0FCA3E0FD8D828C83E5822433
:108263000BF582E5833400F583EFF09068EEE0FFD1
:10827300744B2FF582E43459F583E0FF9068ECE00A
:10828300FCA3E0FD8D828C83E582240CF582E583DB
:108293003400F583EFF09068EEE0FF744D2FF58224
:1082A300E43459F583E0FF9068ECE0FCA3E0FD8D36
:1082B300828C83E582240DF582E5833400F583EF18
:1082C300F09068EEE0FF74A82FF582E4345EF58346
:1082D300E0FF9068ECE0FCA3E0FD8D828C83E582F7
:1082E300240EF582E5833400F583EFF09068EEE029
:1082F300FF74F62FF582E4345DF583E0FF9068ECBC
:10830300E0FCA3E0FD8D828C83E582240FF582E5FA
:10831300833400F583EFF09068EEE0FF744F2FF5A0
:1083230082E43459F583E0FF9068ECE0FCA3E0FDC0
:108333008D828C83E5822410F582E5833400F583F6
:10834300EFF09068EEE0FF74512FF582E43459F5B5
:1083530083E0FF9068ECE0FCA3E0FD8D828C83E575
:10836300822411F582E5833400F583EFF09068EE03
:10837300E0FF74C92FF582E4345EF583E0FF906873
:10838300ECE0FCA3E0FD8D828C83E5822412F58270
:10839300E5833400F583EFF09068EEE0FF74012F7E
:1083A300F582E4345EF583E0FF9068ECE0FCA3E043
:1083B300FD8D828C83E5822413F582E5833400F5F9
:0483C30083EFF02232
:109C6F009068B3EEF0A3EFF09068B5ECF0A3EDF0D1
:109C7F009068B7EBF09068B7E0FF74922FF582E42D
:109C8F00340CF583E0FF9068B3E0FCA3E0FD8D8218
:109C9F008C83EFF09068B7E0FF74F12FF582E43416
:109CAF0050F583E0FF9068B3E0FCA3E0FD8D828C5C
:109CBF0083A3EFF09068B7E0FF74202FF582E434B0
:109CCF0055F583E0FF9068B3E0FCA3E0FD8D828C37
:109CDF0083A3A3EFF09068B7E0FF74262FF582E41B
:109CEF003455F583E0FF9068B3E0FCA3E0FD8D826F
:109CFF008C83A3A3A3EFF09068B5E0FEA3E0FF8FE2
:109D0F00828E83E5822443F582E5833400F583E078
:109D1F00FF9068B3E0FCA3E0FD8D828C83E5822485
:109D2F0004F582E5833400F583EFF09068B5E0FE2B
:109D3F00A3E0FF8F828E83E582241DF582E58334B5
:109D4F0000F583E0FF9068B3E0FCA3E0FD8D828C0B
:109D5F0083E5822405F582E5833400F583EFF090E7
:109D6F0068B3E0FEA3E0FF8F828E83E5822406F5C1
:109D7F0082E5833400F583E4F0905945E0FF906865
:109D8F00B3E0FCA3E0FD8D828C83E5822407F5828E
:109D9F00E5833400F583EFF0905946E0FF9068B308
:109DAF00E0FCA3E0FD8D828C83E5822408F582E53B
:109DBF00833400F583EFF0905947E0FF9068B3E0EC
:109DCF00FCA3E0FD8D828C83E5822409F582E58377
:109DDF003400F583EFF0905948E0FF9068B3E0FC52
:109DEF00A3E0FD8D828C83E582240AF582E583341E
:109DFF0000F583EFF0905949E0FF9068B3E0FCA3C2
:109E0F00E0FD8D828C83E582240BF582E58334009F
:059E1F00F583EFF022C5
:1083C7009068C6EEF0A3EFF09068C8ECF0A3EDF06C
:1083D7009068C8E0FEA3E0FF8F828E83E582240CBD
:1083E700F582E5833400F583E0FF9068C6E0FCA3DF
:1083F700E0FD8D828C83EFF09068C8E0FEA3E0FF7C
:108407008F828E83E582240DF582E5833400F58320
:10841700E0FF9068C6E0FCA3E0FD8D828C83A3EFAC
:10842700F09068C8E0FEA3E0FF8F828E83E5822488
:108437000EF582E5833400F583E0FF9068C6E0FC23
:10844700A3E0FD8D828C83A3A3EFF09068C8E0FEC4
:10845700A3E0FF8F828E83E582240FF582E58334C4
:1084670000F583E0FF9068C6E0FCA3E0FD8D828CF9
:1084770083A3A3A3EFF09068C8E0FEA3E0FF8F8279
:108487008E83E5822410F582E5833400F583E0FFCF
:108497009068C6E0FCA3E0FD8D828C83E58224040E
:1084A700F582E5833400F583EFF09068C8E0FEA31A
:1084B700E0FF8F828E83E5822411F582E583340005
:1084C700F583E0FF9068C6E0FCA3E0FD8D828C8316
:1084D700E5822405F582E5833400F583EFF09068A3
:1084E700C8E0FEA3E0FF8F828E83E5822412F58227
:1084F700E5833400F583E0FF9068C6E0FCA3E0FD68
:108507008D828C83E5822406F582E5833400F5832A
:10851700EFF09068C8E0FEA3E0FF8F828E83E582CC
:108527002413F582E5833400F583E0FF9068C6E005
:10853700FCA3E0FD8D828C83E5822407F582E58329
:108547003400F583EFF09068C8E0FEA3E0FF8F8268
:108557008E83E5822414F582E5833400F583E0FFFA
:108567009068C6E0FCA3E0FD8D828C83E582240839
:10857700F582E5833400F583EFF09068C8E0FEA349
:10858700E0FF8F828E83E5822415F582E583340030
:10859700F583E0FF9068C6E0FCA3E0FD8D828C8345
:1085A700E5822409F582E5833400F583EFF09068CE
:1085B700C8E0FEA3E0FF8F828E83E5822416F58252
:1085C700E5833400F583E0FF9068C6E0FCA3E0FD97
:1085D7008D828C83E582240AF582E5833400F58356
:1085E700EFF09068C8E0FEA3E0FF8F828E83E582FC
:1085F7002417F582E5833400F583E0FF9068C6E031
:10860700FCA3E0FD8D828C83E582240BF582E58354
:108617003400F583EFF09068C8E0FEA3E0FF8F8297
:108627008E83E5822418F582E5833400F583E0FF25
:108637009068C6E0FCA3E0FD8D828C83E582240C64
:10864700F582E5833400F583EFF09068C8E0FEA378
:10865700E0FF8F828E83E5822419F582E58334005B
:10866700F583E0FF9068C6E0FCA3E0FD8D828C8374
:10867700E582240DF582E5833400F583EFF09068F9
:10868700C8E0FEA3E0FF8F828E83E582241AF5827D
:10869700E5833400F583E0FF9068C6E0FCA3E0FDC6
:1086A7008D828C83E582240EF582E5833400F58381
:1086B700EFF09068C8E0FEA3E0FF8F828E83E5822B
:1086C700241BF582E5833400F583E0FF9068C6E05C
:1086D700FCA3E0FD8D828C83E582240FF582E58380
:1086E7003400F583EFF09068C8E0FEA3E0FF8F82C7
:1086F7008E83E582241CF582E5833400F583E0FF51
:108707009068C6E0FCA3E0FD8D828C83E58224108F
:0B871700F582E5833400F583EFF022CB
:10BD1E009068CAEEF0A3EFF09068CCECF0A3EDF0D3
:10BD2E009068CCE0FEA3E0FF8F828E83E582240C28
:10BD3E00F582E5833400F583E0FF9068CAE0FCA34A
:10BD4E00E0FD8D828C83E0FEEE6F70739068CCE028
:10BD5E00FEA3E0FF8F828E83E582241AF582E583AF
:10BD6E003400F583E0FF9068CAE0FCA3E0FD8D820D
:10BD7E008C83E582240EF582E5833400F583E0FEA4
:10BD8E00EEB5073B9068CCE0FEA3E0FF8F828E837A
:10BD9E00E582241BF582E5833400F583E0FF90688D
:10BDAE00CAE0FCA3E0FD8D828C83E582240FF58230
:10BDBE00E5833400F583E0FEEEB507037F00227FB6
:02BDCE00012250
:109AB9009068B8EEF0A3EFF09068BAECF0A3EDF07F
:109AC9009068BCEBF09068BCE0FF74902FF582E4DD
:109AD900340AF583E0FF9068B8E0FCA3E0FD8D82CD
:109AE9008C83EFF09068BAE0FEA3E0FF8F828E834B
:109AF900E5822443F582E5833400F583E0FF90682D
:109B0900B8E0FCA3E0FD8D828C83A3EFF09068BAE6
:109B1900E0FEA3E0FF8F828E83E582241DF582E5B6
:109B2900833400F583E0FF9068B8E0FCA3E0FD8D85
:109B3900828C83A3A3EFF09068BAE0FEA3E0FF8FC5
:109B4900828E83E5822442F582E5833400F583E041
:109B5900FF9068B8E0FCA3E0FD8D828C83A3A3A3EA
:109B6900EFF09068B8E0FEA3E0FF8F828E83E58274
:109B79002404F582E5833400F583E4F09068BAE0C3
:109B8900FEA3E0FF8F828E83E5822440F582E58380
:109B99003400F583E0FF9068B8E0FCA3E0FD8D8216
:109BA9008C83E5822405F582E5833400F583EFF0A3
:109BB9009068B8E0FEA3E0FF8F828E83E5822406D9
:109BC900F582E5833400F583E4F0905945E0FF9090
:109BD90068B8E0FCA3E0FD8D828C83E5822407F55B
:109BE90082E5833400F583EFF0905946E0FF9068F1
:109BF900B8E0FCA3E0FD8D828C83E5822408F58220
:109C0900E5833400F583EFF0905947E0FF9068B899
:109C1900E0FCA3E0FD8D828C83E5822409F582E5D1
:109C2900833400F583EFF0905948E0FF9068B8E07D
:109C3900FCA3E0FD8D828C83E582240AF582E5830D
:109C49003400F583EFF0905949E0FF9068B8E0FCE3
:109C5900A3E0FD8D828C83E582240BF582E58334B4
:069C690000F583EFF0227C
:10AFB9009068CEEFF09068CFEBF0A3EAF0A3E9F048
:10AFC9009068CFE0FBA3E0FAA3E0F975820C7583E2
:10AFD90000128E28FFEF700302B0EB9068CEE0FFFD
:10AFE900741B2FF582E43467F583E0FFEF600302F9
:10AFF900B0EB9068CFE0FBA3E0FAA3E0F975820C0F
:10B00900758300128E28FFEF64FA700302B0EB908B
:10B0190068CFE0FBA3E0FAA3E0F975820C75830021
:10B02900128E28FFEF64F5700302B0EB9068CEE052
:10B03900FFEF75F011A42470F582E4344EF583AF67
:10B0490082AE839068CFE0FBA3E0FAA3E0F9AC02FB
:10B05900AD0112BD1EEF700302B0EB9068CEE0FFA8
:10B06900EF75F011A42470F582E4344EF583AF82B4
:10B07900AE839068CFE0FBA3E0FAA3E0F9AC02ADA0
:10B08900011283C79068CEE0FF7EADEF8EF0A4FF7A
:10B09900AEF0743F2FF974553EFA7B01C003C0022C
:10B0A900C0019068CEE0FF7E11EF8EF0A4FFAEF0F4
:10B0B90074702FF9744E3EFA7B01C003C002C001BF
:10B0C9007B017A6779ECA801AC02AD03D001D0020B
:10B0D900D0037E007F11128DE9D001D002D0031276
:03B0E900A8162284
:10CB04009068EFEBF0A3EAF0A3E9F09068EFE0FBA4
:10CB1400A3E0FAA3E0F97582AB758300E4128E6793
:10CB24009068EFE0FBA3E0FAA3E0F97582AA7583AD
:10CB340000E4128E679068EFE0FBA3E0FAA3E0F94B
:0BCB44007582AC758300E4128E67223E
:0BC7BE009068D2EBF0A3EAF0A3E9F0D2
:10C7C9009068D5E4F09068D2E0FBA3E0FAA3E0F921
:10C7D9007582AC758300128E28FFEF70349068D291
:10C7E900E0FBA3E0FAA3E0F97582AB758300128E32
:10C7F90028FF9068D2E0FBA3E0FAA3E0F97582AACA
:10C80900758300128E28FEEEB507069068D574016F
:06C81900F09068D5E0FF7D
:01C81F0022F6
:0BA816009067E9EBF0A3EAF0A3E9F083
:10A821009067E9E0FBA3E0FAA3E0F97582AA7583DA
:10A8310000128E28FF9067E9E0FBA3E0FAA3E0F99C
:10A841007582AB758300128E28FEC3EE9FFFEF0465
:10A85100FF9067FDEFF07B017A6779ECC003C002DE
:10A86100C0019067E9E0FBA3E0FAA3E0F97582ABD0
:10A87100758300128E28FF7E11EF8EF0A4FFAEF0DB
:10A881009067E9E0FBA3E0FAA3E0F9E92FF9EA3EDA
:10A89100FAA801AC02AD03D001D002D0037E007F43
:10A8A10011128DE99067E9E0FBA3E0FAA3E0F975E5
:10A8B10082AB758300128E28FF7E00EF2401FFEE2C
:10A8C1003400FE7C007D0A128E9BAF059067E9E0A3
:10A8D100FBA3E0FAA3E0F97582AB758300EF128E5A
:10A8E100679067E9E0FBA3E0FAA3E0F97582AB7535
:10A8F1008300128E28FFEF701F9067FDE0FFEFB419
:10A901000A169067E9E0FBA3E0FAA3E0F97582ACCF
:10A911007583007401128E679067E9E0FBA3E0FA8A
:10A92100A3E0F97582AC758300128E28FFEF602ACF
:10A931009067E9E0FBA3E0FAA3E0F97582AB7583C8
:10A9410000128E28FF9067E9E0FBA3E0FAA3E0F98B
:0AA951007582AA758300EF128E676D
:01A95B0022D9
:10C4C5009068F2EBF0A3EAF0A3E9F09068F2E0FBE4
:10C4D500A3E0FAA3E0F912C7BEEF70529068F2E04C
:10C4E500FBA3E0FAA3E0F97582AC758300E4128E34
:10C4F500679068F2E0FBA3E0FAA3E0F97582AA75FC
:10C505008300128E28FF7E00EF2401FFEE3400FE2B
:10C515007C007D0A128E9BAF059068F2E0FBA3E0DC
:0FC52500FAA3E0F97582AA758300EF128E6722E0
:10CCC5009068F5EBF0A3EAF0A3E9F09068F5E0FBD6
:10CCD500A3E0FAA3E0F97582AA758300128E28FFF6
:10CCE500EF75F00A84AFF07E11EF8EF0A4FFAEF081
:10CCF5009068F5E0FBA3E0FAA3E0F9E92FF9EA3E35
:02CD0500FA2210
:10CB4F009068F8EBF0A3EAF0A3E9F09068F8E0FB47
:10CB5F00A3E0FAA3E0F9758279758300E4128E677A
:10CB6F009068F8E0FBA3E0FAA3E0F975827875838B
:10CB7F0000E4128E679068F8E0FBA3E0FAA3E0F9F7
:0BCB8F0075827A758300E4128E672225
:0BC820009068D6EBF0A3EAF0A3E9F06B
:10C82B009068D9E4F09068D6E0FBA3E0FAA3E0F9B6
:10C83B0075827A758300128E28FFEF70349068D65C
:10C84B00E0FBA3E0FAA3E0F9758279758300128E01
:10C85B0028FF9068D6E0FBA3E0FAA3E0F975827895
:10C86B00758300128E28FEEEB507069068D9740109
:06C87B00F09068D9E0FF17
:01C881002294
:0BA95C00906822EBF0A3EAF0A3E9F002
:10A96700906822E0FBA3E0FAA3E0F975827875838B
:10A9770000128E28FF906822E0FBA3E0FAA3E0F91B
:10A98700758279758300128E28FEC3EE9FFFEF0450
:10A99700FF906831EFF07B017A687925C003C00228
:10A9A700C001906822E0FBA3E0FAA3E0F975827981
:10A9B700758300128E28FF7E0CEF8EF0A4FFAEF099
:10A9C700906822E0FBA3E0FAA3E0F9E92FF9EA3E59
:10A9D700FAA801AC02AD03D001D002D0037E007FFC
:10A9E7000C128DE9906822E0FBA3E0FAA3E0F97569
:10A9F7008279758300128E28FF7E00EF2401FFEE17
:10AA07003400FE7C007D0A128E9BAF05906822E021
:10AA1700FBA3E0FAA3E0F9758279758300EF128E44
:10AA270067906822E0FBA3E0FAA3E0F975827975E5
:10AA37008300128E28FFEF701F906831E0FFEFB49C
:10AA47000A16906822E0FBA3E0FAA3E0F975827A80
:10AA57007583007401128E67906822E0FBA3E0FA09
:10AA6700A3E0F975827A758300128E28FFEF602ABA
:10AA7700906822E0FBA3E0FAA3E0F9758279758379
:10AA870000128E28FF906822E0FBA3E0FAA3E0F90A
:0AAA9700758278758300EF128E6758
:01AAA1002292
:10C534009068FBEBF0A3EAF0A3E9F09068FBE0FB62
:10C54400A3E0FAA3E0F912C820EF70529068FBE070
:10C55400FBA3E0FAA3E0F975827A758300E4128EF6
:10C56400679068FBE0FBA3E0FAA3E0F975827875B5
:10C574008300128E28FF7E00EF2401FFEE3400FEBC
:10C584007C007D0A128E9BAF059068FBE0FBA3E064
:0FC59400FAA3E0F9758278758300EF128E6722A3
:10CD07009068FEEBF0A3EAF0A3E9F09068FEE0FB81
:10CD1700A3E0FAA3E0F9758278758300128E28FFE5
:10CD2700EF75F00A84AFF07E0CEF8EF0A4FFAEF043
:10CD37009068FEE0FBA3E0FAA3E0F9E92FF9EA3EE9
:02CD4700FA22CE
:10CB9A00906901EBF0A3EAF0A3E9F0906901E0FBE8
:10CBAA00A3E0FAA3E0F97582B1758304E4128E67F3
:10CBBA00906901E0FBA3E0FAA3E0F97582B07583FE
:10CBCA0004E4128E67906901E0FBA3E0FAA3E0F99E
:0BCBDA007582B2758304E4128E67229E
:0BC882009068DAEBF0A3EAF0A3E9F005
:10C88D009068DDE4F09068DAE0FBA3E0FAA3E0F94C
:10C89D007582B2758304128E28FFEF70349068DABA
:10C8AD00E0FBA3E0FAA3E0F97582B1758304128E63
:10C8BD0028FF9068DAE0FBA3E0FAA3E0F97582B0F7
:10C8CD00758304128E28FEEEB507069068DD74019F
:06C8DD00F09068DDE0FFB1
:01C8E3002232
:0BAAA200906832EBF0A3EAF0A3E9F0AB
:10AAAD00906832E0FBA3E0FAA3E0F97582B07583FC
:10AABD0004128E28FF906832E0FBA3E0FAA3E0F9C0
:10AACD007582B1758304128E28FEC3EE9FFFEF04CD
:10AADD00FF906841EFF07B017A687935C003C002C1
:10AAED00C001906832E0FBA3E0FAA3E0F97582B1F2
:10AAFD00758304128E28FF7E0CEF8EF0A4FFAEF04E
:10AB0D00906832E0FBA3E0FAA3E0F9E92FF9EA3E01
:10AB1D00FAA801AC02AD03D001D002D0037E007FB4
:10AB2D000C128DE9906832E0FBA3E0FAA3E0F97511
:10AB3D0082B1758304128E28FF7E00EF2401FFEE93
:10AB4D003400FE7C007D64128E9BAF05906832E070
:10AB5D00FBA3E0FAA3E0F97582B1758304EF128EC1
:10AB6D0067906832E0FBA3E0FAA3E0F97582B17556
:10AB7D008304128E28FFEF701F906841E0FFEFB441
:10AB8D006416906832E0FBA3E0FAA3E0F97582B297
:10AB9D007583047401128E67906832E0FBA3E0FAAE
:10ABAD00A3E0F97582B2758304128E28FFEF602A37
:10ABBD00906832E0FBA3E0FAA3E0F97582B17583EA
:10ABCD0004128E28FF906832E0FBA3E0FAA3E0F9AF
:0AABDD007582B0758304EF128E67D5
:01ABE700224B
:10C5A300906904EBF0A3EAF0A3E9F0906904E0FBDF
:10C5B300A3E0FAA3E0F912C882EF7052906904E095
:10C5C300FBA3E0FAA3E0F97582B2758304E4128E4B
:10C5D30067906904E0FBA3E0FAA3E0F97582B07504
:10C5E3008304128E28FF7E00EF2401FFEE3400FE49
:10C5F3007C007D64128E9BAF05906904E0FBA3E091
:0FC60300FAA3E0F97582B0758304EF128E6722F7
:10CD4900906907EBF0A3EAF0A3E9F0906907E0FB2B
:10CD5900A3E0FAA3E0F97582B0758304128E28FF67
:10CD6900EF75F06484AFF07E0CEF8EF0A4FFAEF0A7
:10CD7900906907E0FBA3E0FAA3E0F9E92FF9EA3E9D
:02CD8900FA228C
:10C2DD009068BDEFF09068BEEBF0A3EAF0A3E9F033
:10C2ED009068C1E4F09068BEE0FBA3E0FAA3E0F92A
:10C2FD007582B2758304128E28FFEF70489068BD69
:10C30D00E0FF74572FF582E4345BF583E0FFEF70A7
:10C31D00349068BEE0FBA3E0FAA3E0F97582B17535
:10C32D008304128E28FF9068BEE0FBA3E0FAA3E021
:10C33D00F97582B0758304128E28FEEEB50706904E
:0AC34D0068C17401F09068C1E0FFC0
:01C3570022C3
:10A42000906811EFF0906812EBF0A3EAF0A3E9F066
:10A43000906811E0FFEF600302A575906812E0FBE1
:10A44000A3E0FAA3E0F97582B0758304128E28FFA9
:10A45000906812E0FBA3E0FAA3E0F97582B175837E
:10A4600004128E28FEC3EE9FFFEF04FF906821EFD9
:10A47000F07B017A687915C003C002C001906812B0
:10A48000E0FBA3E0FAA3E0F97582B1758304128EB4
:10A4900028FF7E0CEF8EF0A4FFAEF0906812E0FB78
:10A4A000A3E0FAA3E0F9E92FF9EA3EFAA801AC0229
:10A4B000AD03D001D002D0037E007F0C128DE99055
:10A4C0006812E0FBA3E0FAA3E0F97582B17583049A
:10A4D000128E28FF7E00EF2401FFEE3400FE7C0088
:10A4E0007D64128E9BAF05906812E0FBA3E0FAA397
:10A4F000E0F97582B1758304EF128E67906812E0FF
:10A50000FBA3E0FAA3E0F97582B1758304128E28EB
:10A51000FFEF701F906821E0FFEFB464169068129F
:10A52000E0FBA3E0FAA3E0F97582B275830474013D
:10A53000128E67906812E0FBA3E0FAA3E0F975823F
:10A54000B2758304128E28FFEF602A906812E0FB38
:10A55000A3E0FAA3E0F97582B1758304128E28FF97
:10A56000906812E0FBA3E0FAA3E0F97582B075836E
:05A5700004EF128E67EC
:01A5750022C3
:10CBE50090690AEBF0A3EAF0A3E9F090690AE0FB8B
:10CBF500A3E0FAA3E0F97582C9758300E4128E6794
:10CC050090690AE0FBA3E0FAA3E0F97582C8758391
:10CC150000E4128E6790690AE0FBA3E0FAA3E0F94D
:0BCC25007582CA758300E4128E67223E
:0BC8E4009068DEEBF0A3EAF0A3E9F09F
:10C8EF009068E1E4F09068DEE0FBA3E0FAA3E0F9E2
:10C8FF007582CA758300128E28FFEF70349068DE40
:10C90F00E0FBA3E0FAA3E0F97582C9758300128EEC
:10C91F0028FF9068DEE0FBA3E0FAA3E0F97582C878
:10C92F00758300128E28FEEEB507069068E174013C
:06C93F00F09068E1E0FF4A
:01C9450022CF
:0BABE8009067A6EBF0A3EAF0A3E9F0F1
:10ABF3009067A6E0FBA3E0FAA3E0F97582C875832A
:10AC030000128E28FF9067A6E0FBA3E0FAA3E0F909
:10AC13007582C9758300128E28FEC3EE9FFFEF0471
:10AC2300FF9067BDEFF07B017A6779A9C003C0028B
:10AC3300C0019067A6E0FBA3E0FAA3E0F97582C91F
:10AC4300758300128E28FF7E14EF8EF0A4FFAEF002
:10AC53009067A6E0FBA3E0FAA3E0F9E92FF9EA3E47
:10AC6300FAA801AC02AD03D001D002D0037E007F6D
:10AC730014128DE99067A6E0FBA3E0FAA3E0F9754F
:10AC830082C9758300128E28FF7E00EF2401FFEE38
:10AC93003400FE7C007D0A128E9BAF059067A6E010
:10ACA300FBA3E0FAA3E0F97582C9758300EF128E66
:10ACB300679067A6E0FBA3E0FAA3E0F97582C97584
:10ACC3008300128E28FFEF701F9067BDE0FFEFB483
:10ACD3000A169067A6E0FBA3E0FAA3E0F97582CA1F
:10ACE3007583007401128E679067A6E0FBA3E0FAF8
:10ACF300A3E0F97582CA758300128E28FFEF602ADC
:10AD03009067A6E0FBA3E0FAA3E0F97582C9758317
:10AD130000128E28FF9067A6E0FBA3E0FAA3E0F9F8
:0AAD23007582C8758300EF128E6779
:01AD2D002203
:10C6120090690DEBF0A3EAF0A3E9F090690DE0FB5D
:10C62200A3E0FAA3E0F912C8E4EF705290690DE0BA
:10C63200FBA3E0FAA3E0F97582CA758300E4128EC7
:10C642006790690DE0FBA3E0FAA3E0F97582C87573
:10C652008300128E28FF7E00EF2401FFEE3400FEDD
:10C662007C007D0A128E9BAF0590690DE0FBA3E072
:0FC67200FAA3E0F97582C8758300EF128E672274
:10CD8B00906910EBF0A3EAF0A3E9F0906910E0FBD7
:10CD9B00A3E0FAA3E0F97582C8758300128E28FF11
:10CDAB00EF75F00A84AFF07E14EF8EF0A4FFAEF0B7
:10CDBB00906910E0FBA3E0FAA3E0F9E92FF9EA3E52
:02CDCB00FA224A
:10CC3000906913EBF0A3EAF0A3E9F0906913E0FB2D
:10CC4000A3E0FAA3E0F975822175831CE4128E67D4
:10CC5000906913E0FBA3E0FAA3E0F97582207583E5
:10CC60001CE4128E67906913E0FBA3E0FAA3E0F9DD
:0BCC700075822275831CE4128E67227F
:0BC946009068E2EBF0A3EAF0A3E9F038
:10C951009068E5E4F09068E2E0FBA3E0FAA3E0F977
:10C9610075822275831C128E28FFEF70349068E265
:10C97100E0FBA3E0FAA3E0F975822175831C128E16
:10C9810028FF9068E2E0FBA3E0FAA3E0F9758220BA
:10C9910075831C128E28FEEEB507069068E57401BA
:06C9A100F09068E5E0FFE4
:01C9A700226D
:0BAD2E00906751EBF0A3EAF0A3E9F0FE
:10AD3900906751E0FBA3E0FAA3E0F97582207583DF
:10AD49001C128E28FF906751E0FBA3E0FAA3E0F9FB
:10AD590075822175831C128E28FEC3EE9FFFEF04B6
:10AD6900FF906784EFF07B017A677954C003C002D2
:10AD7900C001906751E0FBA3E0FAA3E0F9758221D5
:10AD890075831C128E28FF7E30EF8EF0A4FFAEF083
:10AD9900906751E0FBA3E0FAA3E0F9E92FF9EA3E55
:10ADA900FAA801AC02AD03D001D002D0037E007F26
:10ADB90030128DE9906751E0FBA3E0FAA3E0F97541
:10ADC900822175831C128E28FF7E00EF2401FFEE7D
:10ADD9003400FE7C007D96128E9BAF05906751E092
:10ADE900FBA3E0FAA3E0F975822175831CEF128EAB
:10ADF90067906751E0FBA3E0FAA3E0F9758221753A
:10AE0900831C128E28FFEF701F906784E0FFEFB458
:10AE19009616906751E0FBA3E0FAA3E0F975822248
:10AE290075831C7401128E67906751E0FBA3E0FAE9
:10AE3900A3E0F975822275831C128E28FFEF602A20
:10AE4900906751E0FBA3E0FAA3E0F97582217583CD
:10AE59001C128E28FF906751E0FBA3E0FAA3E0F9EA
:0AAE690075822075831CEF128E67BE
:01AE730022BC
:10C68100906916EBF0A3EAF0A3E9F0906916E0FBDC
:10C69100A3E0FAA3E0F912C946EF7052906916E0DF
:10C6A100FBA3E0FAA3E0F975822275831CE4128EE4
:10C6B10067906916E0FBA3E0FAA3E0F975822075A3
:10C6C100831C128E28FF7E00EF2401FFEE3400FE52
:10C6D1007C007D96128E9BAF05906916E0FBA3E06E
:0FC6E100FAA3E0F975822075831CEF128E672291
:10CDCD00906919EBF0A3EAF0A3E9F0906919E0FB83
:10CDDD00A3E0FAA3E0F975822075831C128E28FF5B
:10CDED007E007C007D96128E9B7E007F30128E8998
:10CDFD00906919E0FBA3E0FAA3E0F9E92FF9EA3E07
:02CE0D00FA2207
:107B5800906929EFF0906929E0FF74A62FF582E477
:107B6800345EF583E0FFEF7003027D0D906929E034
:107B7800FF74A62FF582E4345EF583E4F0D290908A
:107B88006929E0FF74052FF582E43459F583E4F0A0
:107B9800906929E0FF74D12FF582E43450F583749D
:107BA80001F0906929E0FF749A2FF582E4340CF50E
:107BB80083E4F0906929E0FF7E00EF7F00FE7462A5
:107BC8002FF582745B3EF583E0FF906929E0FEEEB5
:107BD80075F003A424BEF582E43467F583EFF090D2
:107BE8006929E0FF7E00EF7F00FE74632FF5827441
:107BF8005B3EF583E0FF906929E0FEEE75F003A493
:107C080024BFF582E43467F583EFF0906929E0FF3B
:107C18007E00EF7F00FE74642FF582745B3EF5836F
:107C2800E0FF906929E0FEEE75F003A424C0F58218
:107C3800E43467F583EFF0906929E0FF7E00EF7F79
:107C480000FE74652FF582745B3EF583E0FF906952
:107C580029E0FE74CC2EF582E43467F583EFF090CA
:107C68006929E0FF74CC2FF582E43467F583E0FFDF
:107C7800EF240EFF906929E0FE74EA2EF582E434C1
:107C880062F583EFF0906929E0FF7E00EF7F00FE48
:107C9800745A2FF9745B3EFA7B01C003C002C0011D
:107CA800906929E0FF7E00EF7F00FE74E82FF974E9
:107CB800603EFA7B01906891EBF0A3EAF0A3E9F04B
:107CC800906929E0FF74EA2FF582E43462F583E0D5
:107CD800FF906894EFF0D001D002D00312CA5B90F5
:107CE8006929E0FF74D92FF582E43460F583740EB6
:107CF800F0906929E0FF74EC2FF582E43462F58393
:107D0800E4F002800D906929E0FF74FA2FF582E40F
:107D1800345DF583E0FFEF7003027EBD906929E0D2
:107D2800FF74FA2FF582E4345DF583E4F0D2909085
:107D38006929E0FF74052FF582E43459F583E4F0EE
:107D4800906929E0FF74D12FF582E43450F583E47B
:107D5800F0906929E0FF749A2FF582E4340CF583DA
:107D68007401F0906929E0FF7E00EF7F00FE745EE9
:107D78002FF58274593EF583E0FF906929E0FEEE05
:107D880075F003A424CEF582E43467F583EFF09010
:107D98006929E0FF7E00EF7F00FE745F2FF5827493
:107DA800593EF583E0FF906929E0FEEE75F003A4E3
:107DB80024CFF582E43467F583EFF0906929E0FF7A
:107DC8007E00EF7F00FE74602FF58274593EF583C4
:107DD800E0FF906929E0FEEE75F003A424D0F58257
:107DE800E43467F583EFF0906929E0FF7E00EF7FC8
:107DF80000FE74612FF58274593EF583E0FF9069A7
:107E080029E0FE74C82EF582E43467F583EFF0901C
:107E18006929E0FF74EA2FF582E43462F583740E71
:107E2800F0906929E0FF7E00EF7F00FE74562FF97D
:107E380074593EFA7B01C003C002C001906929E071
:107E4800FF7E00EF7F00FE74E82FF974603EFA7B36
:107E580001906891EBF0A3EAF0A3E9F0906929E0BA
:107E6800FF74EA2FF582E43462F583E0FF906894AA
:107E7800EFF0D001D002D00312CA5B906929E0FF6D
:107E880074C82FF582E43467F583E0FFEF240EFF12
:107E9800906929E0FE74D92EF582E43460F583EF09
:107EA800F0906929E0FF74EC2FF582E43462F583E1
:107EB800E4F002800DD290906929E0FF74052FF557
:107EC80082E43459F5837401F0906929E0FF74D194
:107ED8002FF582E43450F583E4F0906929E0FF74CB
:107EE8009A2FF582E4340CF583E4F0906929E0FFD9
:107EF800EF75F003A424A6F582E4344EF583E4F08C
:107F0800906929E0FFEF75F003A424A7F582E43413
:107F18004EF58374D4F0906929E0FFEF75F003A45F
:107F280024A8F582E4344EF583E4F0906929E0FF53
:107F380074002FF582E43459F5837433F09069297D
:107F4800E0FF74C42FF582E43467F5837440F09041
:107F58006929E0FFEF75F007A42403F582E4345E95
:107F6800F583AF82AE83C006C007906929E0FFEFB2
:107F780075F003A424A6F582E4344EF583AD82ACF3
:107F880083906929E0FF74002FF582E43459F58362
:107F9800E0FB906929E0FF74C42FF582E43467F5AB
:107FA80083E0FF906867EFF0906929E0FF7E00EFBB
:107FB8007F00FE74E82FF58274603EF583AF82AED1
:107FC80083906868EEF0A3EFF0D007D00612B34BA9
:107FD800906929E0FF74EA2FF582E43462F583742E
:107FE8000EF0906929E0FF74D92FF582E43460F52A
:107FF80083744EF0906929E0FF74EC2FF582E43425
:1080080062F583E4F0906929E0FFEF700890673229
:108018007401F0800F906929E0FFEFB401069067C2
:0B802800337401F000000000D2992228
:0DC04100906887EFF0906888ECF0A3EDF0B8
:10C04E00756B0090688C74FFF090688D74FFF075BE
:10C05E006A01906887E0FFE56AD39F504B9068882D
:10C06E00E0FEA3E0FF8F828E83E0FF90688CE0FEFF
:10C07E00EE6FF56BAF6BEF908F5F93FF90688DE077
:10C08E00FEEE6FFF90688CEFF0AF6BEF90905F93CA
:10C09E00FF90688DEFF0906889E004F0700690686C
:10C0AE0088E004F0056A80AA90688CE0FF90688BA7
:10C0BE00EFF090688DE0FF90688AEFF090688AE06C
:04C0CE00FEA3E0FFEE
:01C0D200224B
:03000B0002C1DE51
:10C1DE00C0E0C0F0C083C082C0D075D000C000C027
:10C1EE0001C002C003C004C005C006C007758CDFC5
:10C1FE00758A739067A4E004F09067A5E004F09050
:10C20E0067A4E0FFEFC39404401A9067A4E4F01211
:10C21E00CFF012B94B12CAB012CF2612C358120069
:10C22E000E12B6909067A5E0FFEFC39405400890FC
:10C23E0067A5E4F012B0ECD007D006D005D004D03C
:10C24E0003D002D001D000D0D0D082D083D0F0D095
:02C25E00E032CC
:10CFF00012C0D312B87E129FBD12C15A12BBA31227
:09D00000BC6212CE4F12C3D32210
:10C0D300906788E0FFEF7005906785E4F0906788CC
:10C0E300E004F0906788E0FFEFC39419406890671D
:10C0F30088E4F09067857401F09067927401F09082
:10C103006789E0FFEFF4FF906789EFF0906789E0BC
:10C11300FFEF602390674A7401F0906712E0FFEF2E
:10C123006008906716E0FFEF602C90671F7401F0C2
:10C133009067207401F02290674AE4F0906712E060
:10C14300FFEF6008906716E0FFEF600A90671FE457
:07C15300F0906720E4F022E8
:10B87E0090679AE0FFEF7005906799E4F090679AF1
:10B88E00E004F090679AE0FFEFC39432500302B9E0
:10B89E004A90679AE4F09067997401F090679F74EC
:10B8AE0001F090679CE0FFEFF4FF90679CEFF012C1
:10B8BE00B79090668DE0FFEF703890668EE0FFEFE8
:10B8CE00703090678DE004F0900AA2E0FFEF7006F2
:10B8DE00900AA2741EF0900AA2E0FF90678DE0FE1F
:10B8EE00EEC39F40179067877401F090678DE4F068
:10B8FE00800A906787E4F090678DE4F0905DFEE03B
:10B90E00FFEF703890678CE004F0700690678BE064
:10B91E0004F09056B9E0FFEF70069056B9740AF035
:10B92E009056B9E0FF7E0090678BE0FCA3E0FDC36C
:0DB93E00ED9FEC9E4006905DFE7401F0222E
:109FBD00906799E0FFEF700302A141751C00E51C4D
:109FCD00C39402400302A141AF1C741C2FF582E41F
:109FDD003455F583E0FFEF700302A13CAF1CEF2574
:109FED00E0243AF582E43459F583E0FEA3E0FFC3A3
:109FFD00EF9418EE9400400302A0F5AF1CEF25E09E
:10A00D002473F582E43409F583E475F001128EF0C2
:10A01D00AF1CEF25E02473F582E43409F583E0FEEF
:10A02D00A3E0FFD3EF9410EE940E400302A13CAFDA
:10A03D001CEF25E02473F582E43409F583E0FEA3DB
:10A04D00E0FF7C007D0A128E9BED4C7055AF1C7E9F
:10A05D00007C1C7D23128E8974B82FF9740C3EFA86
:10A06D007B01C003C002C001AF1C7E00EF7F00FE6C
:10A07D0074C02FF9744E3EFA7B01C003C002C001BB
:10A08D007B017A677954A801AC02AD03D001D002EF
:10A09D00D0037E007F30128DE9D001D002D00312A3
:10A0AD00AD2EAF1CEF25E02473F582E43409F58362
:10A0BD00E0FEA3E0FFC3EF9410EE940E4071AF1CD1
:10A0CD00EF25E02473F582E43409F583E4F0A3E48D
:10A0DD00F0AF1CEF25E0243AF582E43459F583E422
:10A0ED0075F001128EF08047AF1CEF25E02473F55B
:10A0FD0082E43409F583E4F0A3E4F0AF1C741C2F63
:10A10D00F582E43455F583E4F0AF1CEF25E0243AF5
:10A11D00F582E43459F583E4F0A3E4F0E51C700511
:10A12D00906729E4F0E51CB4010590672AE4F00579
:04A13D001C029FCB96
:01A1410022FB
:10C15A00751D00E51DC394025079AF1D74AE2FF50D
:10C16A0082E4345EF583E0FFEF6064AF1DEF25E003
:10C17A00248EF582E43467F583E475F001128EF0BB
:10C18A00AF1DEF25E0248EF582E43467F583E0FEE7
:10C19A00A3E0FFC3EF94FAEE94004033AF1DEF25FE
:10C1AA00E0248EF582E43467F583E4F0A3E4F0AF8B
:10C1BA001D74AE2FF582E4345EF583E4F0E51D705C
:10C1CA000890674E7401F0800690674F7401F0057D
:03C1DA001D808045
:01C1DD00223F
:10BBA300751E00E51EC39402400302BC61905ED67D
:10BBB300E0FFEF6039906799E0FFEF6031905EAB93
:10BBC300E004F07006905EAAE004F0905EAAE0FE46
:10BBD300A3E0FFEFB40817EEB40713905DFC740104
:10BBE300F0905ED6E4F0905EAAE4F0A3E4F0AF1E1A
:10BBF30074132FF582E4345EF583E0FFEF605A900F
:10BC03006799E0FFEF6052AF1EEF25E02495F582C0
:10BC1300E43467F583E475F001128EF0AF1EEF256F
:10BC2300E02495F582E43467F583E0FEA3E0FFC3E7
:10BC3300EF9408EE94074021AF1E74132FF582E4AE
:10BC4300345EF583E4F0AF1EEF25E02495F582E43E
:0EBC53003467F583E4F0A3E4F0051E02BBA6FF
:01BC610022C0
:10BC6200751F00E51FC39402400302BD1DAF1F7480
:10BC72001B2FF582E43467F583E0FFEF700302BD0A
:10BC820005906799E0FFEF700302BD18AF1FEF2523
:10BC9200E024A0F582E43467F583E475F001128EA6
:10BCA200F0AF1FEF25E024A0F582E43467F583E0CE
:10BCB200FEA3E0FFC3EF9410EE940E4059AF1F7441
:10BCC2001B2FF582E43467F583E4F0AF1F74212F54
:10BCD200F582E43467F583E4F0AF1FEF25E024A09A
:10BCE200F582E43467F583E4F0A3E4F0E51F70071E
:10BCF20090671FE4F0801FE51FB4011A906720E4EB
:10BD0200F08013AF1FEF25E024A0F582E43467F53D
:0BBD120083E4F0A3E4F0051F02BC6511
:01BD1D002203
:10CE4F00906799E0FFEF6035906794E004F070060B
:10CE5F00906793E004F0906793E0FEA3E0FFE4FC9B
:10CE6F00FD7BC07AA879007800D3128F06500E9000
:0ECE7F0067867401F0906793E4F0A3E4F0225C
:10C3D300906786E0FFEF6071906786E4F090679E58
:10C3E300E004F090679EE0FFEFC39402405B906728
:10C3F3009B7401F090679EE4F09067E1E0FFEF60CB
:10C403000C90671BE0FFEF70047F0180027F0090B8
:10C4130056F5EFF09067E2E0FFEF600C90671CE0E9
:10C42300FFEF70047F0180027F009056F6EFF090DB
:10C4330056F5E0FFEF6005906744E4F09056F6E0B0
:0AC44300FFEF6005906745E4F0226A
:10B79000905949E004F0905949E0FFEFC3943C50C0
:10B7A0000302B87D905949E4F0905948E004F090C4
:10B7B0005948E0FFEFC3943C500302B87D905948CC
:10B7C000E4F0905947E004F0905947E0FFEFC3944C
:10B7D00018500302B87D905947E4F0905946E004B0
:10B7E000F0905945E0FFEF6404601D905945E0FF7B
:10B7F000EF64066013905945E0FFEF64096009901B
:10B800005945E0FFEFB40B0890692A741EF0802BB5
:10B81000905945E0FFEFB4021C905944E0FFEF540B
:10B8200003FFEF700890692A741DF0800E90692A5A
:10B83000741CF0800690692A741FF090692AE0FF5A
:10B84000905946E0FEEED39F40339059467401F084
:10B85000905945E004F0905945E0FFEFC3940D4046
:10B860001C9059457401F0905944E004F0905944FB
:0DB87000E0FFEFC394634005905944E4F0FD
:01B87D0022A8
:10CE8D009060E3E0FFEF701143A640758DF0758B58
:10CE9D00F07598D05387BF801B9060E3E0FFEFB42F
:10CEAD00011243A640758DF1758BF175985043872E
:07CEBD00805387BFD28E22D3
:03002300029355F0
:0F935500C0E0C083C082C0D075D000C006C00782
:10936400906789E0FFEF7003756700906789E0FFFD
:10937400EFB4FF03756701209903029446C299AFC5
:109384006774EA2FF582E43462F583E0FFAE677414
:10939400EC2EF582E43462F583E0FEEEC39F4003D5
:1093A400029427AF677E00EF7F00FE74E82FF582FA
:1093B40074603EF583C083C082AF6774EC2FF5827E
:1093C400E43462F583E0FFD082D083E5822FF58216
:1093D400E43583F583E0FFEFA2D0929BAF677E0074
:1093E400EF7F00FE74E82FF58274603EF583C0833E
:1093F400C082AF6774EC2FF582E43462F583E0FF3A
:10940400D082D083E5822FF582E43583F583E0FFB3
:109414008F99AF6774EC2FF582E43462F583E0042E
:10942400F0801FAF6774E62FF582E43460F583742F
:1094340001F0AF6774DB2FF582E43460F583E4F068
:10944400C290209803029534C298AF6774DF2FF559
:1094540082E43460F583E4F0AF6774E82FF582E4C6
:109464003462F583E4F0AF6774D92FF582E4346095
:10947400F583E0FFAE6774DB2EF582E43460F58398
:10948400E0FEEEC39F5079AF677E00EF7F00FE746D
:10949400D92FF582745E3EF583C083C082AF6774B2
:1094A400DB2FF582E43460F583E0FFD082D083E5DE
:1094B400822FF582E43583F583E599F0AF677E006A
:1094C400EF7F00FE74D92FF582745E3EF583C0836E
:1094D400C082AF6774DB2FF582E43460F583E0FF6C
:1094E400D082D083E5822FF582E43583F583E0FFD3
:1094F400EFAF6774DB2FF582E43460F583E004F0AA
:10950400AF6774D92FF582E43460F583E0FFAE676A
:1095140074DB2EF582E43460F583E0FEEEC39F40F5
:109524000FAF6774EE2FF582E43462F5837401F0B3
:0D953400D007D006D0D0D082D083D0E03256
:10B94B00756800E568C39402400302BA17AF6874C8
:10B95B00E62FF582E43460F583E0FFEF700302BA63
:10B96B0012AF6874E42FF582E43460F583E004F0E1
:10B97B00AF6874E42FF582E43460F583E0FFEFD316
:10B98B009419500302BA12AF6874E42FF582E434B1
:10B99B0060F583E4F0AF6874E62FF582E43460F56C
:10B9AB0083E4F0AF6874DF2FF582E43460F583E055
:10B9BB0004F0AF6874DF2FF582E43460F583E0FFA9
:10B9CB00900AA1E0FEEFD39E403DAF6874E82FF5DF
:10B9DB0082E43462F5837401F075690CE569D394E4
:10B9EB004B5024AF687E00EF7F00FE74B42FF582BE
:10B9FB00744E3EF583AF69E5822FF582E43583F50E
:0CBA0B0083E4F0056980D5056802B94E9F
:01BA1700220C
:07000300313233343536378A
:0BA2B400906842EBF0A3EAF0A3E9F091
:10A2BF00906842E0FBA3E0FAA3E0F98B3E8A3F8966
:10A2CF0040753D0090684CE0FFE53DC39F504590C1
:10A2DF006845E0FBA3E0FAA3E0F9128E0FFF906848
:10A2EF0042E0FBA3E0FAA3E0F9128E0FFEEEB507F2
:10A2FF0016906843E475F001128EF0906846E4758D
:10A30F00F001128EF0800990684CE0FFEF04F53DEC
:10A31F00053D80B090684CE0FFE53DB507067F0234
:10A32F002202A41DAB3EAA3FA940906842EBF0A3C6
:10A33F00EAF0A3E9F0753D0090684CE0FFE53DC3FE
:10A34F009F5048906842E0FBA3E0FAA3E0F9128E19
:10A35F000FFF906848E0FCA3E0FD8D828C83E0FE48
:10A36F00EFB5061A906843E475F001128EF090680D
:10A37F0049E004F07006906848E004F080099068A6
:10A38F004CE0FFEF04F53D053D80AD90684CE0FFDC
:10A39F00E53DB507057F00228074AB3EAA3FA9407B
:10A3AF00906842EBF0A3EAF0A3E9F0753D009068E6
:10A3BF004CE0FFE53DC39F5048906842E0FBA3E0AF
:10A3CF00FAA3E0F9128E0FFF90684AE0FCA3E0FDBC
:10A3DF008D828C83E0FEEFB5061A906843E475F02A
:10A3EF0001128EF090684BE004F0700690684AE01E
:10A3FF0004F0800990684CE0FFEF04F53D053D80C7
:10A40F00AD90684CE0FFE53DB507037F01227F0368
:01A41F00221A
:10BFA9009068A1EFF09068A2EBF0A3EAF0A3E9F0A2
:10BFB900787076009068A574FFF09068A674FFF019
:10BFC900786F76019068A1E0FF786FE6FEEED39F67
:10BFD90050509068A2E0FBA3E0FAA3E0F9128E0F9B
:10BFE900FF9068A5E0FEEE6FFF7870A6077870E60F
:10BFF900FFEF908F5F93FF9068A6E0FEEE6FFF90D2
:10C0090068A5EFF07870E6FFEF90905F93FF906876
:10C01900A6EFF09068A3E475F001128EF0786F0630
:10C0290080A29068A6E0FF9068A5E0FEEE4FFFEFC2
:07C0390060037F00227F017C
:01C0400022DD
:0BCA5B0090688EEBF0A3EAF0A3E9F076
:10CA660078717600906894E0FF7871E6FEEEC39FD9
:10CA7600503790688EE0FBA3E0FAA3E0F9128E0F20
:10CA8600FF906891E0FBA3E0FAA3E0F9EF128E5560
:10CA960090688FE475F001128EF0906892E475F05C
:09CAA60001128EF078710680BBCC
:01CAAF002264
:10695C00AF4174D72FF582E4345EF5837401F09067
:10696C00668EE0FFEF6015905ED7E0FFEF600D9054
:10697C005E11E4F0905E127401F0801B90668DE065
:10698C00FFEF6013905ED8E0FFEF600B905E117428
:10699C0001F0905E12E4F090660CE004F0905DFE65
:1069AC007401F0905DFF7401F0905E007401F09042
:1069BC0063FCE0FFEF70030270189063FAE4F09050
:1069CC0063FCE4F09062F4E0FF7B017A6379FE12E1
:1069DC00BFA9EF7003026FFA90674B7401F07B0153
:1069EC007A6379FEC003C002C0017B017A5E79CE66
:1069FC00906891EBF0A3EAF0A3E9F0906894740727
:106A0C00F0D001D002D00312CA5B906405E0FF9075
:106A1C00594AEFF0906406E0FF905E15EFF0906439
:106A2C0007E0FF905E16EFF0906408E0FF905E17B1
:106A3C00EFF07B017A5E79CEC003C002C0017BFF10
:106A4C007A007903906845EBF0A3EAF0A3E9F07EB5
:106A5C005E7F03906848EEF0A3EFF07E5E7F0A90B5
:106A6C00684AEEF0A3EFF090684C7407F0D001D0B8
:106A7C0002D00312A2B48F41E54164026003026D9F
:106A8C006090594AE0FFEF640370657B017A5E7990
:106A9C001512C9A87B007A2079007800C3128F1CCC
:106AAC006003027013905EAD7401F090640AE0FF15
:106ABC00905944EFF090640BE0FF905945EFF09043
:106ACC00640CE0FF905946EFF090640DE0FF905994
:106ADC0047EFF090640EE0FF905948EFF090640F90
:106AEC00E0FF905949EFF090660CE004F00270134F
:106AFC0090594AE0FFEF64266003026C227B017A16
:106B0C005E791512C9A87B007A2079007800C3122F
:106B1C008F1C7039905D5E7401F07B017A6379FE95
:106B2C00C003C002C0017B017A5E7918906891EBBA
:106B3C00F0A3EAF0A3E9F09062F4E0FF906894EF20
:106B4C00F0D001D002D00312CA5B0270137B017A21
:106B5C005E791512C9A87B017A2079007800C312DE
:106B6C008F1C701F9064FE7401F09065AF7401F07F
:106B7C0090660D7401F09062F5E4F09065DAE4F043
:106B8C000270137B017A5E791512C9A87B027A20F8
:106B9C0079007800C3128F1C70279066A2E0FFEF7B
:106BAC00601F9065307401F09065AF7401F09065D2
:106BBC00DC7401F09062F5E4F09065DAE4F00270B8
:106BCC00137B017A5E791512C9A87B037A307900A0
:106BDC007800C3128F1C60030270139065917401CE
:106BEC00F09065B17401F07B017A64790AC003C03E
:106BFC0002C0017B017A6579E2906891EBF0A3EA1F
:106C0C00F0A3E9F09068947410F0D001D002D00396
:106C1C0012CA5B02701390594AE0FFEF6423707044
:106C2C007B017A5E791512C9A87B007A20790078ED
:106C3C0000C3128F1C7036905B567401F07B017A86
:106C4C006379FEC003C002C0017B017A5D79669056
:106C5C006891EBF0A3EAF0A3E9F09062F4E0FF9006
:106C6C006894EFF0D001D002D00312CA5B7B017A9A
:106C7C005E791512C9A87B007A2179007800C312BD
:106C8C008F1C6003027013905EAC7401F0027013E1
:106C9C0090594AE0FFEF64136003026D4A7B017A5E
:106CAC005E791512C9A87B007A9079007800C3121E
:106CBC008F1C7039905D637401F07B017A6379FEEF
:106CCC00C003C002C0017B017A5E79B0906891EB81
:106CDC00F0A3EAF0A3E9F09062F4E0FF906894EF7F
:106CEC00F0D001D002D00312CA5B0270137B017A80
:106CFC005E791512C9A87B007A6079007800C312FE
:106D0C008F1C7017905B597401F0905ED67401F073
:106D1C00905EAAE4F0A3E4F00270137B017A5E7932
:106D2C001512C9A87B007A8079007800C3128F1CD9
:106D3C006003027013905D5B7401F0027013905944
:106D4C004AE0FFEF64166003027013905D5A740101
:106D5C00F0027013E5416009E541640160030270C3
:106D6C001390594AE0FFEF64067062AF4174D72F5D
:106D7C00F582E4345EF5837401F090668EE0FFEFEB
:106D8C006015905ED7E0FFEF600D905E11E4F0901F
:106D9C005E127401F0801B90668DE0FFEF60139023
:106DAC005ED8E0FFEF600B905E117401F0905E1204
:106DBC00E4F090660CE004F0905DFE7401F0905DE0
:106DCC00FF7401F0905E007401F002701390594A48
:106DDC00E0FFEF64266003026E807B017A5E79151A
:106DEC0012C9A87B007A3079007800C3128F1C700E
:106DFC0012AF4174542FF582E43459F5837401F0C9
:106E0C000270137B017A5E791512C9A87B017A3066
:106E1C0079007800C3128F1C7012AF4174612FF58A
:106E2C0082E4345DF5837401F00270137B017A5EA9
:106E3C00791512C9A87B027A3079007800C3128FB9
:106E4C001C600302701390640AE0FF7E00EF7F0069
:106E5C00FE90640BE0FD7C00EF2DFFEE3CFEAD419F
:106E6C00ED25E024C9F582E43450F583EEF0A3EF70
:106E7C00F002701390594AE0FFEF6436704EAF4148
:106E8C0074A62FF582E4345EF5837401F07B017AED
:106E9C006379FEC003C002C001AF417E00EF7F00EA
:106EAC00FE745A2FF9745B3EFA7B01906891EBF0FB
:106EBC00A3EAF0A3E9F09062F4E0FF906894EFF09D
:106ECC00D001D002D00312CA5B02701390594AE071
:106EDC00FFEF6433704EAF4174FA2FF582E4345DEA
:106EEC00F5837401F07B017A6379FEC003C002C0A4
:106EFC0001AF417E00EF7F00FE74562FF974593EAE
:106F0C00FA7B01906891EBF0A3EAF0A3E9F09062B0
:106F1C00F4E0FF906894EFF0D001D002D00312CAD5
:106F2C005B02701390594AE0FFEF64236003027018
:106F3C0013AF4174572FF582E4345BF583E0FFEF18
:106F4C007012AF4174572FF582E4345BF5837401F2
:106F5C00F0027013AF4174F82FF582E4345DF583C1
:106F6C00E0FFEF7003027013AF4174F82FF582E469
:106F7C00345DF583E4F090660CE004F0AF417E00E4
:106F8C007C047DB3128E89740A2FF974453EFA7B0A
:106F9C000190691CEBF0A3EAF0A3E9F0AF41745F38
:106FAC002FF582E4345DF583E0FF90691CE0FBA3D0
:106FBC00E0FAA3E0F97582B0758304EF128E67AF27
:106FCC004174F42FF582E4345DF583E0FFEF603714
:106FDC00AF4174F42FF582E4345DF583E4F0AF41F6
:106FEC0074572FF582E4345BF583E4F080199067D5
:106FFC004BE4F09062F0E4F09062F6E4F09062F70B
:0F700C00E4F09062F9E4F09062F8E4F01275CBD2
:01701B002252
:1075CB00754200E542C394024003027B57905D6312
:1075DB00E0FFEF6064905D63E4F0905E13E0FFEF1B
:1075EB007008905E14E0FFEF60499066A3E0FFEF38
:1075FB0060397B017A5E79B0C003C002C0017B01A8
:10760B007A6679B29068AAEBF0A3EAF0A3E9F0D01E
:10761B0001D002D00312BE72EF600890660E7401A7
:10762B00F080169065DD7401F0800E90660E74018B
:10763B00F080069065DD7401F0905B59E0FFEF7010
:10764B00030276DC905B59E4F0905DFD7401F090E1
:10765B005E13E0FFEF603990671DE4F090675074A4
:10766B0001F0905946E0FF90594BEFF0905947E0ED
:10767B00FF90594DEFF0905948E0FF905EA8EFF066
:10768B00905949E0FF905DF6EFF0905D64E004F0F7
:10769B00905E14E0FFEF603990671EE4F09067187E
:1076AB007401F0905946E0FF90594CEFF090594718
:1076BB00E0FF90594EEFF0905948E0FF905EA9EF34
:1076CB00F0905949E0FF905DF7EFF0905D65E004B5
:1076DB00F0905D5BE0FFEF700B905DFCE0FFEF70F7
:1076EB0003027893905D5BE4F0905DFCE4F0905EB8
:1076FB00CD7401F0AF42EF25E02495F582E43467B9
:10770B00F583E4F0A3E4F0905ED6E4F0905EAAE497
:10771B00F0A3E4F0905E13E0FFEF70030277D990D3
:10772B005D64E0FF905ECBE0FEEE6F70030277D4FA
:10773B00905D64E0FF905ECBEFF090671D7401F0FD
:10774B00906750E4F09045007401F0905946E0FFCB
:10775B0090594FEFF0905947E0FF905951EFF0904F
:10776B005948E0FF905EC9EFF0905949E0FF905EF9
:10777B0001EFF0754300E543C3940C5017AF43EF93
:10778B0025E02400F582E43465F583E4F0A3E4F00E
:10779B00054380E2754300905EBBE0FFE543C39F6A
:1077AB005027AF4374BC2FF582E4345EF583E0FFC2
:1077BB007E00AD43ED25E02400F582E43465F583CE
:1077CB00EEF0A3EFF0054380CE905E13E4F0905EF5
:1077DB0014E0FFEF7003027893905D65E0FF905E1D
:1077EB00CCE0FEEE6F700302788E905D65E0FF904B
:1077FB005ECCEFF090671E7401F0906718E4F09088
:10780B0045017401F0905946E0FF905950EFF0900C
:10781B005947E0FF905952EFF0905948E0FF905EC6
:10782B00CAEFF0905949E0FF905E02EFF07543000C
:10783B00E543C3940C5017AF43EF25E02418F582B2
:10784B00E43465F583E4F0A3E4F0054380E275438B
:10785B0000905EBBE0FFE543C39F5027AF4374BC72
:10786B002FF582E4345EF583E0FF7E00AD43ED251A
:10787B00E02418F582E43465F583EEF0A3EFF00510
:10788B004380CE905E14E4F0905EADE0FFEF600BB2
:10789B00905EADE4F0905ED57401F0905D5AE0FF20
:1078AB00EF601F905D5AE4F09065AFE4F09065DAFD
:1078BB007401F09065F2E4F09065DCE4F090660DF5
:1078CB00E4F0905D5EE0FFEF606B905D5EE4F07B5B
:1078DB00017A5E7924C003C002C0017B017A66790C
:1078EB0092906891EBF0A3EAF0A3E9F0906894749E
:1078FB0080F0D001D002D00312CA5B7B017A66798B
:10790B00927F8012BFA9EF70079065DEE4F08025AF
:10791B009065DE7401F0128A2A90669074F0F0A3E1
:10792B00E4F0906690E0FCA3E0FD7B017A6679922F
:10793B007F8012C6F09065B1E0FFEF640160030237
:10794B007A049065B1E4F07B017A6579E2C003C0FB
:10795B0002C0017B017A667992906891EBF0A3EA01
:10796B00F0A3E9F0906894740FF0D001D002D0032B
:10797B0012CA5B9065F1E0FF9066DCEFF07C667DF0
:10798B00927F7E12C0418E448F45906710E545F083
:10799B00906711E544F0128A2A90669074F0F0A378
:1079AB00E4F0906690E0FCA3E0FD7B017A667992AF
:1079BB007F8012C6F07B017A667927906690E0FE95
:1079CB00A3E0FF906899EEF0A3EFF07F0F12CA06C9
:1079DB007B017A667936906690E0FEA3E0FFEF2498
:1079EB004AFFEE3400FE906899EEF0A3EFF07F01B2
:1079FB0012CA069064FF7401F0AF4274D72FF58260
:107A0B00E4345EF583E0FFEF7003027B32AF427428
:107A1B00D72FF582E4345EF583E4F09065D4E0FF74
:107A2B00EF64017073AF427E7BEF8EF0A4FFAEF07C
:107A3B0074942FF974093EFA7B0112C534AF42EFEF
:107A4B0075F00CA4240FF582E43466F583E0FFEFA8
:107A5B00D394605003027B2DAF42EF75F00CA4243E
:107A6B000FF582E43466F583E0FFEFC394654003C2
:107A7B00027B2DE542700590674EE4F0E542B401C0
:107A8B000590674FE4F0AF4274AE2FF582E4345E9D
:107A9B00F5837401F0027B2D9065D4E0FFEFB40207
:107AAB001AAF427EADEF8EF0A4FFAEF0743F2FF90C
:107ABB0074553EFA7B0112C4C580679065D4E0FF14
:107ACB00EFB4031AAF427E007C047DB3128E89742F
:107ADB000B2FF974003EFA7B0112C5A3804490650D
:107AEB00D4E0FFEFB4051AAF427ECBEF8EF0A4FFCC
:107AFB00AEF074B32FF9740A3EFA7B0112C61280F2
:107B0B00219065D4E0FFEFB40618AF427E007C1CD9
:107B1B007D23128E8974B82FF9740C3EFA7B0112F7
:107B2B00C6819065D4E4F0AF4274612FF582E434E2
:107B3B005DF583E0FFEF600FAF4274132FF582E426
:0C7B4B00345EF5837401F005420275CE33
:017B5700220B
:0BC9A80090691FEBF0A3EAF0A3E9F098
:10C9B30075460090691FE0FBA3E0FAA3E0F9128E2D
:10C9C3000FFF8F47906920E475F001128EF0906994
:10C9D3001FE0FBA3E0FAA3E0F9128E0FFF8F48904C
:10C9E3006920E475F001128EF090691FE0FBA3E06B
:10C9F300FAA3E0F9128E0FFF8F49AF49AE48AD4756
:02CA0300AC463F
:01CA0500220E
:0BBE72009068A7EBF0A3EAF0A3E9F052
:10BE7D009068A7E0FBA3E0FAA3E0F975820B758348
:10BE8D0000128E28FF7E00EF2408FFEE3400FE9096
:10BE9D0068A7E0FBA3E0FAA3E0F9E92FF9EA3EFA7F
:10BEAD00AE02AF018E4C8F4D754A01E54AD3940A0F
:10BEBD00504D754B01E54BD3940450379068AAE073
:10BECD00FBA3E0FAA3E0F9128E0FFFAC4CAD4D8D44
:10BEDD00828C83E0FEEFB5061A054DE54D70020527
:10BEED004C9068ABE475F001128EF0800280040571
:10BEFD004B80C2E54BB405037F0122054A80AC7F20
:01BF0D000033
:01BF0E002210
:10474D0090692BEFF09062F1E0FFEF6003025DB531
:10475D0090660EE0FFEF70030247F390660EE4F0F3
:10476D007BFF7A007903C003C002C0017B017A662A
:10477D00793A906891EBF0A3EAF0A3E9F090689490
:10478D007407F0D001D002D00312CA5B90668A7410
:10479D0013F07E657FDF9068B1EEF0A3EFF07F0040
:1047AD007E507D007C0012C7587E667F3AC006C0E1
:1047BD00077C657DDF90668AE0FB90686FE4F07E94
:1047CD00627FFA906870EEF0A3EFF0D007D006127A
:1047DD00A1429062F2EFF09063FBE4F043AA0290E5
:1047ED0062F17401F0229065DDE0FFEF7003024885
:1047FD00899065DDE4F07BFF7A007903C003C00288
:10480D00C0017B017A66793A906891EBF0A3EAF0EA
:10481D00A3E9F09068947407F0D001D002D0031290
:10482D00CA5B90668A7413F07E657FDF9068B1EE87
:10483D00F0A3EFF07F007E707D007C0012C7587EE4
:10484D00667F3AC006C0077C657DDF90668AE0FB17
:10485D0090686FE4F07E627FFA906870EEF0A3EFDF
:10486D00F0D007D00612A1429062F2EFF09063FBF8
:10487D00E4F043AA029062F17401F022905DFDE034
:10488D00FFEF7003024928905DFDE4F09065D8E4D8
:10489D00F0A37401F07BFF7A007903C003C002C05E
:1048AD00017B017A66793A906891EBF0A3EAF0A367
:1048BD00E9F09068947407F0D001D002D00312CAC9
:1048CD005B90668A7413F07E657FDF9068B1EEF0C1
:1048DD00A3EFF07F007E607D007C0012C7587E66DE
:1048ED007F3AC006C0077C657DDF90668AE0FB904D
:1048FD00686FE4F07E627FFA906870EEF0A3EFF0DF
:10490D00D007D00612A1429062F2EFF09063FBE463
:10491D00F043AA029062F17401F022905ECDE0FFA7
:10492D00EF70030249C6905ECDE4F09065D8E4F0D7
:10493D00A3E4F07BFF7A007903C003C002C0017BC2
:10494D00017A66793A906891EBF0A3EAF0A3E9F069
:10495D009068947407F0D001D002D00312CA5B9016
:10496D00668A7413F07E657FDF9068B1EEF0A3EF79
:10497D00F07F007E807D007C0012C7587E667F3AF6
:10498D00C006C0077C657DDF90668AE0FB90686F8E
:10499D00E4F07E627FFA906870EEF0A3EFF0D0073E
:1049AD00D00612A1429062F2EFF09063FBE4F04367
:1049BD00AA029062F17401F0229064FEE0FFEF70A4
:1049CD0003024A5C9064FEE4F07BFF7A007903C039
:1049DD0003C002C0017B017A66793A906891EBF0D1
:1049ED00A3EAF0A3E9F09068947407F0D001D00227
:1049FD00D00312CA5B90668A7426F07E657FDF90C5
:104A0D0068B1EEF0A3EFF07F017E207D007C0012F7
:104A1D00C7587E667F3AC006C0077C657DDF90660D
:104A2D008AE0FB90686FE4F07E627FFA906870EE2A
:104A3D00F0A3EFF0D007D00612A1429062F2EFF092
:104A4D009063FBE4F043AA029062F17401F02290AE
:104A5D006530E0FFEF7003024AF2906530E4F07BC1
:104A6D00FF7A007903C003C002C0017B017A667929
:104A7D003A906891EBF0A3EAF0A3E9F09068947492
:104A8D0007F0D001D002D00312CA5B90668A74265B
:104A9D00F07E657FDF9068B1EEF0A3EFF07F027ED0
:104AAD00207D007C0012C7587E667F3AC006C00785
:104ABD007C657DDF90668AE0FB90686FE4F07E6236
:104ACD007FFA906870EEF0A3EFF0D007D00612A138
:104ADD00429062F2EFF09063FBE4F043AA02906221
:104AED00F17401F0229065AFE0FFEF7003024C29E5
:104AFD009062F5E0FFEF6003024C299065DAE0FF6C
:104B0D00EF6003025DB59065F2E004F09065F2E0B0
:104B1D00FFEFD3940A401B9065DA7401F09065F2B3
:104B2D00E4F09065AFE4F09065DCE4F090660DE4A0
:104B3D00F0227BFF7A007903C003C002C0017B0124
:104B4D007A66793A906891EBF0A3EAF0A3E9F090D8
:104B5D0068947407F0D001D002D00312CA5B90663E
:104B6D008A7416F07E657FDF9068B1EEF0A3EFF0EA
:104B7D007F007E107D007C0012C7589065DCE0FF41
:104B8D00EF60427E667F3AC006C0077C657DDF9090
:104B9D00668AE0FB9068527406F0906853E4F07EEC
:104BAD00627FFA906854EEF0A3EFF07E667FA690D8
:104BBD006856EEF0A3EFF0D007D00612971A906268
:104BCD00F2EFF0804890660DE0FFEF60407E667F6B
:104BDD003AC006C0077C657DDF90668AE0FB906871
:104BED00527406F0906853E4F07E627FFA90685438
:104BFD00EEF0A3EFF07E667FAC906856EEF0A3EF7B
:104C0D00F0D007D00612971A9062F2EFF09063FB86
:104C1D00E4F043AA029062F17401F0229065DEE0A7
:104C2D00FFEF7003024CBF9065DEE4F07BFF7A006E
:104C3D007903C003C002C0017B017A66793A90689E
:104C4D0091EBF0A3EAF0A3E9F09068947407F0D02B
:104C5D0001D002D00312CA5B90668A7426F07E657D
:104C6D007FDF9068B1EEF0A3EFF07F007E207D0036
:104C7D007C0012C7587E667F3AC006C0077C657DF2
:104C8D00DF90668AE0FB90686FE4F07E627FFA90B9
:104C9D006870EEF0A3EFF0D007D00612A14290623B
:104CAD00F2EFF09063FBE4F043AA029062F174011D
:104CBD00F022905B56E0FFEF7003024D67905B565C
:104CCD00E4F07BFF7A007903C003C002C0017B01D1
:104CDD007A66793A906891EBF0A3EAF0A3E9F09047
:104CED0068947407F0D001D002D00312CA5B9066AD
:104CFD008A7423F07E657FDF9068B1EEF0A3EFF04C
:104D0D007F007E207D007C0012C7587E667F3AC0F2
:104D1D0006C0077C657DDF90668AE0FB9068527463
:104D2D0080F0906853E4F07E627FFA906854EEF064
:104D3D00A3EFF07E667F92906856EEF0A3EFF0D071
:104D4D0007D00612971A9062F2EFF09063FBE4F031
:104D5D0043AA029062F17401F022905EACE0FFEF85
:104D6D007003024E0F905EACE4F07BFF7A00790386
:104D7D00C003C002C0017B017A66793A906891EB5D
:104D8D00F0A3EAF0A3E9F09068947407F0D001D095
:104D9D0002D00312CA5B90668A7423F07E657FDFB2
:104DAD009068B1EEF0A3EFF07F007E217D007C00D6
:104DBD0012C7587E667F3AC006C0077C657DDF90BE
:104DCD00668AE0FB9068527408F0906853E4F07EB8
:104DDD00627FFA906854EEF0A3EFF07E677FD49077
:104DED006856EEF0A3EFF0D007D00612971A906236
:104DFD00F2EFF09063FBE4F043AA029062F17401CC
:104E0D00F02290692BE0FF74AC2FF582E43465F548
:104E1D0083E0FFEF7003024EF990692BE0FF7457AA
:104E2D002FF582E4345BF583E0FFEF7003024EF95A
:104E3D0090692BE0FF7E07EF8EF0A4FFAEF07403B8
:104E4D002FF9745E3EFA7B01C003C002C0017B01E5
:104E5D007A66793A906891EBF0A3EAF0A3E9F090C5
:104E6D0068947407F0D001D002D00312CA5B90662B
:104E7D008A7423F07E657FDF9068B1EEF0A3EFF0CA
:104E8D007F007E507D007C0012C75890692BE0FF9B
:104E9D007E007C047DB3128E89740A2FF974453E11
:104EAD00FA7B01906806EBF0A3EAF0A3E9F09069B4
:104EBD002BE0FFC0077C667D3A7A657BDF90668AC2
:104ECD00E0FF906803EFF07E627FFA906804EEF0E9
:104EDD00A3EFF0D0071287229062F2EFF09063FB00
:104EED00E4F043AA029062F17401F02290692BE084
:104EFD00FF74542FF582E43459F583E0FFEF70030E
:104F0D00024FCB90692BE0FF74542FF582E4345996
:104F1D00F583E4F090692BE0FF74062FF582E434FD
:104F2D0045F5837401F090692BE0FF7E07EF8EF05D
:104F3D00A4FFAEF074032FF9745E3EFA7B01C0033B
:104F4D00C002C0017B017A66793A906891EBF0A3BB
:104F5D00EAF0A3E9F09068947407F0D001D002D084
:104F6D000312CA5B90668A7426F07E657FDF9068B7
:104F7D00B1EEF0A3EFF07F007E307D007C0012C714
:104F8D00587E667F3AC006C0077C657DDF90668AD5
:104F9D00E0FB90686FE4F07E627FFA906870EEF04F
:104FAD00A3EFF0D007D00612A1429062F2EFF0907D
:104FBD0063FBE4F043AA029062F17401F022906960
:104FCD002BE0FF74612FF582E4345DF583E0FFEF94
:104FDD00700302508B90692BE0FF74612FF582E412
:104FED00345DF583E4F090692BE0FF7E07EF8EF0E2
:104FFD00A4FFAEF074032FF9745E3EFA7B01C0037B
:10500D00C002C0017B017A66793A906891EBF0A3FA
:10501D00EAF0A3E9F09068947407F0D001D002D0C3
:10502D000312CA5B90668A7426F07E657FDF9068F6
:10503D00B1EEF0A3EFF07F017E307D007C0012C752
:10504D00587E667F3AC006C0077C657DDF90668A14
:10505D00E0FB90686FE4F07E627FFA906870EEF08E
:10506D00A3EFF0D007D00612A1429062F2EFF090BC
:10507D0063FBE4F043AA029062F17401F02290699F
:10508D002BE0FF74CA2FF582E43467F583E0FFEF60
:10509D00700302514790692BE0FF74CA2FF582E42B
:1050AD003467F583E4F090692BE0FF7E07EF8EF017
:1050BD00A4FFAEF074032FF9745E3EFA7B01C003BA
:1050CD00C002C0017B017A66793A906891EBF0A33A
:1050DD00EAF0A3E9F09068947407F0D001D002D003
:1050ED000312CA5B90668A7436F090692BE0FFEF6D
:1050FD0075F003A424BEF582E43467F583AD82AC6C
:10510D0083C004C0057E667F3A90668AE0FB906896
:10511D006FE4F07C627DFA906870ECF0A3EDF0D056
:10512D0005D00412A1429062F2EFF09063FBE4F01F
:10513D0043AA029062F17401F02290692BE0FF7492
:10514D00C62FF582E43467F583E0FFEF700302525A
:10515D007590692BE0FF74C62FF582E43467F583F3
:10516D00E4F090692BE0FF7E07EF8EF0A4FFAEF028
:10517D0074032FF9745E3EFA7B01C003C002C001B7
:10518D007B017A66793A906891EBF0A3EAF0A3E996
:10519D00F09068947407F0D001D002D00312CA5B6E
:1051AD0090668A7433F090692BE0FFEF75F003A4DD
:1051BD0024CEF582E43467F583E0FF9065DFEFF0F0
:1051CD0090692BE0FFEF75F003A424CFF582E43452
:1051DD0067F583E0FF9065E0EFF090692BE0FFEF5E
:1051ED0075F003A424D0F582E43467F583E0FF90D5
:1051FD0065E1EFF07E667F3AC006C0077C657DDF16
:10520D0090668AE0FB90692BE0FF74C82FF582E46D
:10521D003467F583E0FF906852EFF0906853E4F047
:10522D007E627FFA906854EEF0A3EFF090692BE068
:10523D00FF7E00EF7F00FE74142FF58274533EF550
:10524D0083AF82AE83906856EEF0A3EFF0D007D017
:10525D000612971A9062F2EFF09063FBE4F043AA06
:10526D00029062F17401F022906591E0FFEF7003FE
:10527D0002532D9064FFE0FFEF700302532D9064F5
:10528D00FFE4F0906591E4F07BFF7A007903C003B1
:10529D00C002C0017B017A66793A906891EBF0A368
:1052AD00EAF0A3E9F09068947407F0D001D002D031
:1052BD000312CA5B90668A7426F07E657FDF906864
:1052CD00B1EEF0A3EFF07F037E307D007C0012C7BE
:1052DD00587E667F3AC006C0077C657DDF90668A82
:1052ED00E0FB9068527410F0906853E4F07E627F9A
:1052FD00FA906854EEF0A3EFF07E667F2790685623
:10530D00EEF0A3EFF0D007D00612971A9062F2EFED
:10531D00F09063FBE4F043AA029062F17401F02275
:10532D0090692BE0FF748D2FF582E43466F583E0F0
:10533D00FFEF70030259EF905DFEE0FFEF70030287
:10534D0059EF90692BE0FF74112FF582E4345EF56F
:10535D0083E0FFEF70030259EF90692BE0FF74FFBC
:10536D002FF582E4345DF583E0FFEF70030259EF12
:10537D00905DFEE4F090678BE4F0A3E4F090692B70
:10538D00E0FFEF700D905DFF7401F0905E00E4F0B2
:10539D00800B905DFFE4F0905E007401F090692B3E
:1053AD00E0FF74D62FF582E43465F583E0FFEF70EE
:1053BD00030254EB9065D4E0FFEF6402600B90653F
:1053CD00D4E0FFEF60030254EB90692BE0FF7E0702
:1053DD00EF8EF0A4FFAEF074032FF9745E3EFA7BEE
:1053ED0001C003C002C0017B017A66793A906891D1
:1053FD00EBF0A3EAF0A3E9F09068947407F0D00104
:10540D00D002D00312CA5B90668A7406F07E657F67
:10541D00DF9068B1EEF0A3EFF07F007E307D007C71
:10542D000012C75890692BE0FF7EADEF8EF0A4FF00
:10543D00AEF0743F2FF974553EFA7B0112CCC5C006
:10544D0003C002C00190692BE0FF7E11EF8EF0A426
:10545D00FFAEF074B22FF974653EFA7B01A801AC72
:10546D0002AD03D001D002D0037E007F11128DE971
:10547D0090692BE0FFEF75F011A424B2F582E434AE
:10548D0065F583AF82AE83906856EEF0A3EFF07EA4
:10549D00667F3AC006C0077C657DDF90668AE0FBBB
:1054AD009068527411F09068537401F07E627FFA27
:1054BD00906854EEF0A3EFF0D007D00612971A9033
:1054CD0062F2EFF09063FBE4F09065D47402F04368
:1054DD00AA0290674BE4F09062F17401F02290699A
:1054ED002BE0FF74412FF582E43466F583E0FFEF86
:1054FD00700302562C9065D4E0FFEF6401600B90B1
:10550D0065D4E0FFEF600302562C90692BE0FF7E1F
:10551D0007EF8EF0A4FFAEF074032FF9745E3EFA20
:10552D007B01C003C002C0017B017A66793A9068A5
:10553D0091EBF0A3EAF0A3E9F09068947407F0D032
:10554D0001D002D00312CA5B90668A7406F07E65A4
:10555D007FDF9068B1EEF0A3EFF07F007E207D003D
:10556D007C0012C75890692BE0FF7E7BEF8EF0A474
:10557D00FFAEF074942FF974093EFA7B0112CD073A
:10558D00C003C002C00190692BE0FF7E0CEF8EF0CE
:10559D00A4FFAEF0740F2FF974663EFA7B01A801DB
:1055AD00AC02AD03D001D002D0037E007F0C128D72
:1055BD00E990692BE0FFEF75F00CA4240FF582E460
:1055CD003466F583AF82AE83906856EEF0A3EFF0AC
:1055DD007E667F3AC006C0077C657DDF90668AE0F7
:1055ED00FB906852740CF09068537401F07E627FEA
:1055FD00FA906854EEF0A3EFF0D007D00612971A88
:10560D009062F2EFF09063FBE4F09065D47401F0DA
:10561D0043AA0290674BE4F09062F17401F022907E
:10562D00692BE0FF74382FF582E43466F583E0FFD3
:10563D00EF700302576D9065D4E0FFEF6403600BCC
:10564D009065D4E0FFEF600302576D90692BE0FF8A
:10565D007E07EF8EF0A4FFAEF074032FF9745E3E5B
:10566D00FA7B01C003C002C0017B017A66793A90D2
:10567D006891EBF0A3EAF0A3E9F09068947407F059
:10568D00D001D002D00312CA5B90668A7406F07EF8
:10569D00657FDF9068B1EEF0A3EFF07F007E407D77
:1056AD00007C0012C75890692BE0FF7E007C047DC2
:1056BD00B3128E89740B2FF974003EFA7B0112CD53
:1056CD0049C003C002C00190692BE0FF7E0CEF8E34
:1056DD00F0A4FFAEF074F32FF974653EFA7B01A8C8
:1056ED0001AC02AD03D001D002D0037E007F0C12BD
:1056FD008DE990692BE0FFEF75F00CA424F3F58292
:10570D00E43465F583AF82AE83906856EEF0A3EF77
:10571D00F07E667F3AC006C0077C657DDF90668AA5
:10572D00E0FB906852740CF09068537401F07E6247
:10573D007FFA906854EEF0A3EFF0D007D0061297E1
:10574D001A9062F2EFF09063FBE4F09065D474036D
:10575D00F043AA0290674BE4F09062F17401F022DD
:10576D0090692BE0FF746D2FF582E43466F583E0CC
:10577D00FFEF70030258AE9065D4E0FFEF64056053
:10578D000B9065D4E0FFEF60030258AE90692BE0FB
:10579D00FF7E07EF8EF0A4FFAEF074032FF9745E59
:1057AD003EFA7B01C003C002C0017B017A66793AE3
:1057BD00906891EBF0A3EAF0A3E9F0906894740778
:1057CD00F0D001D002D00312CA5B90668A7406F045
:1057DD007E657FDF9068B1EEF0A3EFF07F007E6015
:1057ED007D007C0012C75890692BE0FF7ECBEF8EB9
:1057FD00F0A4FFAEF074B32FF9740A3EFA7B0112D8
:10580D00CD8BC003C002C00190692BE0FF7E14EF69
:10581D008EF0A4FFAEF074452FF974663EFA7B014D
:10582D00A801AC02AD03D001D002D0037E007F14DD
:10583D00128DE990692BE0FFEF75F014A42445F566
:10584D0082E43466F583AF82AE83906856EEF0A3A2
:10585D00EFF07E667F3AC006C0077C657DDF9066FF
:10586D008AE0FB9068527414F09068537401F07ED6
:10587D00627FFA906854EEF0A3EFF0D007D00612D5
:10588D00971A9062F2EFF09063FBE4F09065D47498
:10589D0005F043AA0290674BE4F09062F17401F0B9
:1058AD002290692BE0FF74922FF582E43465F58325
:1058BD00E0FFEF7003025DB59065D4E0FFEF640685
:1058CD00600B9065D4E0FFEF6003025DB590692B2E
:1058DD00E0FF7E07EF8EF0A4FFAEF074032FF97496
:1058ED005E3EFA7B01C003C002C0017B017A66797E
:1058FD003A906891EBF0A3EAF0A3E9F09068947404
:10590D0007F0D001D002D00312CA5B90668A7406EC
:10591D00F07E657FDF9068B1EEF0A3EFF07F007E43
:10592D00707D007C0012C75890692BE0FF7E007CD3
:10593D001C7D23128E8974B82FF9740C3EFA7B01ED
:10594D0012CDCDC003C002C00190692BE0FF7E30A7
:10595D00EF8EF0A4FFAEF074312FF974653EFA7B33
:10596D0001A801AC02AD03D001D002D0037E007FAF
:10597D0030128DE990692BE0FFEF75F030A42431E2
:10598D00F582E43465F583AF82AE83906856EEF010
:10599D00A3EFF07E667F3AC006C0077C657DDF9081
:1059AD00668AE0FB9068527430F09068537401F091
:1059BD007E627FFA906854EEF0A3EFF0D007D00628
:1059CD0012971A9062F2EFF09063FBE4F09065D4B9
:1059DD007406F043AA0290674BE4F09062F17401F3
:1059ED00F022906671E0FFEF7003025CD990667152
:1059FD00E4F07BFF7A007903C003C002C0017B0194
:105A0D007A66793A906891EBF0A3EAF0A3E9F09009
:105A1D0068947407F0D001D002D00312CA5B90666F
:105A2D008A7403F07E657FDF9068B1EEF0A3EFF02E
:105A3D007F007E207D007C0012C7587B017A5E7945
:105A4D0003C003C002C0017B017A63795E90689147
:105A5D00EBF0A3EAF0A3E9F09068947407F0D0019D
:105A6D00D002D00312CA5B7B017A557933C003C0D3
:105A7D0002C0017B017A637965906891EBF0A3EA2E
:105A8D00F0A3E9F09068947406F0D001D002D00331
:105A9D0012CA5B7B017A5079BBC003C002C0017B87
:105AAD00017A63796B906891EBF0A3EAF0A3E9F0CA
:105ABD009068947406F0D001D002D00312CA5B7BBB
:105ACD00017A4E79F9C003C002C0017B017A637976
:105ADD0071906891EBF0A3EAF0A3E9F090689474EB
:105AED0002F0D001D002D00312CA5B7B017A5E793D
:105AFD000AC003C002C0017B017A6379739068917B
:105B0D00EBF0A3EAF0A3E9F09068947407F0D001EC
:105B1D00D002D00312CA5B7B017A557939C003C01C
:105B2D0002C0017B017A63797A906891EBF0A3EA68
:105B3D00F0A3E9F09068947406F0D001D002D00380
:105B4D0012CA5B7B017A5079C1C003C002C0017BD0
:105B5D00017A637980906891EBF0A3EAF0A3E9F004
:105B6D009068947406F0D001D002D00312CA5B7B0A
:105B7D00017A4F79F9C003C002C0017B017A6379C4
:105B8D0086906891EBF0A3EAF0A3E9F09068947425
:105B9D0002F0D001D002D00312CA5B7B017A677983
:105BAD00D4C003C002C0017B017A637988906891EB
:105BBD00EBF0A3EAF0A3E9F09068947408F0D0013B
:105BCD00D002D00312CA5B7B017A0C79ACC003C042
:105BDD0002C0017B017A637990906891EBF0A3EAA2
:105BED00F0A3E9F09068947406F0D001D002D003D0
:105BFD0012CA5B7B017A557910C003C002C0017BCC
:105C0D00017A637996906891EBF0A3EAF0A3E9F03D
:105C1D009068947406F0D001D002D00312CA5B7B59
:105C2D00017A0C79B2C003C002C0017B017A63799D
:105C3D009C906891EBF0A3EAF0A3E9F0906894745E
:105C4D0006F0D001D002D00312CA5B7B017A5579E0
:105C5D0016C003C002C0017B017A6379A2906891DE
:105C6D00EBF0A3EAF0A3E9F09068947406F0D0018C
:105C7D00D002D00312CA5B7E667F3AC006C0077C95
:105C8D00657DDF90668AE0FB906852744AF09068FB
:105C9D00537401F07E627FFA906854EEF0A3EFF03A
:105CAD007E637F5E906856EEF0A3EFF0D007D006CE
:105CBD0012971A9062F2EFF09063FBE4F043AA02A0
:105CCD0090674BE4F09062F17401F0229065B0E0C2
:105CDD00FFEF7003025DB59065B0E4F07BFF7A00D5
:105CED007903C003C002C0017B017A66793A9068DE
:105CFD0091EBF0A3EAF0A3E9F09068947407F0D06B
:105D0D0001D002D00312CA5B90668A7403F09067CB
:105D1D0012E0FFEF70197E657FDF9068B1EEF0A3A2
:105D2D00EFF07F057E207D007C0012C758803890F3
:105D3D006716E0FFEF60197E657FDF9068B1EEF0CA
:105D4D00A3EFF07F047E207D007C0012C7588017E2
:105D5D007E657FDF9068B1EEF0A3EFF07F067E20C9
:105D6D007D007C0012C7587E667F3AC006C0077C56
:105D7D00657DDF90668AE0FB90686FE4F07E627F60
:105D8D00FA906870EEF0A3EFF0D007D00612A142A2
:105D9D009062F2EFF09063FBE4F043AA0290674B40
:095DAD00E4F09062F17401F022AF
:10BDD000905ED5E0FFEF704790668DE0FFEF703F1B
:10BDE00090668EE0FFEF7037906787E0FFEF70039B
:10BDF00002BE719058FBE0FFEF60089062E8E0FF40
:10BE0000EF60109058FBE0FFEF60669062E8E0FFA3
:10BE1000EF705E906787E4F09066717401F0229095
:10BE2000679BE0FFEF604A90668DE0FFEF70429005
:10BE3000668EE0FFEF703A9058FBE0FFEF600890ED
:10BE400062E8E0FFEF60109058FCE0FFEF602290A6
:10BE500062E9E0FFEF701A90679BE4F090667174FE
:10BE600001F0905ED5E4F0906787E4F090678DE490
:02BE7000F022BE
:10CF5400905ED5E0FFEF602390668DE0FFEF701BDD
:10CF640090668EE0FFEF7013906787E0FFEF600B31
:0CCF7400906787E4F09065B07401F02233
:10954100750800E508C394024003029719AF087E2D
:10955100007C047DB3128E89740B2FF974003EFADE
:109561007B0112C882EF70047F0180027F00AE0888
:1095710074382EF582E43466F583EFF0AF087E7B14
:10958100EF8EF0A4FFAEF074942FF974093EFA7BCC
:109591000112C820EF70047F0180027F00AE0874C1
:1095A100412EF582E43466F583EFF0AF087EADEF2E
:1095B1008EF0A4FFAEF0743F2FF974553EFA7B0193
:1095C10012C7BEEF70047F0180027F00AE0874D61F
:1095D1002EF582E43465F583EFF0AF087ECBEF8E94
:1095E100F0A4FFAEF074B32FF9740A3EFA7B0112B6
:1095F100C8E4EF70047F0180027F00AE08746D2E15
:10960100F582E43466F583EFF0AF087E007C1C7DC3
:1096110023128E8974B82FF9740C3EFA7B0112C99A
:1096210046EF70047F0180027F00AE0874922EF530
:1096310082E43465F583EFF0AF0874572FF582E4C7
:10964100345BF583E0FFEF6033AF087E007C047D7F
:10965100B3128E89740A2FF974453EFA7B01AF0863
:1096610012C2DDEF70047F0180027F00AE0874AC8E
:109671002EF582E43465F583EFF0800EAF0874AC0B
:109681002FF582E43465F583E4F0AF0874382FF5E3
:1096910082E43466F583E0FFEF7055AF0874412F23
:1096A100F582E43466F583E0FFEF7044AF08746D32
:1096B1002FF582E43466F583E0FFEF7033AF087471
:1096C100D62FF582E43465F583E0FFEF7022AF0811
:1096D10074AC2FF582E43465F583E0FFEF7011AFD0
:1096E1000874922FF582E43465F583E0FFEF60049E
:1096F1007F0180027F00AE08748D2EF582E434660E
:10970100F583EFF0AF0874112FF582E4345EF58331
:089711007401F0050802954403
:01971900222D
:06C758009068AD128F2D68
:10C75E009068ADE0FCA3E0FDA3E0FEA3E0FF8F0C2C
:10C76E008E0B8D0A8C099068B1E0FEA3E0FF8F82DC
:10C77E008E83E50AF09068B2E004F070069068B11E
:10C78E00E004F09068B1E0FEA3E0FF8F828E83E5B7
:10C79E000BF09068B2E004F070069068B1E004F01F
:0FC7AE009068B1E0FEA3E0FF8F828E83E50CF070
:01C7BD002259
:10A1420090686AEEF0A3EFF090686CECF0A3EDF08B
:05A1520090686EEBF0C7
:10A15700906870E0FEA3E0FF8E0E8F0F906870E0AE
:10A16700FEA3E0FF8F828E837430F0906871E00465
:10A17700F07006906870E004F0906870E0FEA3E06D
:10A18700FF8F828E83E4F0906871E004F070069090
:10A197006870E004F0750D00E50DC39407503C901E
:10A1A700686AE0FEA3E0FF8F828E83E0FF9068700D
:10A1B700E0FCA3E0FD8D828C83EFF0906871E004F2
:10A1C700F07006906870E004F090686BE004F0703F
:10A1D7000690686AE004F0050D80BD90686EE0FFA8
:10A1E700906870E0FCA3E0FD8D828C83EFF09068AF
:10A1F70071E004F07006906870E004F0750D00E5FA
:10A207000DC39403503C90686CE0FEA3E0FF8F827F
:10A217008E83E0FF906870E0FCA3E0FD8D828C8365
:10A22700EFF0906871E004F07006906870E004F059
:10A2370090686DE004F0700690686CE004F0050D1E
:10A2470080BD90686FE0FF906870E0FCA3E0FD8D33
:10A25700828C83EFF0906871E004F070069068706C
:10A26700E004F090686FE0FFEF240EFFAD0FAC0E37
:10A2770012C0418E108F11906870E0FEA3E0FF8F2F
:10A28700828E83E511F0906871E004F070069068A3
:10A2970070E004F0906870E0FEA3E0FF8F828E8389
:0CA2A700E510F090686FE0FFEF2410FF5E
:01A2B3002288
:10971A0090684DEEF0A3EFF090684FECF0A3EDF0F7
:05972A00906851EBF016
:10972F00906854E0FEA3E0FF8E138F14906854E00E
:10973F00FEA3E0FF8F828E837430F0906855E004B3
:10974F00F07006906854E004F0906853E0FFEF600B
:10975F001590660CE0FF906854E0FCA3E0FD8D824D
:10976F008C83EFF0800E906854E0FEA3E0FF8F82B1
:10977F008E83E4F0906855E004F07006906854E032
:10978F0004F0751200E512C39407503C90684DE049
:10979F00FEA3E0FF8F828E83E0FF906854E0FCA36E
:1097AF00E0FD8D828C83EFF0906855E004F0700639
:1097BF00906854E004F090684EE004F070069068F2
:1097CF004DE004F0051280BD906851E0FF906854A1
:1097DF00E0FCA3E0FD8D828C83EFF0906855E004F0
:1097EF00F07006906854E004F0751200E512C3940F
:1097FF0003503C90684FE0FEA3E0FF8F828E83E022
:10980F00FF906854E0FCA3E0FD8D828C83EFF09015
:10981F006855E004F07006906854E004F0906850CA
:10982F00E004F0700690684FE004F0051280BD90E0
:10983F006852E0FF906854E0FCA3E0FD8D828C83BA
:10984F00EFF0906855E004F07006906854E004F073
:10985F00751200906852E0FFE512C39F503C90686C
:10986F0056E0FEA3E0FF8F828E83E0FF906854E006
:10987F00FCA3E0FD8D828C83EFF0906855E004F03F
:10988F007006906854E004F0906857E004F070069A
:10989F00906856E004F0051280B9906852E0FFEF2F
:1098AF00240EFFAD14AC1312C0418E158F169068A5
:1098BF0054E0FEA3E0FF8F828E83E516F09068558B
:1098CF00E004F07006906854E004F0906854E0FEF5
:1098DF00A3E0FF8F828E83E515F0906852E0FFEFD3
:0398EF002410FF43
:0198F2002253
:108722009067FEEFF09067FFECF0A3EDF090680128
:05873200EAF0A3EBF0EA
:10873700906804E0FEA3E0FF906809EEF0A3EFF075
:10874700906804E0FEA3E0FF8F828E837430F09080
:108757006805E004F07006906804E004F090660C89
:10876700E0FF906804E0FCA3E0FD8D828C83EFF0CE
:10877700906805E004F07006906804E004F075174F
:1087870000E517C39407503C9067FFE0FEA3E0FFA6
:108797008F828E83E0FF906804E0FCA3E0FD8D826A
:1087A7008C83EFF0906805E004F07006906804E0B1
:1087B70004F0906800E004F070069067FFE004F0B2
:1087C700051780BD906803E0FF906804E0FCA3E014
:1087D700FD8D828C83EFF0906805E004F0700690C1
:1087E7006804E004F0751700E517C39403503C9044
:1087F7006801E0FEA3E0FF8F828E83E0FF906804AC
:10880700E0FCA3E0FD8D828C83EFF0906805E00427
:10881700F07006906804E004F0906802E004F070DD
:1088270006906801E004F0051780BD906804E0FE3B
:10883700A3E0FF90680DEEF0A3EFF0906805E00469
:10884700F07006906804E004F0751800906806E080
:10885700FBA3E0FAA3E0F97582B0758304128E28B2
:10886700FF9067FEE0FE745F2EF582E4345DF583CA
:10887700EFF0751700E517C3940A40030289AD901E
:108887006806E0FBA3E0FAA3E0F97582B2758304FA
:10889700128E28FFEF702D906806E0FBA3E0FAA385
:1088A700E0F97582B1758304128E28FF9067FEE0A8
:1088B700FE745F2EF582E4345DF583E0FEEE6F70A3
:1088C700030289A8906806E0FBA3E0FAA3E0F97524
:1088D70082B2758304E4128E679067FEE0FF745FCF
:1088E7002FF582E4345DF583E0FF7E0CEF8EF0A474
:1088F700FFAEF0906806E0FBA3E0FAA3E0F9E92FEA
:10890700F9EA3EFAAE02AF0190680FEEF0A3EFF07E
:1089170090680FE0FEA3E0FF90680BEEF0A3EFF086
:10892700751900E519C3940C503C90680BE0FEA341
:10893700E0FF8F828E83E0FF906804E0FCA3E0FDF8
:108947008D828C83EFF0906805E004F070069068E4
:1089570004E004F090680CE004F0700690680BE007
:1089670004F0051980BD740C2518F5189067FEE012
:10897700FF745F2FF582E4345DF583E0FF7E00EF3F
:108987002401FFEE3400FE7C007D64128E9BAF0550
:108997009067FEE0FE745F2EF582E4345DF583EFA9
:1089A700F0051702887C90680DE0FEA3E0FF8F8238
:1089B7008E83E518F0E51870129067FEE0FF74F4F7
:1089C7002FF582E4345DF5837401F09067FEE0FFD4
:1089D70074F82FF582E4345DF5837401F0E518240B
:1089E7000EFF906809E0FCA3E0FD12C0418E1A8FCC
:1089F7001B906804E0FEA3E0FF8F828E83E51BF0E7
:108A0700906805E004F07006906804E004F0906850
:108A170004E0FEA3E0FF8F828E83E51AF0E51824B9
:028A270010FF3E
:018A2900222A
:10C358009062F3E0FFEF6009906643E4F0A3E4F035
:10C36800229065AFE0FFEF70619065D8E0FEA3E032
:10C37800FFEF4E7055906712E0FFEF700890671658
:10C38800E0FFEF70459066A2E0FFEF603D906644E5
:10C39800E004F07006906643E004F0906643E0FE27
:10C3A800A3E0FFC3EF9410EE9427401E906643E489
:10C3B800F0A3E4F09065AF7401F09065DAE4F090D2
:0BC3C80065DC7401F09062F5E4F022E7
:108F5F0000C1814001C0804101C0804100C18140FA
:108F6F0001C0804100C1814000C1814001C08041EA
:108F7F0001C0804100C1814000C1814001C08041DA
:108F8F0000C1814001C0804101C0804100C18140CA
:108F9F0001C0804100C1814000C1814001C08041BA
:108FAF0000C1814001C0804101C0804100C18140AA
:108FBF0000C1814001C0804101C0804100C181409A
:108FCF0001C0804100C1814000C1814001C080418A
:108FDF0001C0804100C1814000C1814001C080417A
:108FEF0000C1814001C0804101C0804100C181406A
:108FFF0000C1814001C0804101C0804100C181405A
:10900F0001C0804100C1814000C1814001C0804149
:10901F0000C1814001C0804101C0804100C1814039
:10902F0001C0804100C1814000C1814001C0804129
:10903F0001C0804100C1814000C1814001C0804119
:10904F0000C1814001C0804101C0804100C1814009
:10905F0000C0C101C30302C2C60607C705C5C404C9
:10906F00CC0C0DCD0FCFCE0E0ACACB0BC90908C839
:10907F00D81819D91BDBDA1A1EDEDF1FDD1D1CDC29
:10908F0014D4D515D71716D6D21213D311D1D01099
:10909F00F03031F133F3F23236F6F737F53534F489
:1090AF003CFCFD3DFF3F3EFEFA3A3BFB39F9F838F9
:1090BF0028E8E929EB2B2AEAEE2E2FEF2DEDEC2CE9
:1090CF00E42425E527E7E62622E2E323E12120E059
:1090DF00A06061A163A3A26266A6A767A56564A449
:1090EF006CACAD6DAF6F6EAEAA6A6BAB69A9A868B9
:1090FF0078B8B979BB7B7ABABE7E7FBF7DBDBC7CA9
:10910F00B47475B577B7B67672B2B373B17170B018
:10911F005090915193535292965657975595945408
:10912F009C5C5D9D5F9F9E5E5A9A9B5B9959589878
:10913F00884849894B8B8A4A4E8E8F4F8D4D4C8C68
:10914F0044848545874746868242438341818040D8
:0300630002B21DC9
:10B21D00C0E0C0F0C083C082C0D075D000C000C0F7
:10B22D0001C002C003C004C005C006C007E5AA30B6
:10B23D00E13753AAFD9062F3E4F09062F2E0FF90E3
:10B24D0063FBE0FEEEC39F501B9063FBE0FF74FABF
:10B25D002FF582E43462F583E0FF8F9A9063FBE073
:10B26D0004F080059062F1E4F0E5AA20E00302B35A
:10B27D003053AAFE9062F37401F09062F57401F000
:10B28D009062F8E0FFEF600302B3309062F0E0FFF0
:10B29D00EFC394FF400302B3309062F0E0FF74FE01
:10B2AD002FF582E43463F583E59AF09062F7E0FFC1
:10B2BD00EF704A9062F0E0FFEF6406704E7E637FA0
:10B2CD00FE7BFF7A0079037C5E7D0390685DECF078
:10B2DD00A3EDF07C5E7D0A90685FECF0A3EDF0903D
:10B2ED0068617407F0129E249062F7EFF09062F798
:10B2FD00E0FFEF70169063FD7401F0800E9063FA1D
:10B30D00E0FFEF70069063FA7401F09062F0E004D4
:10B31D00F09063FDE0FFEF600A9063FDE4F0906252
:10B32D00F0E4F0D007D006D005D004D003D002D081
:0EB33D0001D000D0D0D082D083D0F0D0E0324A
:10CAB0009063FAE0FFEF604B9062F0E0FF9062F667
:10CAC000E0FEEEB507339063FCE0FFEF7035906257
:10CAD000F0E0FF9062F4EFF09063FC7401F090627C
:10CAE000F87401F09062F0E4F09062F6E4F0906285
:10CAF000F7E4F09062F9E4F0229062F0E0FF9062D7
:04CB0000F6EFF0223A
:10CF26009062F0E0FFEF60259062F9E004F0906215
:10CF3600F9E0FFEFD3941440149062F9E4F09062A4
:0ECF4600F6E4F09062F0E4F09062F7E4F0227E
:0DD0350043A60475BABF75AA5043A6102289
:109E2400906858EEF0A3EFF090685AEBF0A3EAF0D4
:039E3400A3E9F0AF
:109E3700906858E0FEA3E0FF786DA60608A60778AD
:109E47006C7600906861E0FF786CE6FEEEC39F5089
:109E57004C90685AE0FBA3E0FAA3E0F9128E0FFFDB
:109E6700906858E0FCA3E0FD8D828C83E0FEEEB5A0
:109E7700071A906859E004F07006906858E004F0FB
:109E870090685BE475F001128EF0800C906861E0D9
:109E9700FFEF04FF786CA607786C0680A6906861D0
:109EA700E0FF786CE6FEEEB507067F0122029FBA57
:109EB700786DE6FE08E6FF906858EEF0A3EFF078BD
:109EC7006C7600906861E0FF786CE6FEEEC39F5009
:109ED7004F90685DE0FEA3E0FF8F828E83E0FF90E6
:109EE7006858E0FCA3E0FD8D828C83E0FEEEB507A9
:109EF7001E906859E004F07006906858E004F090EE
:109F0700685EE004F0700690685DE004F0800C90F5
:109F17006861E0FFEF04FF786CA607786C0680A302
:109F2700906861E0FF786CE6FEEEB507067F0122D8
:109F3700029FBA786DE6FE08E6FF906858EEF0A338
:109F4700EFF0786C7600906861E0FF786CE6FEEEE3
:109F5700C39F504F90685FE0FEA3E0FF8F828E8320
:109F6700E0FF906858E0FCA3E0FD8D828C83E0FE63
:109F7700EEB5071E906859E004F07006906858E047
:109F870004F0906860E004F0700690685FE004F009
:109F9700800C906861E0FFEF04FF786CA607786C8F
:109FA7000680A3906861E0FF786CE6FEEEB50703D4
:059FB7007F01227F0084
:019FBC002282
:108D1900E709F608DFFA8046E709F208DFFA803E3C
:108D290088828C83E709F0A3DFFA8032E309F60829
:108D3900DFFA8078E309F208DFFA807088828C8391
:108D4900E309F0A3DFFA806489828A83E0A3F60845
:108D5900DFFA805889828A83E0A3F208DFFA804C1F
:108D690080D280FA80C680D4806980F280338010F6
:108D790080A680EA809A80A880DA80E280CA80335F
:108D890089828A83ECFAE493A3C8C582C8CCC583D7
:108D9900CCF0A3C8C582C8CCC583CCDFE9DEE780A7
:108DA9000D89828A83E493A3F608DFF9ECFAA9F026
:108DB900EDFB2289828A83ECFAE0A3C8C582C8CC7C
:108DC900C583CCF0A3C8C582C8CCC583CCDFEADE95
:108DD900E880DB89828A83E493A3F208DFF980CCF7
:108DE90088F0EF60010E4E60C388F0ED2402B404F0
:108DF9000050B9F582EB2402B4040050AF23234597
:068E09008223908D6973C5
:108E0F00BB010689828A83E0225002E722BBFE0261
:098E1F00E32289828A83E4932294
:108E2800BB010CE58229F582E5833AF583E02250FF
:108E380006E92582F8E622BBFE06E92582F8E22249
:0D8E4800E58229F582E5833AF583E4932263
:108E5500BB010689828A83F0225002F722BBFE01FC
:028E6500F322F6
:108E6700F8BB010DE58229F582E5833AF583E8F041
:108E7700225006E92582C8F622BBFE05E92582C8ED
:028E8700F222D5
:108E8900EF8DF0A4A8F0CF8CF0A428CE8DF0A42EFD
:028E9900FE22B7
:108E9B00BC000BBE0029EF8DF084FFADF022E4CCBB
:108EAB00F875F008EF2FFFEE33FEEC33FCEE9DEC84
:108EBB00984005FCEE9DFE0FD5F0E9E4CEFD22EDCA
:108ECB00F8F5F0EE8420D21CFEADF075F008EF2F14
:108EDB00FFED33FD4007985006D5F0F222C398FD05
:058EEB000FD5F0EA22A2
:108EF000C5F0F8A3E028F0C5F0F8E582158270020D
:068F00001583E038F022A9
:108F0600EB9FF5F0EA9E42F0E99D42F0EC6480C8E2
:068F160064809845F02282
:108F1C00EB9FF5F0EA9E42F0E99D42F0E89C45F0AB
:018F2C002222
:0C8F2D00ECF0A3EDF0A3EEF0A3EFF022B7
:108F3900D083D082F8E4937012740193700DA3A3C7
:108F490093F8740193F5828883E4737402936860DB
:068F5900EFA3A3A380DFDB
:00000001FF
